:100000000C94BB060C94FF060C94FF060C94FF06A0
:100010000C94FF060C94FF060C94FF060C94FF064C
:100020000C94FF060C945A190C94FF060C94FF06CE
:100030000C94A3330C94FF060C94FF060C94FF065B
:100040000C94FF060C94FF060C9416160C94FF06F5
:100050000C942C0C0C94FF060C94F60B0C94FF06DD
:100060000C94161C0C94FF060C94362F0C94FF066F
:100070000C9471770C94FF060C946D72411C461C15
:100080004B1C541C6B1C821C921CA21CBF1CAB1E64
:10009000821C6D1D7E1DAD1DCB1DE81D421E9D1ECB
:1000A0007B200D21CA214A22B32263236A25C7255A
:1000B00034267E26C92616276727C9272828C2285E
:1000C0005D29572A552F892FCC2F3C30543095303D
:1000D0004C311332133213321332133213321332C0
:1000E0001332133213321332C831CA31CF31E731F0
:1000F000E9310A0D426174743A0020256420436599
:100100006C6C732000204C6F77207761726E696E83
:1001100067206C6576656C3A2025642E2564000A9C
:100120000D466F756E6420424C2D4374726C3A20FC
:10013000002564000A0D0A0D2121204D4953534921
:100140004E4720424C2D4354524C3A2025642021E6
:1001500021000A0D3D3D3D3D3D3D3D3D3D3D3D3D8B
:100160003D3D3D3D3D3D3D3D3D3D3D3D3D3D3D3DBF
:100170003D3D3D3D3D3D3D000A0D43616C69627270
:100180006174696E67207072657373757265207330
:10019000656E736F722E2E004F4B0A0D000A0D46CE
:1001A0006C696768742D74696D65202575206D69AB
:1001B0006E2020546F74616C3A2575206D696E0055
:1001C0000A0D436F6E74726F6C3A2000486561646B
:1001D000696E67486F6C64004E6F726D616C2028A9
:1001E0004143432D4D6F646529000A0D3D3D3D3D62
:1001F0003D3D3D3D3D3D3D3D3D3D3D3D3D3D3D3D2F
:100200003D3D3D3D3D3D3D3D3D3D3D3D3D3D3D0A51
:100210000D00416E676C654E69636B2020202020C5
:100220002020416E676C65526F6C6C20202020206E
:1002300020204163634E69636B2020202020202012
:100240002020416363526F6C6C20202020202020EE
:1002500020205961774779726F20202020202020AC
:1002600020204865696768742056616C7565202098
:1002700020204163635A202020202020202020209D
:1002800020204761732020202020202020202020B3
:100290002020436F6D706173732056616C7565200B
:1002A0002020566F6C74616765205B302E31565D7F
:1002B00020205265636569766572204C6576656CB1
:1002C00020204779726F20436F6D70617373202017
:1002D00020204D6F746F722031202020202020209C
:1002E00020204D6F746F722032202020202020208B
:1002F00020204D6F746F722033202020202020207A
:1003000020204D6F746F7220342020202020202068
:1003100020203136202020202020202020202020B6
:1003200020203137202020202020202020202020A5
:100330002020313820202020202020202020202094
:100340002020313920202020202020202020202083
:100350002020536572766F2020202020202020202E
:100360002020486F7665726761732020202020204E
:10037000202043757272656E74205B302E31415DB2
:1003800020204361706163697479205B6D41685D11
:100390002020486967687420536574706F696E74B3
:1003A0002020323520202020202020202020202026
:1003B0002020323620202020202020202020202015
:1003C0002020436F6D7061737320536574706F6983
:1003D0006E744932432D4572726F722020202020A6
:1003E0002020424C204C696D697420202020202060
:1003F00020204750535F4E69636B2020202020202F
:1004000020204750535F526F6C6C2020202020200A
:10041000202021212120494E434F4D504154494233
:100420004C4520212121002E000A0D20444143206B
:100430006F7220493243204552524F522120436867
:1004400065636B204932432C2033567265662C203D
:1004500044414320616E6420424C2D4374726C0011
:100460005B25695D005B25695D002B204D696B7222
:100470006F4B6F70746572202B0048573A56256495
:100480002E25642053573A25642E25642563005396
:10049000657474696E673A2564202573004861723B
:1004A0006477617265204572726F7220313A2564FB
:1004B000202121004D697373696E6720424C2D43E2
:1004C00074726C3A25642121004D6978657220456B
:1004D00072726F722100493243204552524F5221AD
:1004E0002121004865696768743A20202535690034
:1004F000536574706F696E743A2535690050726582
:1005000073737572653A253569004F666673657455
:100510003A20202535690048656967687420636F53
:100520006E74726F6C0044495341424C454400481C
:10053000656967687420636F6E74726F6C004449FC
:100540005341424C4544006163742E2062656172E0
:10055000696E67004E69636B3A20202020202025B9
:10056000356900526F6C6C3A202020202020253500
:100570006900436F6D706173733A202020253569DF
:10058000004B313A25346920204B323A253469201A
:10059000004B333A25346920204B343A2534692006
:1005A000004B353A25346920204B363A25346920F2
:1005B000004B373A25346920204B383A25346920DE
:1005C000004E693A2534692020526F3A253469205B
:1005D0000047733A253469202047693A2534692059
:1005E0000050313A253469202050323A25346920B0
:1005F0000050333A253469202050343A253469209C
:10060000004779726F202D2053656E736F72004E14
:1006100069636B25346920282533692E25692900F3
:10062000526F6C6C25346920282533692E25692981
:100630000047696572253469202825336929004EF1
:1006400069636B2025346920282533692E25782994
:1006500000526F6C6C2025346920282533692E25C3
:1006600078290059617720202534692028253369AD
:1006700029004E69636B20253469202825336929B8
:10068000282533692900526F6C6C20253469202895
:1006900025336929282533692900596177202025C8
:1006A00034692028253369292825336929004143E5
:1006B00043202D2053656E736F72004E69636B206B
:1006C00025346920282533692900526F6C6C202558
:1006D0003469202825336929005A20202020253418
:1006E0006920282533692900566F6C746167653A63
:1006F0002020202533692E253169560043757272FA
:10070000656E743A2020202533692E253169410019
:10071000506F7765723A20202020202534695700D9
:100720004469736368617267653A202535696D4174
:10073000680052656365697665720052432D5253B5
:1007400053493A202020202534690052432D517509
:10075000616C6974793A202534690052432D4368ED
:10076000616E6E656C733A25346900436F6D70611C
:1007700073730048656164696E673A2020253569A6
:100780000056616C75653A2020202025356900539C
:100790006F6C6C3A202020202025356900506F7442
:1007A00069313A202025336900506F7469323A204C
:1007B0002025336900506F7469333A20202533694E
:1007C00000506F7469343A202025336900506F74EB
:1007D00069353A202025336900506F7469363A2014
:1007E0002025336900506F7469373A20202533691A
:1007F00000506F7469383A202025336900536572C0
:10080000766F202000536574706F696E7420202508
:10081000336900506F736974696F6E3A20253369CC
:100820000052616E67653A2533692D2533690045AD
:10083000787465726E436F6E74726F6C2020004E18
:10084000693A2534692020526F3A253469200047DF
:10085000733A253469202047693A253469200048D5
:10086000693A253469202043663A253469200042DC
:100870004C2D4374726C204572726F727320002588
:10088000336420253364202533642025336420001D
:1008900025336420253364202533642025336420E8
:1008A00000253364202533642025336420253364F8
:1008B0002000424C2054656D7065726174757265DC
:1008C00000253369202533692025336920253369C4
:1008D00020002533692025336920253369202533FD
:1008E00069200025336920253369202533692025B7
:1008F00033692000424C2D4374726C20666F756E14
:1009000064200020256320202025632020202563EB
:10091000202020256320002025632020202563201F
:10092000202025632020202563200020256320200F
:10093000202D2020202D2020202D2000313000319E
:100940003100313200466C696768742D54696D65F9
:10095000202000546F74616C3A2535756D696E0006
:100960004163743A20202535756D696E00287265E3
:1009700073657429000A0D47656E65726174696E4E
:10098000672064656661756C7420506172616D6585
:1009900074657220536574202564000A0D557369CF
:1009A0006E6720506172616D657465722053657465
:1009B000202564000A0D47656E65726174696E6773
:1009C0002064656661756C74204D69786572205489
:1009D00061626C65000A0D4D697865722D436F6E1A
:1009E0006669673A202725732720282575204D6FD3
:1009F000746F727329000A0D3D3D3D3D3D3D3D3D07
:100A00003D3D3D3D3D3D3D3D3D3D3D3D3D3D3D3D16
:100A10003D3D3D3D3D3D000A0D414343206E6F7419
:100A20002063616C69627261746564210D0A000063
:100A3000008F001E01AD013B02CA025803E6037499
:100A40000402058F051B06A7063307BE074808D218
:100A5000085B09E3096B0AF20A780BFD0B810C04B1
:100A60000D860D070E870E060F840F00107B10F504
:100A7000106E11E5115B12CF124213B313231492BF
:100A800014FE146A15D3153B16A11605176717C86F
:100A90001727188318DE1837198E19E319361A87A5
:100AA0001AD61A231B6E1BB61BFD1B411C831CC3CD
:100AB0001C001D3C1D751DAB1DE01D121E421E6F4E
:100AC0001E9A1EC31EE91E0D1F2E1F4D1F691F8477
:100AD0001F9B1FB01FC31FD31FE11FEC1FF51FFB80
:100AE0001FFF1F002003010000BB6B00020101AECD
:100AF0006C01030202426D020003039F6D253269FF
:100B00002E25316956002533642563202530336452
:100B10006D00537461747573004552524F523A2000
:100B200025326400253469202532693A253032693E
:100B3000002534696D25630025336920253369203C
:100B40002533692025336900253369202533692041
:100B5000253369202533690054656D7065726174B1
:100B600075726573202020200025634320202020FB
:100B700020002532692E2531695620202533692E23
:100B8000253169410025346957202536696D416852
:100B9000002532756D2F73205361743A256420004F
:100BA00020203344004E6F4678004447505300489D
:100BB0006F6D653A2533646D202533642563004EDF
:100BC0006F204E6176694374726C21000A0D77774D
:100BD000772E4D696B726F4B6F707465722E646502
:100BE0002028632920486953797374656D73204701
:100BF0006D6248000A0D74686520757365206F6624
:100C0000207468697320736F6674776172652069F8
:100C100073206F6E6C79207065726D697474656491
:100C2000200A0D6F6E206F726967696E616C204DCE
:100C3000696B726F4B6F707465722D486172647767
:100C4000617265004143542044534C004A65746905
:100C500020736174656C6C6974005370656B747299
:100C6000756D20736174656C6C697420284C6F77A6
:100C7000207265736F6C7574696F6E2900537065AF
:100C80006B7472756D20736174656C6C6974202867
:100C90003230343829005370656B7472756D20736F
:100CA0006174656C6C6974004D756C746973696707
:100CB0006E616C2050504D000A0D52656365697677
:100CC00065723A2000756E6B6E6F776E2E205573CD
:100CD000696E672050504D2E2E2E006E6F7420735B
:100CE0007570706F727465642062792068617264D7
:100CF0007761726521000A0D3D3D3D3D3D3D3D3D25
:100D00003D3D3D3D3D3D3D3D3D3D3D3D3D3D3D3D13
:100D10003D3D3D3D3D3D3D3D3D3D3D000A0D466C6B
:100D200069676874436F6E74726F6C0A0D48617204
:100D300064776172653A25642E25640A0D536F66E7
:100D400074776172653A5625642E25642563200008
:100D50000A0D3D3D3D3D3D3D3D3D3D3D3D3D3D3D26
:100D60003D3D3D3D3D3D3D3D3D3D3D3D3D3D3D3DB3
:100D70003D3D3D3D3D0011241FBECFEFD0E1DEBF24
:100D8000CDBF11E0A0E0B1E0E4E1F3EF02C00590D7
:100D90000D92AC3FB107D9F718E0ACEFB1E001C05C
:100DA0001D92AC3DB107E1F76AEAE2E0F0E081E2D2
:100DB000809357007491AE014F5F5F4F20EF37EF84
:100DC000DA019FE0F9012F5F3F4F84918D9391509D
:100DD00097FFF8CF773911F40000FECFFA019EE0BB
:100DE000819168276095915097FFFACF888968179D
:100DF00021F0773911F40000FECF0C94C0070C9459
:100E0000000080913306E82FFF27EE0FFF1FE35A03
:100E1000F84F808191818D5E9F4F14F010920301F5
:100E2000808191818A5B9F4FCCF48091030188235C
:100E3000A9F481E080930301809176048F5F809311
:100E40007604853038F088EE93E0909330028093FA
:100E50002F0204C066E970E00E9429378091760471
:100E60009927909304068093030608951F93CF93C8
:100E7000DF93182F882389F082EF90E09F938F9360
:100E80008BEF92E19F938F93E0914204F0914304A2
:100E900009950F900F900F900F9080915606823316
:100EA00008F044C084EF91E00E942117EC01112367
:100EB00029F0CE010E942A178823D9F3C2E0D0E09E
:100EC00026E530E080911E0190911F018217930763
:100ED00030F02196255D3F4FC730D10598F38091C2
:100EE00056069927C89F9001C99F300DD89F300D95
:100EF0001124209300011123D9F068EC70E08C2FAD
:100F00000E942937DF93CF938AEF90E09F938F93CE
:100F10008BEF92E19F938F93E0914204F091430411
:100F200009958DB79EB706968DBF02C080930001CC
:100F3000112311F1809100016AE00E94B578892F98
:100F400099279F938F93809100010E94B5789927EC
:100F50009F938F9385E091E09F938F938BEF92E126
:100F60009F938F93E0914204F091430409952DB72C
:100F70003EB7285F3F4F2DBFDF91CF911F9108955E
:100F8000CFEFD0E1DEBFCDBF8824992414B815B8C7
:100F900007EE13E00253104017FFFCCF189B06C06A
:100FA000199B02C08DE007C08BE005C0199B02C0F1
:100FB00084E101C08AE08093020181E887B93E9A0A
:100FC0008FEF88B98BE184B981E085B98EE38AB966
:100FD00087E48BB9469A84B7877F84BF809160008D
:100FE0008861809360001092600084EC99E0909397
:100FF000300280932F0210922B0310922A0310923A
:1010000062071092610710922D0310922C03109228
:101010002F0310922E0320910201243128F084EC3A
:1010200094E0A0E0B0E004C08BE095E0A0E0B0E088
:1010300080939A0190939B01A0939C01B0939D0192
:101040002A3011F0243110F0289801C0289A0E940B
:101050008A170E945B170E9403130E9487330E9425
:10106000CE1A81E00E94EA2E0E94E9630E948E6EF1
:101070000E94A476809102018C3010F4299A01C05C
:10108000299878940E94092E80917702826080933B
:10109000770210927A020E94544284EF91E00E94FB
:1010A00021178C018091770280FD05C0C8010E9444
:1010B0002A178823B9F38FE191E09F938F93BBEFB9
:1010C000AB2EB2E1BB2EBF92AF92E0914204F09101
:1010D0004304099580EA9FE00E9421178C01C0E03B
:1010E000D0E00F900F900F900F90AFEFEA2EA6E098
:1010F000FA2EF3EBCF2EF6E0DF2E0E9454428091C1
:10110000770280FD05C0C8010E942A178823B9F321
:10111000F60180811816ACF40BC00E9454428091F5
:10112000770280FD05C0C8010E942A178823B9F301
:10113000C8010E942A17882321F4F701808188239F
:1011400064F7F701808187FF18C02196DF93CF9362
:10115000219781E391E09F938F93BF92AF92E091AB
:101160004204F091430409958091FD018F5F8093C3
:10117000FD018DB79EB706968DBF2196E4E0F0E0A5
:10118000CE0EDF1E88E090E0E80EF91ECC30D105CF
:1011900008F4B3CFC0E0D0E00CEF16E0E3EBEE2EA6
:1011A000E6E0FE2EF801838187FD1CC0F7018081F7
:1011B0001816C4F42196DF93CF93219784E391E02E
:1011C0009F938F938BEF92E19F938F93E0914204D3
:1011D000F0914304099582E080932D028DB79EB76C
:1011E00006968DBFF801838180788383219684E001
:1011F00090E0E80EF91E085F1F4FCC30D10590F249
:1012000082E591E09F938F93CBEFD2E1DF93CF9371
:10121000E0914204F0914304099590913106809148
:10122000FD010F900F900F900F90981728F4809168
:101230005C04806180935C0488E791E09F938F93C6
:10124000DF93CF93E0914204F0914304099588EE37
:1012500093E00E9421178C010E94D41A0F900F90E6
:101260000F900F90C8010E942A178823D9F388E9AC
:1012700091E09F938F93DF93CF93E0914204F0919D
:101280004304099580E00E94EB37809102010F90A2
:101290000F900F900F908A3011F0843110F0289841
:1012A00001C0289A80ED97E09093300280932F023E
:1012B00085E5809378048EE090E00E949B2C99272E
:1012C000182F00278FE090E00E949B2C080F111D23
:1012D00010930302009302028AE090E00E949B2C8C
:1012E0009927182F00278BE090E00E949B2C080F75
:1012F000111D10930102009300020F5F1F4F39F080
:1013000080910202909103028F5F9F4F41F41092EF
:1013100003021092020210920102109200028091C8
:101320000002909101029F938F938091020290910D
:1013300003029F938F938DE991E09F938F93DF93A7
:10134000CF93E0914204F091430409958DB79EB785
:1013500008968DBF80EC91E09F938F93DF93CF939E
:10136000E0914204F0914304099580913F060F906B
:101370000F900F900F90E0914204F091430482FF90
:1013800007C08CEC91E09F938F93DF93CF9308C0BD
:1013900088ED91E09F938F938BEF92E19F938F93D2
:1013A00009950F900F900F900F900E94F21F88E800
:1013B00093E1909393018093920181E0809377046D
:1013C0000E943607809159060E940A768AEE91E0C3
:1013D0009F938F93DF93CF93E0914204F091430466
:1013E000099580ED97E00E9421178C018AEF90E02B
:1013F0000E942117EC0183E08093DB051092FC0131
:101400000F900F900F900F90809105028111FFCFE8
:10141000CE010E942A17882339F084E690E00E94CA
:101420002117EC010E94607780913302882309F430
:10143000D5C180911001882309F4D0C110923302E4
:1014400080917604882319F00E94010702C00E944F
:1014500070450E945442209102012A3011F024313B
:1014600010F0289801C0289A8091300390915C0474
:10147000882339F080913003815080933003977F27
:101480000AC080916F00806280936F0010925E07A7
:1014900010925D07986090935C0480919201909106
:1014A000930101979093930180939201809192010F
:1014B00090919301892B21F0809178028823C9F1C2
:1014C0008091920190919301892BD9F40E94142F5D
:1014D00085E090E0909393018093920180911506AE
:1014E00090911606019690931606809315068091AA
:1014F0005C04816080935C048091DC058260809351
:10150000DC0580910801909109018F5F9F4F19F5CB
:10151000809127038823F9F080E197E290933002CD
:1015200080932F0280E890E0909309018093080156
:1015300012C02A3011F0243110F0289801C0289AE6
:1015400080912F0290913002892B29F480915C04C4
:101550008E7F80935C0480913302882309F03EC122
:1015600080910E01882311F00E94A1170E9446135A
:101570000E947C0EC8010E942A17882309F42AC100
:101580000C5E1F4F8091780290915C04882339F0A3
:10159000926090935C048091DC0582600CC09D7F1A
:1015A00090935C048091920190919301079728F0A9
:1015B0008091DC058D7F8093DC0580919201909174
:1015C0009301079728F080915C048E7F80935C04E0
:1015D00080910501882321F081508093050125C069
:1015E0008093820410920103109200031092FF0274
:1015F0001092FE021092FD021092FC0280910801EE
:10160000909109018F5F9F4F81F48091300388236F
:1016100061F488E99AE39093300280932F0280E08E
:101620009CE090930901809308018091F201893C2C
:1016300048F081508093F20180915C048B7F80930D
:101640005C0430C080913B088823E1F080915C0409
:10165000846080935C0480910801909109018F5F00
:101660009F4F81F480912703882361F088E99AE3F2
:101670009093300280932F0280E098EA90930901C2
:101680008093080110920C0410920B0410920A042B
:10169000109209048FEF9FEF90936B0880936A0874
:1016A0001092F20180910001282F332780911E01B2
:1016B00090911F0182179307CCF48091F50280620C
:1016C0008093F50280910801909109018F5F9F4FEF
:1016D000C1F480E797E19093300280932F0280E07D
:1016E00093E090930901809308010BC080912F0231
:1016F00090913002892B29F48091F5028F7D80939F
:10170000F5020E946F6884E080932E028091270387
:10171000882329F45AEA852E55E0952E12C080912F
:1017200004028F5F80930402813359F41092040203
:101730008091FE019091FF0101969093FF018093AB
:10174000FE010894811C911CF2E78F16FBE09F06B6
:1017500009F040C0882499242091020230910302AC
:101760002F5F3F4F309303022093020280910002CB
:101770009091010201969093010280930002832FC1
:101780009927682F8EE090E00E94A12C80910202A0
:10179000909103029070682F8FE090E00E94A12C3E
:1017A0008091000290910102892F9927682F8AE089
:1017B00090E00E94A12C8091000290910102907013
:1017C000682F8BE090E00E94A12C84E190E00E94C1
:1017D00021178C010E94BF680E94A56E80912E0285
:1017E000882309F011CE0E940A640ECE1F920F9238
:1017F0000FB60F9211248F939F93EF93FF938091D5
:1018000007018823E1F480911F0290912002019644
:101810009093200280931F02FC01EF5CFA4FE0815D
:10182000ED3019F08A3A910539F4109220021092A5
:101830001F0281E080930701E093C60004C010926C
:10184000200210921F02FF91EF919F918F910F90B4
:101850000FBE0F901F9018951F920F920FB60F9208
:1018600011242F933F934F935F936F937F938F93A5
:101870009F93AF93BF93CF93EF93FF9390E08091AB
:101880000502813029F48091C6008093CE00CCC03F
:1018900080910502823029F48091C60080938504EE
:1018A000C3C08091C60080931702509125025A3A16
:1018B00010F090932602809117028D3009F065C0D8
:1018C00080912602823009F060C090932602852F15
:1018D00099278B579B4FFC01329740812091210221
:1018E00030912202241B3109DC0111978C91281BB5
:1018F0003109C9019F70909322028093210246E032
:10190000969587954A95E1F7982F935C90932302DB
:101910002F733070235C209324028081981729F460
:101920008C91281711F491E006C090E08091140288
:101930008F5F80931402C0911602CC2309F074C00B
:10194000992309F471C081E080931602580F5093D7
:1019500013025150E52FFF27EB57FB4F8DE080839B
:1019600080918704823509F05FC00E94F21F88E1F0
:1019700090E02CE00FB6F894A895809360000FBE1D
:1019800020936000C0932D024FC020912602822F29
:10199000992781309105F9F0823091051CF4892B4B
:1019A00021F040C0029711F13DC0809117028332AF
:1019B00039F480911602882319F481E0809326027D
:1019C000809117028093850481E0809325028091A5
:1019D0001702992722C02F5F20932602E52FFF27A9
:1019E000EB57FB4F80911702808309C0E52FFF273B
:1019F000EB57FB4F8091170280835A3A20F45F5FC8
:101A00005093250202C01092260220911702809165
:101A1000210290912202820F911D909322028093C5
:101A2000210202C010922602FF91EF91CF91BF9147
:101A3000AF919F918F917F916F915F914F913F9166
:101A40002F910F900FBE0F901F901895AC01A0E042
:101A5000B0E09D01A817B90748F4E1E3F5E08191F2
:101A6000280F311D1196A417B507C8F33F70FD016B
:101A7000EF5CFA4FC90156E0969587955A95E1F7C4
:101A8000835C80831196FD01EF5CFA4F2F733070F9
:101A9000822F835C8083AE5CBA4F8DE08C93109272
:101AA0000701809131058093C6000895A0E0B0E061
:101AB000ECE5FDE00C942E792C859D850E85BB24EC
:101AC00083E2809331059F5990933205209333052B
:101AD00033E0E32EF12C002309F49EC0CF84D88894
:101AE000BE016D5E7F4FA989BA890150109709F434
:101AF00093C01097B9F0F601EB0DF11DB3949081EE
:101B0000119791F4002349F1FB016E5F7F4FDB01D8
:101B1000C080D1806E5F7F4F0D90BC91A02DBB2403
:101B2000015002C090E019C01097B9F0F601EB0D1A
:101B3000F11DB3944081119791F4002341F1FB0111
:101B40006E5F7F4FDB01C080D1806E5F7F4F0D9055
:101B5000BC91A02DBB24015002C040E018C01097DA
:101B6000B1F0F601EB0DF11DB3941081119781F4E2
:101B7000002371F0FB013296DB01CD90DC90BF01B8
:101B80006E5F7F4FA081B181BB24015001C010E086
:101B9000F701EF5CFA4F892F86958695835C8083E9
:101BA0000894E11CF11CF701EF5CFA4F892F99278B
:101BB0008370907024E0880F991F2A95E1F75527CC
:101BC0009A0194E0369527959A95E1F7822B835CEC
:101BD00080830894E11CF11CF701EF5CFA4F4F7011
:101BE0005070440F551F440F551F812F992726E031
:101BF000969587952A95E1F7842B835C80830894DA
:101C0000E11CF11CF701EF5CFA4F1F73135C1083AA
:101C10000894E11CF11C6ACFC7010E94260DE9E07F
:101C20000C944A79A3E07A2F409113024650442342
:101C300009F458C0E72FFF27EB57FB4F80818D53E6
:101C40007F5FE72FFF27EB57FB4F20812D537F5FEF
:101C5000E72FFF27EB57FB4F30813D537F5FE72F87
:101C6000FF27EB57FB4F60816D537F5F9927880FEC
:101C7000991F880F991F522F52955F70582B822FF2
:101C800099278F709070F4E0880F991FFA95E1F70B
:101C9000232F26952695282B832F992783709070C4
:101CA000E6E0880F991FEA95E1F7682B41504F3F16
:101CB000C9F0EA2FFF27EB57FB4F5083AF5F41502E
:101CC0004F3F81F0EA2FFF27EB57FB4F2083AF5F99
:101CD00041504F3F39F0EA2FFF27EB57FB4F60830E
:101CE000AF5FA5CF88E894E0909312028093110231
:101CF000A350A09310020895A2E0B0E0E2E8FEE055
:101D00000C94347980911602882309F470C40E94DF
:101D1000120E80918604823609F02AC380918704CE
:101D200099278037910509F4C1C081379105C4F422
:101D30008A36910509F492C28B36910544F48B34AE
:101D4000910571F18636910509F471C111C38D3683
:101D5000910509F47BC08E36910509F45FC008C374
:101D600084379105D1F1853791054CF48137910580
:101D700009F4A3C08337910509F4F1C0F9C287378C
:101D8000910509F42DC2883791052CF4853791050A
:101D900009F4E9C1EDC28937910509F47FC1E8C2B0
:101DA000E0911102F0911202808191819093E30100
:101DB0008093E2012091400330914103821B930BF9
:101DC000845E9D4F68E671E00E94D578845B904008
:101DD00090933F0380933E03CBC280911302A09166
:101DE0001102B0911202853140F080E1E0E6F4E0AA
:101DF0000D9001928A95E1F70DC08D919D910D9006
:101E0000BC91A02D8093600490936104A093620420
:101E1000B093630480EF80930E024BC08091070162
:101E20008823E1F38DE490E09F938F9386EA96E018
:101E30009F938F9381E08F938F938EE48F930E9473
:101E4000560D8DB79EB707968DBF92C2A091110215
:101E5000B09112021C91113081F48DE4E6EAF6E0B3
:101E60000D9001928A95E1F70E94582D1983809177
:101E70005C048F7E80935C0401C01982809107010D
:101E80008823E1F381E090E09F938F93CE01019648
:101E90009F938F9381E08F938F938DE48F930E9414
:101EA000560DADB7BEB71796ADBF62C281E0809345
:101EB00019028FEF809305015BC2E0911102F0914E
:101EC0001202E0818E2F8A508A3058F48983882349
:101ED00011F481E003C0863010F085E0898361E071
:101EE0000EC08E2F84518A3070F48983882311F4B8
:101EF00081E003C0863010F085E0898360E089814D
:101F00000E94CC2D12C0E983EF3F19F40E94BD2D31
:101F100089838981882311F481E003C0863010F021
:101F200085E0898389810E94B02C809107018823F4
:101F3000E1F383E790E09F938F9382E396E09F9392
:101F40008F9381E090E09F938F93CE0101969F93B2
:101F50008F9382E08F9381E08F9381E577C1209109
:101F6000110230911202D9018C918150853008F014
:101F700045C0F9018181853509F040C08091270372
:101F80008823E1F52F5F3F4F83E7E2E3F6E0D901D5
:101F90000D9001928A95E1F7F90182910E94F42C4B
:101FA000809173069927AA27BB27BC01CD0124EC99
:101FB00039E040E050E00E949678DC01CB0180934C
:101FC000DA019093DB01A093DC01B093DD018091F5
:101FD00074069927AA27BB27BC01CD010E949678D9
:101FE000DC01CB018093D6019093D701A093D80157
:101FF000B093D9010E94BD2D898301C019828091BF
:1020000007018823E1F381E090E09F938F93CE0155
:1020100001969F938F9381E08F938F9383E58F93A6
:102020000E94560D8DB79EB707968DBF26C0E091D2
:102030001102F0911202E0818E2F8150853018F448
:102040008E2F0E94B02C0E94BD2D898380910701A4
:102050008823E1F381E090E09F938F93CE01019676
:102060009F938F9381E08F938F9386E48F930E9449
:10207000560DADB7BEB71796ADBF80912703882325
:1020800029F46EE670E089810E94293780E00E9481
:102090003607809159060E940A766AC1E0911102C2
:1020A000F09112028081992787FD9095909378078F
:1020B000809377078181992787FD909590937A0780
:1020C000809379078281992787FD909590937C076B
:1020D00080937B078381992787FD909590937E0756
:1020E00080937D078481992787FD90959093800741
:1020F00080937F078581992787FD9095909382072C
:10210000809381078681992787FD90959093840716
:10211000809383078781992787FD90959093860701
:10212000809385078085992787FD909590938807F0
:10213000809387078185992787FD909590938A07DB
:10214000809389078285992787FD909590938C07C6
:1021500080938B078385992787FD909590938E07B1
:1021600080938D0705C1E0911102F09112028081E8
:102170000E94E0328A83882319F481E0898301C0B8
:102180001982809107018823E1F388E090E09F9312
:102190008F9384EF96E09F938F9321E030E03F93FD
:1021A0002F9380911102909112029F938F933F93EE
:1021B0002F93CE0102969F938F933F932F93CE013F
:1021C000820F931F9F938F9384E08F9381E08F936F
:1021D00085E58F930E94560DEDB7FEB773963CC010
:1021E00080911002893008F4C3C02091110230910F
:1021F00012022F5F3F4F88E0A4EFB6E0F901019093
:102200000D928A95E1F7D9018E910E9436328A8328
:10221000882319F481E0898301C019828091070124
:102220008823E1F321E030E03F932F93CE01029623
:102230009F938F933F932F93CE01820F931F9F9372
:102240008F9382E08F9381E08F9387E58F930E9435
:10225000560DEDB7FEB73B96EDBF8AC00E94BD7527
:102260008983823019F0843009F082C0F89480911B
:10227000C1008F738093C1008091C9008F738093D8
:10228000C9008091C100877E8093C1008091C90000
:10229000877E8093C9008091C80087FF03C080912A
:1022A000CE00F9CF8091C00087FF03C08091C600A7
:1022B000F9CFE0911102F09112028081882359F543
:1022C00081E0809305021092CD0080E490E080933D
:1022D000CC008091CD008093C5008091CC0080938C
:1022E000C4008091CA008F7D8093CA008091CA008B
:1022F0008F7E8093CA008091C9008B7F8093C90034
:102300008091CA0084608093CA008091CA00826074
:102310008093CA0003C082E0809305028091CA00C6
:10232000877F8093CA008091C200877F8093C2001C
:102330008091C9008E7F8093C9008091C10088611F
:102340008093C1008091C90088618093C900809109
:10235000C10080688093C1008091C900806880932B
:10236000C90010926E0010926F0010927000789465
:102370008091870499278436910509F4CDC085366C
:102380009105ACF48136910509F481C0823691053E
:102390002CF48B34910509F45DC021C1823691057E
:1023A00009F482C08336910509F491C018C18C36B6
:1023B000910509F4FFC08D3691054CF487369105DF
:1023C00009F40AC18836910509F4C4C008C18437EC
:1023D000910529F08637910509F4FAC000C1809172
:1023E0001302A0911102B0911202803140F080E1FD
:1023F000E0E6F4E00D9001928A95E1F70DC08D9131
:102400009D910D90BC91A02D8093600490936104E8
:10241000A0936204B0936304809107018823E1F3E1
:102420001F92809104018F9384E58F930E94560D33
:102430008AEF80930E028FEF8093050180EA9FE080
:102440000E94211790930702809306020F900F902D
:102450000F90C5C0E0911102F0911202808191812C
:102460009093E3018093E201209140033091410376
:10247000821B930B845E9D4F68E671E00E94D578C5
:10248000845B904090933F0380933E03A8C0E0910B
:102490001102F0911202808180930601803298F03F
:1024A0008FE1809306010FC0A0911102B09112023A
:1024B0008BE0E8E7F4E00D9001928A95E1F78091D6
:1024C000810480931D068FEF8093050188C0809161
:1024D0000A0290910B02892B89F4E0911102F0918C
:1024E0001202E081EE2351F08AE0E89FC00111243E
:1024F0000E9421179093530480935204E09111029B
:10250000F091120290818AE0989FC001112490936B
:102510000B0280930A0215C08FEF80930501E091B2
:102520001102F091120290818AE0989FC00111245B
:1025300090930D0280930C02892B19F081E0809317
:102540001B0280EA9FE00E9421179093070280936C
:10255000060245C08FEF80930501E0911102F091D2
:102560001202908197FD08C082E0809318021092B9
:102570000902109208021AC0909580917002892B6E
:102580008093700291818AE0989FC00111249093FA
:1025900009028093080284E08093180280EA9FE099
:1025A0000E942117909307028093060281E0809396
:1025B0001C0215C08FEF80930501E0911102F0918C
:1025C000120280818093710281E080931D0207C016
:1025D00081E080931A0203C081E080931E02109272
:1025E0001602109212021092110210921002E3E0F1
:1025F000CE5F0C945079982F8091C00085FFFCCF5E
:102600009093C60008950F931F9388E18093C100B3
:102610008091C00082608093C0008091C10080687A
:102620008093C1008091C10080648093C10000E06C
:1026300010E00093C5008AE290E08093C40080918E
:102640000C0290910D020E942117909355048093E3
:1026500054048CED90E00E942117909384048093A1
:1026600083041092560484E58093570410925A0410
:102670008BE0809358041092590410931202009337
:102680001102109210021F910F910895A0E1B0E085
:10269000ECE4F3E10C94317980910701882309F48B
:1026A000C1C280910602909107020E942A178823D6
:1026B00061F0109209021092080210920D0210921D
:1026C0000C0210920B0210920A0280910802909163
:1026D0000902892B41F080912F05909130050E94CD
:1026E0002A17882329F480911C02882309F460C0EA
:1026F00080910701882309F45BC08091180201E2F0
:1027000011E08430A8F00E94062080E590E09F93BD
:102710008F931F930F9381E08F938F9388E48F9310
:102720000E94560D2DB73EB7295F3F4F2DBF34C0D5
:102730001092720282E194E09F938F938BEF9FE15E
:102740009F938F93E0914204F0914304099584E1B3
:1027500090E09F938F931F930F9381E090E09F935E
:102760008F9388E192E09F938F9382E08F9381E033
:102770008F9388E48F930E94560D80911802982FB2
:102780008F5F809318022DB73EB7215F3F4F2DBF5B
:10279000943010F010921802809108029091090272
:1027A0000E9421179093300580932F0510921C02F0
:1027B00080911D02882351F180910701882331F116
:1027C0000E94062080E590E09F938F9381E291E044
:1027D0009F938F9321E030E03F932F9380E291E02D
:1027E0009F938F933F932F9381E792E09F938F93D3
:1027F00083E08F9381E08F938CE48F930E94560D3A
:1028000010921D028DB79EB70F968DBF80911A0250
:102810008823D1F0809107018823B1F08AE090E00D
:102820009F938F9386E594E09F938F9381E08F939E
:102830008F9386E58F930E94560D10921A022DB742
:102840003EB7295F3F4F2DBF80911E028823D9F0EC
:10285000809107018823B9F08BE090E09F938F93DC
:1028600088E794E09F938F9381E08F938091040198
:102870008F9387E48F930E94560D10921E028DB79E
:102880009EB707968DBF80918304909184040E9427
:102890002A17882309F461C080910701882309F46D
:1028A0005CC080914E069927880F991F880F991F49
:1028B0007C010027F7FC0095102F809182039091F6
:1028C0008303A0918403B0918503BC01CD01A801CD
:1028D00097010E940A7930937104209370048091CB
:1028E0007A0390917B03A0917C03B0917D03BC019E
:1028F000CD01A80197010E940A79309373042093B7
:10290000720480910A038093740480910903809378
:10291000750488E090E09F938F9380E794E09F9305
:102920008F9381E08F9383E08F938BE68F930E9448
:10293000560D809176042DB73EB7295F3F4F2DBFCE
:10294000853018F086E08093760483E690E00E945C
:102950002117909384048093830480910C029091BA
:102960000D02892B41F080915404909155040E94EE
:102970002A17882321F480911B02882339F1809142
:102980000701882319F10E94033682E490E09F93A7
:102990008F938BED95E09F938F9381E08F938F932F
:1029A00084E48F930E94560D10921B028DB79EB740
:1029B00007968DBF80910C0290910D02009731F027
:1029C0000E942117909355048093540480910A0229
:1029D00090910B02892B09F4B8C080915204909118
:1029E00053040E942A17882309F4AFC0809107017D
:1029F000882309F4AAC080914E069927880F991F51
:102A0000880F991F7C010027F7FC0095102F8091FB
:102A1000820390918303A0918403B0918503BC014C
:102A2000CD01A80197010E940A79309345042093B3
:102A3000440480917A0390917B03A0917C03B09130
:102A40007D03BC01CD01A80197010E940A79309352
:102A50004704209346042091230830912408409194
:102A6000250850912608DA01C90163E0880F991FF3
:102A7000AA1FBB1F6A95D1F7820F931FA41FB51F12
:102A8000820F931FA41FB51F20919A0130919B01C3
:102A900040919C0150919D01BC01CD010E940A7999
:102AA000309349042093480480914A0390914B034A
:102AB000A0914C03B0914D0339E0B595A79597953A
:102AC00087953A95D1F780934A0480914603909177
:102AD0004703A0914803B091490329E0B595A79514
:102AE000979587952A95D1F780934B04809152034F
:102AF00090915303A0915403B091550309E0B5950B
:102B0000A795979587950A95D1F780934C048EE009
:102B100090E09F938F9384E494E09F938F9381E060
:102B20008F938F9383E48F930E94560D80910A02B6
:102B300090910B020E9421179093530480935204AA
:102B40002DB73EB7295F3F4F2DBF809106018F3FC4
:102B500071F1992714E0880F991F1A95E1F78E5E9D
:102B60009D4F40E150E0BC01CE0101960E94C47728
:102B700080E190E09F938F93CE0101969F938F9376
:102B800081E090E09F938F9386E091E09F938F93F5
:102B900082E08F9381E08F9381E48F930E94560DA2
:102BA0008FEF809306018DB79EB70B968DBF8091F6
:102BB0001D068823D1F0809107018823B1F081E0C0
:102BC00090E09F938F938DE196E09F938F9381E0A8
:102BD0008F938F9382E48F930E94560D10921D065F
:102BE0002DB73EB7295F3F4F2DBF80911902882333
:102BF000C9F0809107018823A9F084E390E09F93B6
:102C00008F938DE597E09F938F9381E08F938F93C0
:102C100080E58F930E94560D109219028DB79EB7D2
:102C200007968DBFE6E0C05F0C944D791F920F921E
:102C30000FB60F9211242F933F935F936F937F935F
:102C40008F939F93AF93BF93EF93FF9320E0809177
:102C50002E02882329F080912E02815080932E022B
:102C600080912504882319F0815080932504809158
:102C700036028150809336028F3F09F05BC089E0B5
:102C800080933602809134029091350201969093A0
:102C900035028093340280910F018F5F81708093A1
:102CA0000F01882319F481E080933302349903C023
:102CB00081E08093370280912F0290913002892B1E
:102CC00021F180912F02909130020B9750F080916A
:102CD0002F02909130020A979093300280932F0236
:102CE00004C01092300210922F0280912F02909116
:102CF0003002209108013091090182239323892B0E
:102D000011F021E008C020E006C08FEF9FEF909304
:102D100009018093080180910201222331F08A3059
:102D200011F45A9A07C0479A05C08A3011F45A988C
:102D300001C0479880913702882309F472C020911E
:102D4000F201222309F06DC080913F0683FF69C024
:102D500086B19927FC01E071F07084FF14C0809166
:102D600031029091320201969093320280933102A7
:102D70008091310290913202895E934008F451C0F3
:102D8000209337024EC08091310290913202892BFC
:102D900009F443C080913102909132028A569140E9
:102DA000E0F5809131029091320269E270E00E9478
:102DB000C1788091310290913202860F971F9093D3
:102DC00032028093310280913102909132020B974E
:102DD00050F080913102909132020A979093E30172
:102DE0008093E20104C0F093E301E093E20180915B
:102DF000E2019091E3012091400330914103821B55
:102E0000930B845E9D4F68E671E00E94D578845BE9
:102E1000904090933F0380933E03109232021092B1
:102E20003102FF91EF91BF91AF919F918F917F916F
:102E30006F915F913F912F910F900FBE0F901F9058
:102E400018952091340230913502280F391FC9019D
:102E5000019608952091340230913502821B930B24
:102E6000892F99278695807490700895CF93DF936A
:102E70000E942117EC01CE010E942A178823D9F362
:102E8000DF91CF910895CF93DF930E942117EC013A
:102E900009C080911001882329F0909310018FECD4
:102EA00080937A00CE010E942A17982F882389F3F5
:102EB000DF91CF9108959FB7F8945F983E9A469A14
:102EC0008091B0008F708093B0008091B0008360DB
:102ED0008093B0008091B1008B738093B10080919A
:102EE000B1008B608093B1001092B2008FEF80939D
:102EF000B3008091B00080688093B0008091700032
:102F00008A7F80937000809170008260809370004F
:102F10009FBF08958AE090E00E94211790933D02A0
:102F200080933C0282E085BD83EA84BD17BC84EBBC
:102F300088BD86E086BD80916E00816080936E00C2
:102F40000895A0E0B0E0E7EAF7E10C9430798091D1
:102F50006906E82FFF27E056FE4F9681D0808091CA
:102F60000E01A92FBB27A7FDB095CB2FDB2F8130FA
:102F700009F0DDC0209182033091830340918403E6
:102F800050918503BD01CE010E94967897FF04C041
:102F900061587F4F8F4F9F4F7B018C01F7E0159554
:102FA0000795F794E794FA95D1F78D2D992787FD2A
:102FB0009095A92FB92F20917A0330917B034091EE
:102FC0007C0350917D03BC01CD010E94967897FF50
:102FD00004C061587F4F8F4F9F4FE7E095958795CD
:102FE00077956795EA95D1F7F801E701C61BD70BEE
:102FF000E80BF90B2091130430911404C90153E03C
:10300000880F991F5A95E1F7821B930BAA2797FD0A
:10301000A095BA2FC81BD90BEA0BFB0B8091600659
:103020009927AA27BB27BC01CD019E01AF010E94B1
:10303000967897FF04C061507E4F8F4F9F4FFC01E1
:10304000EB0149E0F595E795D795C7954A95D1F7F6
:103050008091C501992736E0880F991F3A95E1F7CD
:1030600040910C0150910D01209168063327841B7B
:10307000950BB9010E94D57880910C0190910D01BA
:10308000860F971F90930D0180930C0180910C0186
:1030900090910D0197FD0F9624E0959587952A95BF
:1030A000E1F790932A02809329028091970680FF8E
:1030B00007C08091290290912A028C0F9D1F06C0A3
:1030C0008091290290912A028C1B9D0B90932A02D9
:1030D0008093290280916106282F3327220F331F06
:1030E000220F331F8091290290912A0282179307A1
:1030F0007CF080916206282F3327220F331F220F86
:10310000331F8091290290912A022817390724F44D
:1031100030932A022093290280910201843108F41D
:10312000C2C080910E018F5F80930E01BEC02091BE
:103130007A0330917B0340917C0350917D03BD0164
:10314000CE010E94967897FF04C061587F4F8F4F41
:103150009F4F7B018C01C7E015950795F794E79485
:10316000CA95D1F78D2D992787FD9095A92FB92F55
:103170002091820330918303409184035091850311
:10318000BC01CD010E9496789B01AC0197FF04C061
:1031900021583F4F4F4F5F4FB7E0559547953795B3
:1031A0002795BA95D1F72E0D3F1D401F511F8091D5
:1031B00064069927AA27BB27BC01CD010E949678F7
:1031C00097FF04C061507E4F8F4F9F4FFC01EB0172
:1031D000A9E0F595E795D795C795AA95D1F7809180
:1031E000C401992776E0880F991F7A95E1F74091FD
:1031F0000A0150910B01209168063327841B950B1F
:10320000B9010E94D57880910A0190910B01860F37
:10321000971F90930B0180930A0180910A0190916E
:103220000B0197FD0F9664E0959587956A95E1F7F8
:1032300090932802809327028091970681FF07C010
:1032400080912702909128028C0F9D1F06C08091CB
:103250002702909128028C1B9D0B9093280280934B
:10326000270280916506282F3327220F331F220F54
:10327000331F8091270290912802821793077CF0D8
:1032800080916606282F3327220F331F220F331F0A
:1032900080912702909128022817390724F430934F
:1032A00028022093270210920E01E7E0CDB7DEB787
:1032B0000C944C791F920F920FB60F9211242F93FA
:1032C0003F934F935F938F939F93EF93FF938091DF
:1032D000020190913802843108F04CC0992309F022
:1032E0001CC18091B00086FF24C08091B0008F7B0C
:1032F0008093B0008091290290912A0287559E4FB9
:1033000090932C0280932B0225E08D3D920718F0BC
:103310008CED95E005C08757914030F487E791E048
:1033200090932C0280932B0280912B0290912C027F
:10333000BAC08091B00080648093B000809167062D
:10334000282F33278DED96E0289FA001299F500D4F
:10335000389F500D1124CA012091390230913A0250
:10336000821B930B90932C0280932B0281E080931D
:103370000E01D0C0992309F0D0C08091B00086FF23
:1033800097C08091B0008F7B8093B000E0913B02AA
:10339000EE23F1F480916706282F33278DED96E018
:1033A000289FA001299F500D389F500D1124CA015C
:1033B0002091390230913A02821B930B90932C0298
:1033C00080932B0210923A0210923902469AA2C0C0
:1033D00089EA93E090932C0280932B028E2F9927F9
:1033E00083309105D9F08430910534F48130910512
:1033F00049F0029761F020C08430910591F0059763
:1034000099F01AC08091290290912A0204C08091FB
:1034100027029091280287559E4F1DC08091F10789
:1034200005C08091CB0702C08091F9079927880FCA
:10343000991F880F991FEFCFFF27EE0FFF1FE35A49
:10344000F84F20813181220F331F80912B02909100
:103450002C02820F931F90932C0280932B02809159
:103460002B0290912C0255E08D3D950718F08CEDC4
:1034700095E005C08757914030F487E791E090933D
:103480002C0280932B0220912B0230912C022C5B7A
:10349000304030932C0220932B028091390290917E
:1034A0003A02820F931F90933A028093390232C0FE
:1034B0008091B00080648093B0008CEB90E090939A
:1034C0002C0280932B028091390290913A0284540D
:1034D0009F4F90933A028093390280912D02882366
:1034E00021F080913003833320F480912D028230CB
:1034F00011F4469801C0469A80913B028F5F8093F9
:103500003B0290916706981728F481E080930E01A2
:1035100010923B0281E08093380220912B0230917F
:103520002C0241E02F37340730F08FEF8093B30047
:103530002F5F30400FC02F3F3105C9F0C0F0A90107
:103540004F5F50404F37510550F480E88093B300EF
:103550002058304030932C0220932B0212C08FEF62
:103560008093B30050932C0240932B020AC08091A9
:103570002B028093B30010922C0210922B02109217
:103580003802FF91EF919F918F915F914F913F9101
:103590002F910F900FBE0F901F90189510927C00E6
:1035A0008FEC80937A000895CF93DF9310924202BC
:1035B00083E090E00E949B2CC82FDD27C531D10508
:1035C00008F02A97C7BD84E690E00E9443178091D7
:1035D0001401909115018052934010F4C0E0D0E0A6
:1035E000CA3FD105F8F4C7BD82E390E00E944317BB
:1035F00087E294E09F938F938BEF92E19F938F9359
:10360000E0914204F0914304099580911401909156
:1036100015010F900F900F900F908052934010F073
:103620002196DECFC0932E066C2F83E090E00E949F
:10363000A12C80913F0680FF0AC080912E068A50FF
:103640008B3E28F080915B04806480935B04C7BD4F
:103650008CE291E00E944317DF91CF910895EF92A1
:10366000FF921F93CF9310E080ED97E00E94211707
:103670007C01CCE8133019F4CB3008F0C9E010E03D
:1036800080915202909153028C5F934024F4809178
:10369000130181500AC080915202909153028750C9
:1036A000944034F0809113018F5F8093130101C027
:1036B00011E080915002909151028C5F934024F46C
:1036C0008091120181500AC0809150029091510264
:1036D0008750944034F0809112018F5F80931201E3
:1036E00001C01F5F80914E0290914F028C5F93400A
:1036F00024F48091110181500AC080914E02909172
:103700004F0287509440C4F0809111018F5F8093E5
:10371000110113C089E294E09F938F938BEF92E1A4
:103720009F938F93E0914204F091430409950F9089
:103730000F900F900F905FC01F5F82E180937D021A
:10374000809177028E7F8093770285EA8093BC0018
:10375000809113018A3040F480915B0481608093F2
:103760005B048AE08093130180911301863F40F04F
:1037700080915B04816080935B0485EF80931301EB
:10378000809112018A3040F480915B0482608093C2
:103790005B048AE08093120180911201863F40F021
:1037A00080915B04826080935B0485EF80931201BB
:1037B000809111018A3040F480915B048460809391
:1037C0005B048AE08093110180911101863F40F0F3
:1037D00080915B04846080935B0485EF809311018A
:1037E00080917D02882339F0C7010E942A1788231F
:1037F00009F090CFF5CF109210018FEC80937A00F2
:10380000809110018823E1F3CA3020F48AE090E02F
:103810000E944317C15009F02DCF86E490E00E942A
:103820004317CF911F91FF90EF9008951F920F9231
:103830000FB60F921124AF92BF92CF92DF92EF9208
:10384000FF920F931F932F933F934F935F936F9329
:103850007F938F939F93AF93BF93EF93FF93809149
:103860005B02282F3327442755278F5F80935B0205
:10387000F9012231310508F08CC3E25CFF4F0C9452
:103880005C79809178009091790046C080917800B1
:10389000909179002CC1809178009091790090935B
:1038A0005E0280935D0257C180918B0390918C03DF
:1038B0002091780030917900821B930B90931F0622
:1038C00080931E0680911E0690911F0690936802B9
:1038D000809367025EC18091780090917900209179
:1038E0008D0330918E03821B930B90932D06809352
:1038F0002C0680912C0690912D0690936A0280935D
:10390000690249C38091610290916202209178001E
:1039100030917900820F931F90936202809361022D
:1039200081E03AC380915F0290916002209178001B
:1039300030917900820F931F9093600280935F0211
:1039400084E02AC380911E0190911F019C01220FE7
:10395000331F280F391F809178009091790063E020
:1039600070E00E94C178260F371F3695279536954F
:10397000279530931F0120931E0185E00DC3809190
:103980007800909179004091870350918803841BBF
:10399000950B909349028093480280914802909140
:1039A0004902029704F122E04E3E520784F420912E
:1039B0005C022B5F20935C0225508091F60290916F
:1039C000F702845F914018F4215F20935C0280919C
:1039D0005C02853684F14F5F5F4F509388034093BC
:1039E0008703845626C080914802909149028F5FD8
:1039F0009F4F0CF532E047325307ECF020915C0208
:103A0000255020935C022B5F8091F6029091F70283
:103A1000845F914018F42F5020935C0280915C02E7
:103A20008C394CF4415050405093880340938703A5
:103A30008C5980935C0281E08093470280917800EA
:103A400090917900909325068093240680914802F6
:103A5000909149029C01442737FD4095542F809155
:103A6000420390914303A0914403B0914503820F18
:103A7000931FA41FB51F8093420390934303A09309
:103A80004403B09345032091420330914303409196
:103A900044035091450357FF04C021503C4F4F4F02
:103AA0005F4F0AE055954795379527950A95D1F7C9
:103AB0008091420390914303A0914403B091450348
:103AC000821B930BA40BB50B80934203909343038B
:103AD000A0934403B09345032EC180915F0290915F
:103AE00060022091780030917900820F931F9093AB
:103AF000600280935F0210925A0250C280910201CC
:103B00008A3071F4809178009091790020915D0263
:103B100030915E02820F931F01969695879517C08C
:103B200040915D0250915E02843158F020917800FE
:103B300030917900240F351F8FEF97E0821B930B94
:103B400006C08091780090917900840F951F909322
:103B50004F0280934E0286E01FC280918B039091AA
:103B60008C032091780030917900821B930B909305
:103B70001F0680931E0680911E0690911F062091BD
:103B8000670230916802820F931F90934D028093D9
:103B90004C0287E001C280917800909179002091D9
:103BA0008D0330918E03821B930B90932D0680938F
:103BB0002C0680912C0690912D062091690230915F
:103BC0006A02820F931F90934B0280934A02E3C1D3
:103BD0002091610230916202809178009091790089
:103BE000280F391F309362022093610280910201F5
:103BF0008A3019F4220F331F04C0220F331F220F03
:103C0000331F309362022093610220916102309150
:103C10006202C90137FD0796A3E095958795AA959D
:103C2000E1F7909353028093520280916302909146
:103C30006402820F931F97FD019695958795909347
:103C40006402809363022091970330919803821B52
:103C5000930B90931D0180931C0120915802309189
:103C6000590280911C0190911D01280F391F37FFC7
:103C700002C02F5F3F4F359527953093590220930F
:103C800058024ECE20915F02309160028091780000
:103C900090917900280F391F3093600220935F02C2
:103CA000809102018A3019F4220F331F04C0220FC1
:103CB000331F220F331F3093600220935F02209145
:103CC0005F0230916002C90137FD079663E0959568
:103CD00087956A95E1F79093510280935002809105
:103CE000650290916602820F931F97FD019695954C
:103CF0008795909366028093650220919503309199
:103D00009603821B930B90931B0180931A012091C1
:103D100056023091570280911A0190911B01280F91
:103D2000391F37FF02C02F5F3F4F359527953093DE
:103D300057022093560283E02FC110925B0281E06C
:103D40008093100180913E0290913F0201969093E2
:103D50003F0280933E028091780090917900909389
:103D60001501809314018091140190911501AA27E7
:103D7000BB27A0906B02B0906C02C0906D02D090F7
:103D80006E02A80EB91ECA1EDB1EA0926B02B09274
:103D90006C02C0926D02D0926E0280916F028F5FB2
:103DA00080936F02823108F4F6C0809116019091E1
:103DB0001701A0911801B09119017C018D0123E038
:103DC000EE0CFF1C001F111F2A95D1F7E81AF90A03
:103DD0000A0B1B0BEA0CFB1C0C1D1D1D80914202E3
:103DE000992787FD9095A92FB92FBC01CD0126EC0D
:103DF00034E240E050E00E949678DC01CB01E81A02
:103E0000F90A0A0B1B0BD801C7010496A11DB11DAD
:103E1000B7FF05C0D801C7010B96A11DB11D13E066
:103E2000B595A795979587951A95D1F78093160123
:103E300090931701A0931801B09319018091260661
:103E4000909127067C010027F7FC0095102F8091A8
:103E5000160190911701A0911801B0911901E81A6B
:103E6000F90A0A0B1B0BE0922203F0922303009342
:103E70002403109325032091430230914402409182
:103E800045025091460257FF04C0215F3F4F4F4FFC
:103E90005F4FF4E05595479537952795FA95D1F7FB
:103EA0008091430290914402A0914502B091460254
:103EB000821B930BA40BB50B809343029093440297
:103EC000A0934502B0934602809143029091440230
:103ED000A0914502B09146028E0D9F1DA01FB11FFB
:103EE0008093430290934402A0934502B09346020C
:103EF0008091400290914102AC01E5E0440F551FD2
:103F0000EA95E1F7481B590B8091430290914402D6
:103F1000A0914502B0914602B7FF03C00F96A11DC4
:103F2000B11D74E0B595A795979587957A95D1F7CA
:103F30002091220330912303281B390B63E0220FC9
:103F4000331F6A95E1F7240F351F37FF02C0215E4A
:103F50003F4F45E0359527954A95E1F7309341026B
:103F600020934002D601C501D7FE03C00196A11DD2
:103F7000B11DB595A7959795879580936B02909302
:103F80006C02A0936D02B0936E0289E080936F0281
:103F900002C010925B0282E080935A0280915A0222
:103FA00080937C0080915B02882319F08FEC8093D2
:103FB0007A00FF91EF91BF91AF919F918F917F9187
:103FC0006F915F914F913F912F911F910F91FF90B2
:103FD000EF90DF90CF90BF90AF900F900FBE0F90FB
:103FE0001F90189590E2E1E2F1E08FE49193815007
:103FF00087FFFCCF089590917202E1E2F1E0E90FB2
:10400000F11D80839F5F909372020895EF92FF925B
:104010000F931F93CF93DF932091700220FF0AC06C
:1040200080917102882311F0815002C0809120019B
:104030008093710221FF0CC0909171028091200148
:10404000981719F41092710203C09F5F9093710248
:10405000822F992780FF04C081FF02C01092710255
:104060000E94F21F80917102282F33275BEFE52E0B
:104070005FE1F52EC0914204D09143048A3098F458
:1040800081E1809372023F932F9380E694E09F93A7
:104090008F93FF92EF92FE0109952DB73EB72A5FED
:1040A0003F4F2DBF11C080E1809372023F932F9349
:1040B00085E694E09F938F93FF92EF92FE0109951E
:1040C0008DB79EB706968DBF20917102822F9927DA
:1040D000AA27BB27FC01429710F00C94B72AE05B9B
:1040E000FF4F4BEFE42E4FE1F42EC0914204D091EC
:1040F00043040C945C79109272028AE694E09F93D8
:104100008F930BEF1FE1FF92EF92FE01099584E17F
:10411000809372020F900F900F900F9081E690E0C5
:104120009F938F9384E590E09F938F931F921F92AC
:10413000809102016AE00E94B578892F99279F93A8
:104140008F93809102010E94B57899279F938F9356
:104150008AE794E09F938F93FF92EF92E09142045D
:10416000F0914304099588E2809372022DB73EB71F
:10417000225F3F4F2DBF87EA96E09F938F930E9467
:10418000BD2D99279F938F938FE894E09F938F93F2
:10419000FF92EF92E0914204F091430409958DB7AC
:1041A0009EB708968DBF90915B04992351F08CE3E4
:1041B00080937202892F99279F938F938DE994E0C2
:1041C00081C690917802992371F08CE380937202FA
:1041D000892F99279F938F9384EB94E09F938F93DC
:1041E0001F930F9391C080915C0484FF07C08CE300
:1041F0008093720289EC94E00C94492A8091920198
:1042000090919301069710F00C94C02A8CE3809350
:10421000720286ED94E00C94492A80913F063BEFB0
:10422000E32E3FE1F32EC0914204D091430480FF7E
:1042300074C0109272028091220390912303A09186
:104240002403B0912503BC01CD0125E030E040E01E
:1042500050E00E940A793F932F9383EE94E09F935E
:104260008F93FF92EF92FE01099584E18093720291
:104270002DB73EB72A5F3F4F2DBF80911E0390910F
:104280001F03A0912003B0912103BC01CD0125E0C3
:1042900030E040E050E00E940A793F932F9380EF96
:1042A00094E09F938F93FF92EF92E0914204F091FC
:1042B0004304099588E2809372028DB79EB70696F3
:1042C0008DBF80911401909115019F938F938DEF75
:1042D00094E09F938F93FF92EF92E0914204F091CC
:1042E000430409958CE3809372022DB73EB72A5F91
:1042F0003F4F2DBF87B599279F938F938AE095E015
:104300009F938F93FF92EF92E0914204F0914304C8
:1043100009958DB79EB7069633C71092720287E152
:1043200095E09F938F93FF92EF92FE01099584E1B0
:10433000809372020F900F900F900F9086E295E09D
:104340009F938F93FF92EF92E0914204F091430488
:10435000099588E2809372020F900F900F900F9052
:104360008FE295E09F938F93FF92EF92E09142044A
:10437000F091430409958CE3809372020F900F90A3
:104380000F900F908EE395E09F938F93FF92EF92A3
:104390000C944D2A1092720287E495E09F938F93BC
:1043A0000BEF1FE1FF92EF92FE01099584E18093EC
:1043B00072020F900F900F900F9080918203909156
:1043C0008303A0918403B0918503B7FF04C081509B
:1043D0009C4FAF4FBF4F2AE0B595A795979587950E
:1043E0002A95D1F7BF93AF939F938F9384E595E080
:1043F0009F938F931F930F93E0914204F091430496
:10440000099588E2809372022DB73EB7285F3F4F2F
:104410002DBF80917A0390917B03A0917C03B09192
:104420007D03B7FF04C081509C4FAF4FBF4FCAE020
:10443000B595A79597958795CA95D1F7BF93AF93F3
:104440009F938F9383E695E09F938F931F930F9392
:10445000E0914204F091430409958CE38093720249
:104460008DB79EB708968DBF8091E2019091E301D0
:104470009F938F9382E795E09F938F931F930F9362
:10448000E0914204F091430409952DB73EB72A5FAD
:104490003F4F11C71092720280916107909162079D
:1044A0009F938F9380915F07909160079F938F9365
:1044B00081E895E09F938F93FF92EF92FE0109951B
:1044C00084E1809372028DB79EB708968DBF80916C
:1044D0006507909166079F938F93809163079091F2
:1044E00064079F938F9381E995E09F938F93FF9249
:1044F000EF92E0914204F0914304099588E28093A1
:1045000072022DB73EB7285F3F4F2DBF80916907DC
:1045100090916A079F938F938091670790916807A6
:104520009F938F9381EA95E09F938F93FF92EF92F1
:10453000E0914204F091430409958CE38093720268
:104540008DB79EB708968DBF80916D0790916E07CD
:104550009F938F9380916B0790916C079F938F939C
:1045600081EB95E0A2C01092720280913406E82F90
:10457000FF27EE0FFF1FE35AF84F808191819F9331
:104580008F9380913306E82FFF27EE0FFF1FE35A2A
:10459000F84F808191819F938F9381EC95E09F9359
:1045A0008F93FF92EF92FE01099584E1809372024E
:1045B0008DB79EB708968DBF80913606E82FFF27EE
:1045C000EE0FFF1FE35AF84F808191819F938F93E5
:1045D00080913506E82FFF27EE0FFF1FE35AF84FB3
:1045E0008081918188589F4F9F938F9381ED95E0B3
:1045F0009F938F93FF92EF92E0914204F0914304D6
:10460000099588E2809372022DB73EB7285F3F4F2D
:104610002DBF80913806E82FFF27EE0FFF1FE35ACA
:10462000F84F8081918181589F4F9F938F93809104
:104630003706E82FFF27EE0FFF1FE35AF84F808160
:10464000918181589F4F9F938F9381EE95E09F9327
:104650008F93FF92EF92E0914204F0914304099509
:104660008CE3809372028DB79EB708968DBF8091C0
:104670003A06E82FFF27EE0FFF1FE35AF84F80811D
:10468000918181589F4F9F938F9380913906E82F96
:10469000FF27EE0FFF1FE35AF84F80819181815869
:1046A0009F4F9F938F9381EF95E09F938F93FF92FE
:1046B000EF92E0914204F091430409952DB73EB783
:1046C000285F3F4FF8C51092720281E096E09F93F9
:1046D0008F930BEF1FE1FF92EF92FE0109958091FE
:1046E00002010F900F900F900F908A3009F09DC03B
:1046F00084E18093720280919703909198039C01CA
:1047000097FF02C0295F3F4F287F821B930B9F9327
:104710008F93809197039091980397FD0796A3E05C
:1047200095958795AA95E1F79F938F93209197038D
:104730003091980337FF02C0295F3F4FF3E0359572
:104740002795FA95E1F78091520290915302821BCE
:10475000930B9F938F938FE096E09F938F931F937C
:104760000F93E0914204F0914304099588E280930D
:1047700072028DB79EB70A968DBF80919503909176
:1047800096039C0197FF02C0295F3F4F287F821B41
:10479000930B9F938F93809195039091960397FD30
:1047A0000796E3E095958795EA95E1F79F938F93B8
:1047B000209195033091960337FF02C0295F3F4F48
:1047C00073E0359527957A95E1F7809150029091A5
:1047D0005102821B930B9F938F9380E296E09F93ED
:1047E0008F931F930F93E0914204F0914304099536
:1047F0008CE3809372022DB73EB7265F3F4F2DBFEB
:1048000080919303909194039F938F93809193034E
:104810009091940320914E0230914F02821B930B92
:104820009F938F9381E396E0A7C38B3019F0843177
:1048300008F4ADC084E18093720280919703909157
:1048400098039C0197FF02C0215F3F4F207F821B8E
:10485000930B97FD0196959587959F938F938091E4
:1048600097039091980397FD0F9654E0959587953F
:104870005A95E1F79F938F93209197033091980376
:1048800037FF02C0295F3F4F43E0359527954A9592
:10489000E1F78091520290915302821B930B9F93F8
:1048A0008F938FE396E09F938F931F930F93E091E5
:1048B0004204F0914304099588E2809372022DB777
:1048C0003EB7265F3F4F2DBF809195039091960391
:1048D0009C0197FF02C0215F3F4F207F821B930BFB
:1048E00097FD0196959587959F938F93809195035A
:1048F0009091960397FD0F96C4E095958795CA957C
:10490000E1F79F938F93209195033091960337FFA2
:1049100002C0295F3F4FB3E035952795BA95E1F77F
:104920008091500290915102821B930B9F938F9321
:1049300081E596E09F938F931F930F93E09142043C
:10494000F091430409958CE3809372028DB79EB772
:104950000A968DBF809193039091940397FD0196E1
:10496000959587959F938F9380919303909194034E
:1049700020914E0230914F02821B930B9F938F9395
:1049800083E696E09F938F931F930F9392CE8D3083
:1049900009F0F6C584E18093720280911301992792
:1049A0009F938F93809197039091980397FD0F9613
:1049B000F4E095958795FA95E1F79F938F93209171
:1049C00097033091980337FF02C0295F3F4FE3E020
:1049D00035952795EA95E1F780915202909153021F
:1049E000821B930B9F938F9382E796E09F938F9305
:1049F0001F930F93E0914204F0914304099588E2DC
:104A0000809372028DB79EB70A968DBF8091120176
:104A100099279F938F93809195039091960397FD8B
:104A20000F9674E0959587957A95E1F79F938F930C
:104A3000209195033091960337FF02C0295F3F4FC5
:104A400063E0359527956A95E1F780915002909142
:104A50005102821B930B9F938F9386E896E09F935E
:104A60008F931F930F93E0914204F09143040995B3
:104A70008CE3809372022DB73EB7265F3F4F2DBF68
:104A80008091110199279F938F9380919303909127
:104A9000940397FD0196959587959F938F938091A9
:104AA00093039091940320914E0230914F02821B08
:104AB000930B9F938F938AE996E09F938F931F9315
:104AC0000F93E0914204F091430409958DB79EB78E
:104AD0000A9656C3109272028EEA96E09F938F93C5
:104AE000FF92EF92FE01099584E1809372020F908C
:104AF0000F900F900F9080918D0390918E039F9354
:104B00008F9380914A0290914B029F938F938BEBEE
:104B100096E09F938F93FF92EF92E0914204F09181
:104B20004304099588E2809372022DB73EB7285F4F
:104B30003F4F2DBF80918B0390918C039F938F9358
:104B400080914C0290914D029F938F938AEC96E056
:104B50009F938F93FF92EF92E0914204F091430470
:104B600009958CE3809372028DB79EB708968DBF2E
:104B700080918703909188039F938F93809148023F
:104B8000909149029F938F9389ED96E08ECD10927C
:104B9000720280911E0190911F016AE070E00E94F4
:104BA000D5789F938F9380911E0190911F016AE0A9
:104BB00070E00E94D5787F936F9388EE96E09F9384
:104BC0008F93FF92EF92FE01099584E18093720228
:104BD0008DB79EB708968DBF8091A8089091A908BF
:104BE0006AE070E00E94C1789F938F938091A8083B
:104BF0009091A9086AE070E00E94C1787F936F935A
:104C00008CEF96E09F938F93FF92EF92E091420496
:104C1000F0914304099588E2809372022DB73EB764
:104C2000285F3F4F2DBF8091AA089091AB089F93BA
:104C30008F9380E197E09F938F93FF92EF92E091A3
:104C40004204F091430409958CE3809372028DB77E
:104C50009EB706968DBF8091AC089091AD089F934A
:104C60008F9380E297E02EC11092720282E397E068
:104C70009F938F93FF92EF92FE01099584E18093B9
:104C800072020F900F900F900F9080915D0790919E
:104C90005E079F938F938BE397E09F938F93FF9291
:104CA000EF92E0914204F0914304099588E28093E9
:104CB00072028DB79EB706968DBF809130039927FB
:104CC0009F938F938BE497E09F938F93FF92EF9244
:104CD000E0914204F091430409958CE380937202C1
:104CE0002DB73EB72A5F3F4F2DBF80915C079927B4
:104CF00001979F938F938BE597E002CB10927202FE
:104D00008BE697E09F938F93FF92EF92FE010995B8
:104D100084E1809372020F900F900F900F9080911A
:104D20003E0390913F039F938F9383E797E09F9378
:104D30008F93FF92EF92E0914204F0914304099522
:104D400088E2809372022DB73EB72A5F3F4F2DBF96
:104D50008091E2019091E3019F938F9381E897E026
:104D60009F938F93FF92EF92E0914204F09143045E
:104D700009958CE3809372028DB79EB706968DBF1E
:104D800080914003909141039F938F938FE897E028
:104D900099C0109272028091310399279F938F934B
:104DA0008DE997E09F938F93FF92EF92FE01099513
:104DB00084E1809372028DB79EB706968DBF809175
:104DC000320399279F938F9389EA97E09F938F935C
:104DD000FF92EF92E0914204F0914304099588E23A
:104DE000809372022DB73EB72A5F3F4F2DBF80914F
:104DF000330399279F938F9385EB97E09F938F932E
:104E0000FF92EF92E0914204F091430409958CE304
:104E1000809372028DB79EB706968DBF8091340342
:104E200099279F938F9381EC97E04CC01092720268
:104E30008091350399279F938F938DEC97E09F93F3
:104E40008F93FF92EF92FE01099584E180937202A5
:104E50008DB79EB706968DBF8091360399279F9395
:104E60008F9389ED97E09F938F93FF92EF92E0915C
:104E70004204F0914304099588E2809372022DB7B1
:104E80003EB72A5F3F4F2DBF8091370399279F93ED
:104E90008F9385EE97E09F938F93FF92EF92E0912F
:104EA0004204F091430409958CE3809372028DB71C
:104EB0009EB706968DBF8091380399279F938F9355
:104EC00081EF97E09F938F93FF92EF92D9CA109250
:104ED00072028DEF97E09F938F930BEF1FE1FF928C
:104EE000EF92FE01099584E1809372020F900F907A
:104EF0000F900F908091C50199279F938F9385E024
:104F000098E09F938F93FF92EF92E0914204F0918B
:104F10004304099588E2809372028DB79EB7069686
:104F20008DBF8091290290912A0297FD0396959555
:104F30008795959587959F938F9383E198E09F93AD
:104F40008F931F930F93E0914204F09143040995CE
:104F50008CE3809372022DB73EB72A5F3F4F2DBF7F
:104F60008091620699279F938F938091610699277C
:104F70009F938F9381E298E09F938F931F930F935A
:104F8000E0914204F091430409958DB79EB70896CD
:104F9000F7C0109272028FE298E09F938F93FF9276
:104FA000EF92FE01099584E1809372020F900F90B9
:104FB0000F900F9080917C04992787FD90959F9387
:104FC0008F9380917B04992787FD90959F938F9372
:104FD0008FE398E09F938F93FF92EF92E0914204CA
:104FE000F0914304099588E2809372022DB73EB791
:104FF000285F3F4F2DBF80917D04992787FD9095B5
:105000009F938F9380917E0499279F938F938FE432
:1050100098E09F938F93FF92EF92E0914204F0917A
:10502000430409958CE3809372028DB79EB708966E
:105030008DBF8091820499279F938F9380917F04E5
:10504000992787FD90959F938F938FE598E02DCBBF
:10505000109272028FE698E09F938F93FF92EF92E7
:10506000FE01099584E1809372020F900F900F90DA
:105070000F908091170799278F7790709F938F9348
:1050800080910F0799278F7790709F938F938091CE
:10509000070799278F7790709F938F938091FF06D2
:1050A00099278F7790709F938F938FE798E09F93C6
:1050B0008F93FF92EF92E0914204F091430409959F
:1050C00088E2809372028DB79EB70C968DBF809157
:1050D000370799278F7790709F938F9380912F0731
:1050E00099278F7790709F938F93809127079927A7
:1050F0008F7790709F938F9380911F0799278F7759
:1051000090709F938F9380E998E09F938F93FF9285
:10511000EF92E0914204F091430409958CE380936F
:1051200072022DB73EB7245F3F4F2DBF80915707C6
:1051300099278F7790709F938F9380914F0799272E
:105140008F7790709F938F938091470799278F77E0
:1051500090709F938F9380913F0799278F779070DE
:105160009F938F9381EA98E09F938F93FF92EF92A2
:10517000E0914204F091430409958DB79EB70C96D7
:105180008DBFFEC11092720282EB98E09F938F93C5
:10519000FF92EF92FE01099584E1809372020F90D5
:1051A0000F900F900F9080911B07992787FD909586
:1051B0009F938F9380911307992787FD90959F93D5
:1051C0008F9380910B07992787FD90959F938F93DD
:1051D00080910307992787FD90959F938F9381EC8A
:1051E00098E09F938F93FF92EF92E0914204F091A9
:1051F0004304099588E2809372022DB73EB7245F7D
:105200003F4F2DBF80913B07992787FD90959F9336
:105210008F9380913307992787FD90959F938F9364
:1052200080912B07992787FD90959F938F9380916D
:105230002307992787FD90959F938F9382ED98E0A0
:105240009F938F93FF92EF92E0914204F091430479
:1052500009958CE3809372028DB79EB70C968DBF33
:1052600080915B07992787FD90959F938F938091FD
:105270005307992787FD90959F938F9380914B07B4
:10528000992787FD90959F938F9380914307992746
:1052900087FD90959F938F9383EE98E09F938F93D4
:1052A000FF92EF92E0914204F091430409952DB7EB
:1052B0003EB7245F3F4F2DBF63C11092720284EF4F
:1052C00098E09F938F930BEF1FE1FF92EF92FE0107
:1052D000099584E1809372020F900F900F900F90C8
:1052E00080911707881F8827881F97E0899FC00132
:1052F00011248D969F938F9380910F07881F882785
:10530000881F96E0899FC00111248D969F938F93EB
:1053100080910707881F8827881F95E0899FC00113
:1053200011248D969F938F938091FF06881F882765
:10533000881F9927880F991F880F991F8D969F9313
:105340008F9383E099E09F938F93FF92EF92E09188
:105350004204F0914304099588E2809372028DB76C
:105360009EB70C968DBF80913707881F8827881FAE
:105370009BE0899FC00111248D969F938F9380910C
:105380002F07881F8827881F9AE0899FC001112452
:105390008D969F938F9380912707881F8827881F5A
:1053A00099E0899FC00111248D969F938F938091DE
:1053B0001F07881F8827881F992723E0880F991FB8
:1053C0002A95E1F78D969F938F9387E199E09F93BC
:1053D0008F93FF92EF92E0914204F091430409957C
:1053E0008CE3809372022DB73EB7245F3F4F2DBFF1
:1053F00080913F07881F8827881F9CE0899FC001F4
:1054000011248D969F938F938BE299E09F938F93B6
:10541000FF92EF92E0914204F0914304099580914C
:1054200047072DB73EB72A5F3F4F2DBF87FF12C0FA
:1054300080E4809372028CE399E09F938F93FF92B4
:10544000EF92E0914204F091430409950F900F9080
:105450000F900F9080914F0787FF12C084E48093D4
:1054600072028FE399E09F938F931F930F93E091C4
:105470004204F091430409950F900F900F900F9004
:105480008091570787FF7CC088E48093720282E492
:1054900099E09F938F931F930F93E0914204F091B3
:1054A000430409950F900F900F900F9069C01092D0
:1054B000720285E499E09F938F93FF92EF92FE0131
:1054C000099584E1809372020F900F900F900F90D6
:1054D00080910002909101029F938F9383E599E060
:1054E0009F938F93FF92EF92E0914204F0914304D7
:1054F000099588E2809372028DB79EB706968DBF9C
:1055000080910202909103029F938F9380E699E02D
:105510009F938F93FF92EF92E0914204F0914304A6
:10552000099589E4809372022DB73EB72A5F3F4FF9
:105530002DBF8DE699E09F938F93FF92EF92E091BC
:105540004204F09143040995809170020F900F90EE
:105550000F900F9083FF14C010920302109202026A
:1055600060E070E08EE090E00E94AB2C09C080917A
:105570002001281719F42150209320011092710264
:1055800010927002E6E0CDB7DEB70C944D794AEA8E
:1055900020E030E02617370740F4FC018191480FE6
:1055A0002F5F3F4F26173707C8F3842F9927089599
:1055B000AC019AEA20E030E02617370750F4DA0110
:1055C000A20FB31F0E946279802D980F2F5F3F4F6B
:1055D000F3CF892F9927089581E08093350682E0E3
:1055E0008093340683E08093330684E0809336060C
:1055F00085E08093370686E08093380687E08093C5
:10560000390688E080933A0689E080933B068AE079
:1056100080933C068BE080933D068CE080933E06B1
:10562000089595E59093320680910201843170F0DF
:105630008AE080935206109276068BE180934E06A4
:105640008EE480937306809374060DC083E080938C
:10565000520680E2809376068EE180934E06909308
:105660007306909374068AE680933F0662E0609327
:10567000980674E07093590610929506109292065F
:1056800048E040934C0656EE50934D0690E49093BC
:105690004F063EE1309340068FEF809342068FE045
:1056A0008093430630934106109245064093460688
:1056B00090934706109248068093440610925B062A
:1056C00010925C0610925D0610925E0610927806AB
:1056D0001092790610927A0610927B0690E89093C9
:1056E0005F0622E32093600660939706809361062D
:1056F00050936206709367068DE780936A068093E5
:105700006B0680936C069093630685E58093640630
:1057100086E4809365068CED809366068CE3809327
:105720006806109269068FE580937C0683EF80936C
:105730007E068AEA809380068093810684E18093C6
:105740007D0680937F0620936D069AE590936E0602
:1057500020936F06109296068EEF8093820624E6C1
:1057600020938306909384069093850690938606F3
:105770008BE4809387068093880680938906109235
:105780008A0686E080938B0640938C0690938D0664
:1057900030938E0685EF80938F062093900660935A
:1057A0009106109293061092940681E28093560619
:1057B0008DE280935706909358060895CF93DF9318
:1057C0000E94112B8EE08093490620E120934A0627
:1057D0003CE030934B0690E59093500686E9809329
:1057E0005106909353068093540686E080935506A5
:1057F00080E280935A068AE5809370069093710642
:1058000081E0809372062093750684E68093770684
:10581000A9E9B6E0E1E7F1E0ED01019009923A95DE
:10582000E1F763E770E0CD01875690400E94C72AF8
:105830008093A506DF91CF910895CF93DF930E94C7
:10584000112B8AE08093490680E180934A0626E086
:1058500020934B069AE59093500688E78093510673
:1058600090935306809354062093550620E220938C
:105870005A069093700680E5809371068CE38093BE
:105880007206209375068BE480937706A9E9B6E04B
:105890008CE0E8E7F1E0ED01019009928A95E1F7EB
:1058A00063E770E0CD01875690400E94C72A80933D
:1058B000A506DF91CF910895CF93DF930E94112B1E
:1058C00088E08093490630E130934A0626E0209331
:1058D0004B0694E69093500688E780935106909388
:1058E0005306809354062093550630935A068AE552
:1058F0008093700680E58093710696E4909372061B
:1059000080E28093750690937706A9E9B6E08CE073
:10591000E0E8F1E0ED01019009928A95E1F763E793
:1059200070E0CD01875690400E94C72A8093A5065B
:10593000DF91CF910895DC010E946279802D992733
:105940000895DC01062E0E9474790895DC010E94FE
:105950006F79CF010895DC010B010E9480790895D1
:10596000FF920F931F93CF93DF93982F8150853031
:1059700008F093E084E7F82E9F9D80011124E80150
:10598000609763E770E0CE010E94D82A982FD80173
:10599000AD59BF4F0E946279802D891731F4DE0125
:1059A0000E946279802D853519F080E090E00AC070
:1059B000E2E3F6E0DE011F2C0E946A790E94B068E3
:1059C00081E090E0E5E0CDB7DEB70C944E7986300B
:1059D00010F085E003C0882309F481E0A2E0B0E084
:1059E000082E0E94747908951F93CF93DF93182F88
:1059F000C2E3D6E080913206853591F5163010F07D
:105A000015E002C0112361F163E770E082E396E0E4
:105A10000E94C72A8093A50684E7189FD00111240D
:105A20005097FE01182E0E948579E3E3F6E0A0E589
:105A3000B0E02CE030E0122E0E948579B90183E3BA
:105A400096E00E94C72AACE5B0E0082E0E94747967
:105A5000812F0E94E72C0E94B06881E090E002C094
:105A600080E090E0DF91CF911F9108956DE470E0A8
:105A700088EE93E00E94D82AA5E3B4E00E94627900
:105A8000902D981739F4A8EEB3E00E946279802D2A
:105A9000813019F080E090E00895E6EAF6E0A8EEA3
:105AA000B3E08EE4182E0E946A7981E090E00895B8
:105AB000CF93DF93C6EAD6E08091A606813089F4C1
:105AC0006DE470E0CE010E94C72A8093F306A8EE31
:105AD000B3E08EE4FE01182E0E94857981E090E00B
:105AE00002C080E090E0DF91CF910895CF93DF93E3
:105AF00081E08093A606E6EAF6E08FE0158616863A
:105B00001786108A8150349687FFF8CF80E48093FF
:105B1000B3068093B4061092B5068093B6068093C0
:105B2000B70690EC9093B8061092B9068093BA0627
:105B30008093BB061092BC069093BD069093BE0660
:105B40008093BF061092C0068093C1069093C20650
:105B5000A7EAB6E087E0EAE8F1E0ED0101900992FA
:105B60008A95E1F76DE470E0CD0101970E94C72AA4
:105B70008093F306DF91CF910895A2E0B0E00E94F8
:105B80006279802D863030F083E0A2E0B0E0082E0C
:105B90000E947479992708951F93CF93C82F162FC9
:105BA000863010F0C5E003C0882309F4C1E08C2FD3
:105BB00099278230910541F08330910544F4019793
:105BC00031F40E94DE2B05C00E941D2C02C00E94F1
:105BD0005C2C1123B1F06CE070E080E590E00E9455
:105BE000D82AACE5B0E00E946279902D981749F46C
:105BF000E3E3F6E0A0E5B0E08CE0182E0E946A79BD
:105C000002C00E94EC2A8C2F0E94F42CCF911F918D
:105C10000895DF92EF92FF920F931F93CF93FF248B
:105C2000DF2CEF2C81E090E00E949B2C853539F031
:105C300031E0E32E65E581E090E00E94A12C6CE06C
:105C400070E080E590E00E94D82AC82FACE5B0E073
:105C50000E946279802D8C1711F421E0D22EC1E0D0
:105C600001E010E0EE2029F48C2F0E94B02C882354
:105C7000B1F591E0F92E1F930F9385E799E09F937B
:105C80008F938BEF92E19F938F93E0914204F09179
:105C9000430409958DB79EB706968DBF0230110556
:105CA00049F0033011054CF40130110531F40E9424
:105CB000DE2B05C00E941D2C02C00E945C2CDD2042
:105CC00049F0E3E3F6E0A0E5B0E08CE0182E0E9496
:105CD0006A7902C00E94EC2A8C2F0E94F42CCF5FBC
:105CE0000F5F1F4FC63008F4BDCFFF2019F083E0CF
:105CF0000E94E72C0E94BD2DC82F0E94B02C8C2F33
:105D000099279F938F938BE999E09F938F930BEF44
:105D100012E11F930F93E0914204F091430409951F
:105D20008DB79EB706968DBFEE2021F40E94362DCA
:105D3000882399F484EB99E09F938F931F930F939B
:105D4000E0914204F091430409950E94762D0E944F
:105D5000582D0F900F900F900F901092310690E0F9
:105D6000E3EBF6E0CFE08081349618160CF49F5FE9
:105D7000C150C7FFF8CF90933106892F99279F9381
:105D80008F9387EA96E09F938F9385ED99E09F9399
:105D90008F931F930F93E0914204F0914304099570
:105DA0008DB79EB708968DBF86EF99E09F938F932E
:105DB0001F930F93E0914204F091430409950F90D3
:105DC0000F900F900F90CF911F910F91FF90EF9038
:105DD000DF900895982F2FB7F8943998389A88B1A2
:105DE000836088B98091B9008C7F8093B9008AE282
:105DF0008093B80010927D0210927B0210927A027A
:105E0000992379F0ECEFF6E08BE010821182128298
:105E1000138214821582168217828150389687FF6A
:105E2000F4CF78942FBF089510927D0284E9809377
:105E3000BC0080E88093BC001092BD001092BA00B4
:105E40001092BB001092B9001092B8001092790223
:105E500080E00E94EA2E1092BB0085E88093BC008F
:105E60008091770282608093770208951F920F924B
:105E70000FB60F9211242F933F934F935F938F93FD
:105E80009F93EF93FF9380917D02282F3327442720
:105E900055278F5F80937D02F9012731310508F086
:105EA000C2C2EE59FF4F0C945C7981E08093790275
:105EB00009C080917B028C3090F480917B028F5FCF
:105EC00080937B0280917B02E82FFF27EE0FFF1F5C
:105ED000EE0FFF1FEA55F94F8585181654F780918C
:105EE0007B028C3070F01092760210927502109244
:105EF0007B0285E080937D0280917A02880F8D5A23
:105F000004C080917B02880F8E5A8093BB0085E885
:105F10007FC280917B02E82FFF2783E0EE0FFF1FF7
:105F20008A95E1F7E450F94F81818093BB0085E8C1
:105F30008093BC0080917B02E82FFF27EE0FFF1FAC
:105F4000EE0FFF1FEE0FFF1FE450F94F808180FF1F
:105F500091C080917B02E82FFF27EE0FFF1FEE0F0D
:105F6000FF1FEE0FFF1FE450F94F8281882329F0B5
:105F700080913106873008F46CC28091750290914F
:105F80007602892B09F065C28091730290917402A8
:105F9000892B09F05EC26EC080917B0221E030E067
:105FA00002C0220F331F8A95E2F78091730290910D
:105FB000740228233923232B79F080917B02E82F68
:105FC000FF27EE0FFF1FEE0FFF1FEE0FFF1FE45026
:105FD000F94F80E184830DC080917B02E82FFF2779
:105FE000EE0FFF1FEE0FFF1FEE0FFF1FE450F94FE4
:105FF000148280917B02E82FFF2753E0EE0FFF1FF2
:106000005A95E1F7E450F94F8481282F332743E074
:10601000220F331F4A95E1F780917B02E82FFF277B
:1060200093E0EE0FFF1F9A95E1F7E450F94F82815C
:106030008770822B8093BB0085E88093BC00209101
:106040007B0281E090E002C0880F991F2A95E2F759
:10605000209175023091760282239323892B51F08F
:1060600084EF96E0909381028093800288E0809391
:106070008202EFC184E089C1E0918002F091810247
:1060800081918093BB0085E88093BC00F0938102EE
:10609000E093800280918202815080938202882363
:1060A00009F4D7C183E071C18091B900803351F503
:1060B00080917E02882329F480917B028F5F8093F8
:1060C0007E0280917B02E82FFF2783E0EE0FFF1F07
:1060D0008A95E1F7E450F94F838199278F77907083
:1060E0008F3791057CF480917B02E82FFF27EE0F1C
:1060F000FF1FEE0FFF1FEE0FFF1FE450F94F8381CC
:106100008F5F838310927D0284E98093BC008AE0D4
:1061100090E0909393018093920180917B028F5F36
:1061200080937B0210927D026DC18091B900803412
:10613000C9F180917A02E82FFF27EE0FFF1FEE0FC3
:10614000FF1FEE0FFF1FE450F94F83818F7783838A
:1061500080917A028F5F80937A0280917A028C30EC
:10616000A0F010927A021092740210927302809141
:106170007F028F5F80937F028C3038F010927F0215
:10618000809177028D7F8093770280917702816082
:106190008093770210927D0284E98093BC00109274
:1061A000790273C080917A02E82FFF27EE0FFF1F5C
:1061B000EE0FFF1FEE0FFF1FE450F94F8381806841
:1061C000838380917A02E82FFF27EE0FFF1FEE0FE7
:1061D000FF1FEE0FFF1FE450F94F808180FF2FC09B
:1061E00080917A02E82FFF2753E0EE0FFF1F5A95A8
:1061F000E1F7E450F94F84819927009751F04097D7
:10620000D9F584EF96E0909381028093800288E034
:1062100031C080917A02992743E0880F991F4A95EF
:10622000E1F78F5F984F9093810280938002909165
:106230007A0280917F029817E1F483E01BC080917D
:106240007A02992733E0880F991F3A95E1F78F5F1B
:10625000984F90938102809380028091770281FD14
:1062600006C090917A0280917F02981711F482E023
:1062700001C081E08093820280918202813011F41A
:1062800085E801C085EC8093BC0080917E028093FC
:10629000780210927E02DDC0E0918002F0918102CE
:1062A0008091BB0080838091800290918102019651
:1062B000909381028093800280918202815080932A
:1062C0008202823010F085EC5DC0813011F485E8E7
:1062D00059C08091770281FF2DC08091F50280FD29
:1062E0001DC080917A02E82FFF2723E0EE0FFF1FE9
:1062F0002A95E1F7E450F94F86818A3F79F480913D
:106300007A02E82FFF2793E0EE0FFF1F9A95E1F73F
:10631000E450F94F8081816080830CC080917A02C3
:10632000E82FFF2783E0EE0FFF1F8A95E1F7E45087
:10633000F94F108280917A028F5F80937A02809168
:106340007A028C30A0F010927A02109274021092AD
:10635000730280917F028F5F80937F028C3038F0D0
:1063600010927F02809177028D7F80937702109246
:106370007D0284E98093BC008091770281608093E4
:10638000770265C08093BC0086E080937D0261C087
:1063900088E9BBCD80917C02880F805FB6CD80916B
:1063A0007C0299278130910561F0823091051CF4BF
:1063B000892B21F04EC0029739F04BC08091130118
:1063C000A4CD80911201A1CD809111019ECD80E8D4
:1063D0009CCD10927D0284E98093BC0010927902DA
:1063E0008AE090E0909393018093920180917C02E7
:1063F000823088F480917C028F5F80937C0282E1FE
:1064000080937D02809177028E7F8093770285EA68
:106410008093BC001EC010927C0280917702816044
:106420008093770216C010927D0284E98093BC00AD
:10643000809177028160809377028AE090E0909368
:1064400093018093920110927B0210927A02109233
:106450007902FF91EF919F918F915F914F913F91C1
:106460002F910F900FBE0F901F9018951F93CF93F1
:10647000DF93182F80912703882321F480910E0247
:10648000882319F081E090E097C01D3008F092C099
:106490001123B1F0E12FFF2723E0EE0FFF1F2A9514
:1064A000E1F7E450F94F35978081359688230CF059
:1064B00081C03897808180FD03C083E090E07CC07C
:1064C0008091F406823019F084E090E075C067E0B6
:1064D00070E084EF96E00E94C72A9091FB0689172E
:1064E00019F085E090E068C080ED97E00E942117E8
:1064F000EC018091770280FD05C0CE010E942A1731
:106500008823B9F3112319F48FEF90E00BC0212FEA
:1065100033272150304081E090E002C0880F991F5E
:106520002A95E2F79093760280937502A1E0B0E09D
:10653000ECEFF6E040E050E06BE0CD01042E02C04D
:10654000880F991F0A94E2F7209175023091760224
:1065500082239323892B11F01182128261504F5FA5
:106560005F4F389667FFE9CF10927B0210927D0251
:10657000809177028E7F8093770285EA8093BC00BA
:106580008091770280FD05C0CE010E942A178823E2
:10659000B9F38091750290917602892B29F0CE0192
:1065A0000E942A17882311F3809175029091760238
:1065B000009711F082E090E0DF91CF911F91089554
:1065C0000F931F93CF93DF93982F809127038823F6
:1065D00021F480910E02882319F081E090E092C0AE
:1065E0009D30A0F4992319F486E090E08BC0C92F68
:1065F000DD27FE0133E0EE0FFF1F3A95E1F7E4508F
:10660000F94F35978081359687FD03C082E090E091
:1066100079C03897808180FD03C083E090E072C02C
:1066200080ED97E00E9421178C018091770280FD18
:1066300005C0C8010E942A178823B9F3219721E0D9
:1066400030E0C90102C0880F991FCA95E2F7909304
:10665000740280937302D901ECEFF6E040E050E061
:106660006BE0CD01042E02C0880F991F0A94E2F757
:10667000209173023091740282239323892B11F0AD
:106680001182128261504F5F5F4F389667FFE9CFEA
:1066900010927A021092F4061092FB0610927D027C
:1066A000809177028E7F8093770285EA8093BC0089
:1066B0008091770280FD05C0C8010E942A178823B7
:1066C000B9F38091730290917402892B29F0C8016B
:1066D0000E942A17882311F38091F406823019F062
:1066E00084E090E00FC067E070E084EF96E00E94E5
:1066F000C72A9091FB06891719F085E090E002C047
:1067000080E090E0DF91CF911F910F91089589E192
:10671000A1E9B7E0EDE5F7E011821082329611961B
:106720001C921E921296815087FFF6CF109294030E
:10673000109293031092960310929503109298036F
:106740001092970308951F920F920FB60F92112483
:106750000F931F932F933F934F935F936F937F9369
:106760008F939F93AF93BF93CF93DF93EF93FF9359
:106770008091980682FDCFC040918600509187009D
:106780008091840290918502481B590B809186006C
:10679000909187009093850280938402CA018D5462
:1067A0009440A0918602B0918702835F9A4178F469
:1067B0008091860280935C07149714F010929401E4
:1067C00081E090E0909387028093860207C2AD300B
:1067D000B1050CF003C2CA018B5F9040845B91400D
:1067E00008F074C0425D5140FD01EA0FFB1FE35AFF
:1067F000F84F80819181FA01E81BF90BCF01F7FF77
:1068000003C0909581959F4F06975CF4809130036B
:10681000883C20F480913003865F01C088EC80932F
:106820003003FD01EA0FFB1FE35AF84F808191818D
:106830009C01220F331F280F391F240F351F37FFEC
:1068400002C02D5F3F4FE901D595C795D595C795F6
:10685000CA0101968C179D0714F4219706C0415078
:106860005040C417D5070CF4219680913003833C27
:10687000E0F08D010A0F1B1FF801E35AF84F8081E9
:1068800091819E01281B390BC90163E070E00E94D1
:10689000D578CB01880F991F860F971F0F56184F79
:1068A000D80111969C938E9307C0AA0FBB1FAF56B9
:1068B000B84F11961C921E92E0918602F0918702C9
:1068C000EE0FFF1FE35AF84FD183C0832091860259
:1068D000309187022F5F3F4F3093870220938602CB
:1068E00080910201843108F079C12530310511F41D
:1068F0005D9A01C05D9880918602909187028630F2
:10690000910511F45C9A01C05C98079711F45B9AA9
:1069100065C15B9863C1409186005091870080916A
:10692000880290918902481B590B809186009091B2
:1069300087009093890280938802CA018D54944005
:106940006091F202835F9A4108F07AC060938302FB
:1069500080918302843008F453C090915C07809149
:106960008302981709F04CC05091F3025B3008F491
:106970003FC0109294011092F20240E05F31C0F0EB
:10698000E42FFF27EE0FFF1F9F0122543D4FDF0131
:10699000A35AB84F8D919C91D9018D939C93DF019F
:1069A000AF56B84F8D919C91E852FD4F91838083F3
:1069B000E42FFF27EE0FFF1F9F01235A384FDF01FF
:1069C000A657BD4F8D919C91D90111969C938E93A2
:1069D000DF01AC55BD4F8D919C91EF56F84F9183DF
:1069E0008083842F8F5F482F8D3040F28093F20296
:1069F0008091F3028F3FB9F08F5F8093F30213C051
:106A00008091F302853620F08AE08093F30202C081
:106A10001092F302809102018A3011F0843110F05B
:106A2000289A01C0289881E08093F2028091270380
:106A3000882309F0D3C08091830280935C07CEC085
:106A40006D3008F0A3C0CA018B5F9040845B914019
:106A500008F07EC0425D5140E62FFF27EE0FFF1F7A
:106A6000E657FD4F80819181FA01E81BF90BCF01B8
:106A700005960B97B0F48091F3028A3120F0809153
:106A80003003865F05C08B3028F0809130038E5F25
:106A90008093300380913003893C18F088EC809318
:106AA0003003E62FFF27EE0FFF1FE657FD4F8081D3
:106AB00091819C01220F331F280F391F240F351F8E
:106AC00037FF02C02D5F3F4FE901D595C795D5959A
:106AD000C795CA0101968C179D0714F4219706C02B
:106AE00041505040C417D5070CF4219680913003D3
:106AF0008E3BD8F0E62FFF27EE0FFF1FDF01A657D2
:106B0000BD4F8D919C919E01281B390BC90163E0FB
:106B100070E00E94D578CB01880F991F860F971FD0
:106B2000EC55FD4F9183808308C0E62FFF27EE0FC1
:106B3000FF1FEC55FD4F118210828091F202E82F69
:106B4000FF27EE0FFF1FE657FD4FD183C08309C01B
:106B5000809102018A3011F0843110F0289A01C02E
:106B6000289880910201843188F48091F202853066
:106B700011F45D9A05C05D98863011F45C9A05C0E9
:106B80005C98873011F45B9A01C05B988091F202A7
:106B9000843120F48F5F8093F20220C08431F1F4BD
:106BA000809102018A3011F0843110F0289A01C0DE
:106BB00028988EE18093F2022CE0C1E9D7E0AEEB99
:106BC000B2E0EDE5F7E08D919D919183808332965F
:106BD000198218822296215027FFF5CFFF91EF915D
:106BE000DF91CF91BF91AF919F918F917F916F91E5
:106BF0005F914F913F912F911F910F910F900FBE79
:106C00000F901F901895EF92FF920F931F93809112
:106C10004E069927880F991F880F991F7C0100271E
:106C2000F7FC0095102F8091820390918303A0912F
:106C30008403B0918503BC01CD01A80197010E9496
:106C40000A793093DE052093DD0580917A039091D7
:106C50007B03A0917C03B0917D03BC01CD01A80111
:106C600097010E940A793093E0052093DF05809117
:106C700017089091180897FD039695958795959517
:106C800087959093E2058093E10580912708909184
:106C9000280897FD039695958795959587959093E8
:106CA000E4058093E30580919303909194032091F0
:106CB0004E0230914F02821B930B9093E605809316
:106CC000E5058091220390912303A0912403B091C4
:106CD0002503BC01CD0125E030E040E050E00E94FA
:106CE0000A793093E8052093E70580914802909156
:106CF00049029093EA058093E9058091E201909121
:106D0000E3019093EE058093ED0580911E01909133
:106D10001F019093F0058093EF0580913003992730
:106D20009093F2058093F1058091230890912408B7
:106D3000A0912508B091260820919A0130919B01DD
:106D400040919C0150919D01BC01CD010E940A79A6
:106D50003093F4052093F3058091FD0699279093D5
:106D6000F6058093F5058091050799279093F8051E
:106D70008093F70580910D0799279093FA058093EA
:106D8000F9058091150799279093FC058093FB05E1
:106D90008091290290912A0290930606809305061D
:106DA0008091A8089091A90890930A0680930906FB
:106DB0008091AC089091AD0890930C0680930B06DF
:106DC00080911E0390911F03A0912003B091210395
:106DD000BC01CD0125E030E040E050E00E940A799E
:106DE00030930E0620930D0680914003909141034D
:106DF00090931406809313068091AE089927909380
:106E000018068093170680910B0490910C049093C0
:106E10001A06809319068091090490910A049093B0
:106E20001C0680931B0680915B04882321F48091CB
:106E30005C04882321F08091DC05816003C080918F
:106E4000DC058E7F8093DC051F910F91FF90EF9002
:106E500008951F93CF93DF93182FEB0180912703A1
:106E60008823A1F411501F3F89F0D0933002C093C2
:106E70002F0280912F0290913002892BD1F7CE0101
:106E80008C0F9D1F0E943617115078F7DF91CF911C
:106E90001F910895CF93DF93809102018D3011F4FB
:106EA0000E942F1B10927A008091520290915302FF
:106EB0009093DE078093DD078091500290915102FC
:106EC0009093CF078093CE0780914E0290914F020E
:106ED00090931D0880931C0820914A0230914B0228
:106EE000C901880F991F880F991F820F931F820F66
:106EF000931F909318088093170820914C023091AB
:106F00004D02C901880F991F880F991F820F931F87
:106F1000820F931F90932808809327088FEC80930B
:106F20007A00A1E3B3E0C7E3D6E097E08991E82FC8
:106F3000FF27EE0FFF1FE35AF84F0190F081E02D7D
:106F4000E158FF4F1E161F061CF0E0E0F0E005C000
:106F5000EF3FF10514F0EFEFF0E08C91282F33278D
:106F6000E217F30714F4815004C02E173F0714F4FE
:106F70008F5F8C939150119697FFD8CF80917306B5
:106F80009927AA27BB27BC01CD0124EC39E040E0BA
:106F900050E00E949678DC01CB018093DA01909357
:106FA000DB01A093DC01B093DD0180917406992789
:106FB000AA27BB27BC01CD010E949678DC01CB013A
:106FC0008093D6019093D701A093D801B093D901B3
:106FD000DF91CF910895A0E0B0E0E1EFF7E30C94EA
:106FE0002B79882EC0E0D0E07E016E0110925B0408
:106FF000469AD0938E03C0938D03D0938C03C09395
:107000008B03D0938803C0938703D0939803C093D6
:107010009703D0939603C0939503D0939403C093A2
:1070200093031092C2011092C101109242020E9479
:107030004A3784E690E00E9443170E944A378091C5
:107040003F0680FF10C08091140190911501875B6D
:10705000934038F480911401909115018E5E924016
:1070600010F40E94D41A0FE18AE090E00E944317C6
:1070700080914E0290914F02C80FD91F8091520209
:1070800090915302E80EF91E8091500290915102A6
:10709000C80ED91E015007FFE7CF9701205F3F4F71
:1070A0003695279536952795309398032093970327
:1070B000C6014096969587959695879590939603E9
:1070C000809395036096F5E0D695C795FA95E1F71C
:1070D000D0939403C093930390939203809391036E
:1070E0003093900320938F03882009F441C080914E
:1070F00017089091180897FF03C0909581959F4FAE
:107100006CE070E00E94D5789B0170938E036093D1
:107110008D03809127089091280897FF03C09095D0
:1071200081959F4F6CE070E00E94D57870938C033E
:1071300060938B0380912406909125069093880399
:1071400080938703B90184E090E00E94AB2C6091AA
:107150008B0370918C0386E090E00E94AB2C6091D1
:1071600087037091880388E090E00E94AB2C65C093
:1071700084E090E00E94A62C90938E0380938D0370
:1071800086E090E00E94A62C90938C0380938B0362
:1071900088E090E00E94A62C9C0190938803809345
:1071A000870380918D0390918E038150984050F415
:1071B00080918B0390918C038150984018F421505A
:1071C0003440D8F187E19AE09F938F938BEF92E15F
:1071D0009F938F93E0914204F0914304099580912D
:1071E00017089091180897FF03C0909581959F4FBD
:1071F0006CE070E00E94D57870938E0360938D03ED
:10720000809127089091280897FF03C09095819559
:107210009F4F6CE070E00E94D57870938C03609370
:107220008B03809124069091250690938803809388
:1072300087030F900F900F900F901092DE0710921F
:10724000DD071092CF071092CE0710921D08109202
:107250001C0884E690E00E94431780914A029091B6
:107260004B029C01220F331F220F331F280F391F9F
:10727000280F391F309318082093170880914C026B
:1072800090914D028C01000F111F000F111F080F6C
:10729000191F080F191F10932808009327088091C1
:1072A0004E06C82EDD24EE24FF24442737FD4095EA
:1072B000542FC701B6010E9496784B015C01609380
:1072C00082037093830380938403909385039801D2
:1072D000442737FD4095542FC701B6010E94967888
:1072E000DC01CB0180937A0390937B03A0937C0312
:1072F000B0937D0380925E0390925F03A09260033F
:10730000B09261038093560390935703A093580360
:10731000B0935903109252031092530310925403E6
:10732000109255038091160190911701A0911801B8
:10733000B09119019093270680932606109241027E
:1073400010924002109242031092430310924403A1
:10735000109245038091E2019091E30190934103E3
:107360008093400384E690E09093DF018093DE01F8
:107370000E94BF6382E390E09093300280932F02DB
:10738000809173069927AA27BB27BC01CD0124EC65
:1073900039E040E050E00E949678DC01CB0188564D
:1073A000954CAF4FBF4F8093DA019093DB01A093D0
:1073B000DC01B093DD01809174069927AA27BB27D1
:1073C000BC01CD010E949678DC01CB018856954C1A
:1073D000AF4FBF4F8093D6019093D701A093D801B0
:1073E000B093D90110929F0110929E018091E20109
:1073F0009091E301AA2797FDA095BA2F20919A01B9
:1074000030919B0140919C0150919D01BC01CD01A7
:107410000E949678DC01CB01809323089093240886
:10742000A0932508B093260810923B0310923A03CC
:1074300081E0809301010E94B0688091F502846030
:107440008093F5028FEF8093A3081092A40880E246
:107450008093A508C1E3D3E0A7E3B6E007E08D91F0
:10746000E82FFF27EE0FFF1FE35AF84F808191812D
:1074700081588993015007FFF2CF84E6809330034F
:1074800080912D02882311F0469A579A8091970394
:107490009091980380569940815C9B4228F080919E
:1074A0005B04816080935B048091950390919603C7
:1074B00080569940815C9B4228F080915B048260F9
:1074C00080935B0480919303909194038C5291403C
:1074D0008957954028F080915B04846080935B0419
:1074E00080918D0390918E038C529140835C9140EA
:1074F00028F080915B04886080935B0480918B030B
:1075000090918C038C529140835C914028F0809143
:107510005B04806180935B04809187039091880372
:10752000805092408355914028F080915B048062A6
:1075300080935B0486E48093D501ECE0CDB7DEB7A1
:107540000C944779A3E1B0E0E8EAFAE30C942579DA
:10755000809193039091940320914E0230914F02B9
:10756000821B930B90931D0880931C0880915802F6
:107570009091590297FD07969C0113E03595279548
:107580001A95E1F73093DE072093DD0780915602CC
:107590009091570297FD0796B3E095958795BA9518
:1075A000E1F79093CF078093CE073093E9072093BC
:1075B000E8079093E1078093E00780911708909186
:1075C0001808AC01440F551F480F591F20914A025B
:1075D00030914B02C901880F991F880F991F820FA4
:1075E000931F820F931F480F591F57FF02C04D5F13
:1075F0005F4F55954795559547955093180840937B
:1076000017088091270890912808AC01440F551F56
:10761000480F591F20914C0230914D02C901880F2B
:10762000991F880F991F820F931F820F931F480F76
:10763000591F57FF02C04D5F5F4F559547955595B0
:107640004795509328084093270820914A0230918B
:107650004B02C901880F991F880F991F820F931F32
:10766000820F931F9C01442737FD4095542F809132
:10767000720390917303A0917403B0917503820F0C
:10768000931FA41FB51F8093720390937303A0935D
:107690007403B093750320914C0230914D02C901DF
:1076A000880F991F880F991F820F931F820F931FB6
:1076B0009C01442737FD4095542F80916E03909193
:1076C0006F03A0917003B0917103820F931FA41FE9
:1076D000B51F80936E0390936F03A0937003B093D4
:1076E00071038091F2079091F30720914A02309143
:1076F0004B02820F931F9093F3078093F2078091C0
:107700001F089091200820914C0230914D02820F69
:10771000931F9093200880931F0880918903909174
:107720008A03019690938A038093890380912406AB
:10773000909125062091870330918803821B930B3B
:107740009C01442737FD4095542F80916A03909106
:107750006B03A0916C03B0916D03820F931FA41F64
:10776000B51F80936A0390936B03A0936C03B0934F
:107770006D038FEC80937A001092100120915A03D0
:1077800030915B0340915C0350915D0329873A87F8
:107790004B875C8729543B46414050402CF028E4FD
:1077A0003BE641E050E00DC089859A85AB85BC85FC
:1077B000885B9449AE4FBF4F4CF428EB34E94EEF51
:1077C0005FEF2D833E834F83588708C089859A8554
:1077D000AB85BC858D839E83AF83B8872091620380
:1077E0003091630340916403509165032D873E8778
:1077F0004F87588B29543B46414050402CF028E499
:107800003BE641E050E00DC08D859E85AF85B8898F
:10781000885B9449AE4FBF4F4CF428EB34E94EEFF0
:107820005FEF29833A834B835C8308C08D859E85F7
:10783000AF85B88989839A83AB83BC83A0911C08E8
:10784000B0911D08BB8BAA8BFD01CF01AA2797FD24
:10785000A095BA2FA0905203B0905303C090540348
:10786000D0905503A80EB91ECA1EDB1EA09252036B
:10787000B0925303C0925403D0925503E090230872
:10788000F09024080091250810912608E80EF91EB2
:107890000A1F1B1FE0922308F0922408009325087A
:1078A00010932608F0911003F98BFF2309F098C17B
:1078B00080910F03882309F093C180913F0686FFD2
:1078C0008FC18091CE079091CF07AA2797FDA095F1
:1078D000BA2FBC01CD0129813A814B815C810E9484
:1078E00096789B01AC0197FF04C02150384F4F4F51
:1078F0005F4FBBE05595479537952795BA95D1F7DA
:107900008091C101682E772488249924CA01B90185
:10791000A40193010E949678DC01CB018093A3031C
:107920009093A403A093A503B093A603B7FF04C04C
:107930008150904FAF4FBF4F1C012D01ACE05594CB
:10794000479437942794AA95D1F72092A3033092B5
:10795000A4034092A5035092A6038091DD07909165
:10796000DE07AA2797FDA095BA2FBC01CD012D8176
:107970003E814F8158850E94967897FF04C06150E0
:10798000784F8F4F9F4FFBE095958795779567953B
:10799000FA95D1F7A40193010E949678DC01CB01FE
:1079A0008093A7039093A803A093A903B093AA037D
:1079B000B7FF04C08150904FAF4FBF4F9C01AD0146
:1079C000ECE05595479537952795EA95D1F72093A3
:1079D000A7033093A8034093A9035093AA0380916F
:1079E000A3039091A4039093C6078093C507809149
:1079F000A7039091A8039093CA078093C9072219FF
:107A00003309440955092093A7033093A8034093F1
:107A1000A9035093AA03E20EF31E041F151FE09260
:107A20002308F092240800932508109326088091DB
:107A3000C0018823B1F457FF04C02F5F3F4F4F4F61
:107A40005F4F5595479537952795A21AB30AC40AF3
:107A5000D50AA0925203B0925303C0925403D0921D
:107A600055032A893B8979010027F7FC0095102FDF
:107A70008091A7039091A803A091A903B091AA03B4
:107A8000E80EF91E0A1F1B1FC801B70129813A81A0
:107A90004B815C810E9496789B01AC0197FF04C0EA
:107AA0002150384F4F4F5F4F6BE0559547953795B5
:107AB00027956A95D1F78091C201A82EBB24CC24CA
:107AC000DD24CA01B901A60195010E949678DC0166
:107AD000CB0180939B0390939C03A0939D03B09351
:107AE0009E03B7FF04C08150904FAF4FBF4F3C0182
:107AF0004D013CE095948794779467943A95D1F73B
:107B000060929B0370929C0380929D0390929E03CF
:107B1000C801B7012D813E814F8158850E9496781A
:107B200097FF04C06150784F8F4F9F4F2BE0959582
:107B30008795779567952A95D1F7A60195010E94BB
:107B40009678DC01CB0180939F039093A003A093D0
:107B5000A103B093A203B7FF04C08150904FAF4F71
:107B6000BF4FAC01BD018CE0759567955795479562
:107B70008A95D1F740939F035093A0036093A1038C
:107B80007093A2032A893B8937FF03C03095219562
:107B90003F4F21343105E4F1D401C30197FE07C002
:107BA000B095A095909581959F4FAF4FBF4F81386D
:107BB0009105A105B10584F4DB01CA0177FF07C077
:107BC000B095A095909581959F4FAF4FBF4F81384D
:107BD0009105A105B105E4F081E080933C0318C054
:107BE0001092CA071092C9071092C6071092C507D3
:107BF00010929F031092A0031092A1031092A2036F
:107C000010929B0310929C0310929D0310929E036E
:107C100080919F039091A003A091A103B091A20332
:107C2000BC01CD0124E630E040E050E00E940A793A
:107C3000E0909B03F0909C03E21AF30AF092DC07B9
:107C4000E092DB0780919B0390919C03A0919D03A0
:107C5000B0919E03BC01CD0124E630E040E050E04D
:107C60000E940A79DA01C90120919F033091A00393
:107C70008C01021B130B1093D1070093D007809146
:107C80009A0190919B01A0919C01B0919D01BC0132
:107C9000CD0128E631E040E050E00E949678209146
:107CA0002308309124084091250850912608261772
:107CB00037074807590764F0261B370B480B590B49
:107CC00020932308309324084093250850932608D6
:107CD00020912308309124084091250850912608CE
:107CE00057FF0CC0260F371F481F591F209323082A
:107CF0003093240840932508509326086091CE07BE
:107D00007091CF076E0D7F1D9B01442737FD409575
:107D1000542F8091560390915703A0915803B0912E
:107D20005903820F931FA41FB51F8093560390938E
:107D30005703A0935803B093590380911503909172
:107D40001603681B790BCB01AA2797FDA095BA2FC4
:107D500029853A854B855C85820F931FA41FB51F2B
:107D600080935A0390935B03A0935C03B0935D03ED
:107D7000C090D601D090D701E090D801F090D90101
:107D8000C816D906EA06FB06C4F488EA91E6A0E024
:107D9000B0E08C199D09AE09BF0980935A039093F6
:107DA0005B03A0935C03B0935D03809356039093B1
:107DB0005703A0935803B093590322273327A901EF
:107DC0002C193D094E095F0980915A0390915B037C
:107DD000A0915C03B0915D0382179307A407B507D8
:107DE000B4F4D701C601885A9146A040B0408093B0
:107DF0005A0390935B03A0935C03B0935D0380935D
:107E0000560390935703A0935803B093590360917E
:107E1000DD077091DE07600F711F9B01442737FD5E
:107E20004095542F80915E0390915F03A091600371
:107E3000B0916103820F931FA41FB51F80935E034F
:107E400090935F03A0936003B09361038091130349
:107E500090911403681B790BCB01AA2797FDA0957D
:107E6000BA2F2D853E854F855889820F931FA41FF9
:107E7000B51F8093620390936303A0936403B09350
:107E80006503E090DA01F090DB010091DC011091D4
:107E9000DD01E816F9060A071B07C4F488EA91E633
:107EA000A0E0B0E08E199F09A00BB10B8093620394
:107EB00090936303A0936403B093650380935E0380
:107EC00090935F03A0936003B0936103222733274D
:107ED000A9012E193F09400B510B8091620390912B
:107EE0006303A0916403B091650382179307A4070D
:107EF000B507B4F4D801C701885A9146A040B040F4
:107F00008093620390936303A0936403B09365032B
:107F100080935E0390935F03A0936003B09361032B
:107F20008091520390915303A0915403B091550353
:107F30008093660390936703A0936803B0936903EB
:107F40008091620390916303A0916403B0916503F3
:107F50008093820390938303A0938403B09385035B
:107F600080915A0390915B03A0915C03B0915D03F3
:107F700080937A0390937B03A0937C03B0937D035B
:107F800080915E0390915F03A0916003B0916103C3
:107F900080937E0390937F03A0938003B09381032B
:107FA0008091560390915703A0915803B0915903C3
:107FB0008093760390937703A0937803B09379032B
:107FC00080911C0190911D0197FD079603E0959506
:107FD00087950A95E1F79093DE078093DD078091FE
:107FE0001A0190911B0197FD079613E095958795CF
:107FF0001A95E1F79093CF078093CE0780915202B4
:10800000909153020F9734F488E19CEF9093DE0730
:108010008093DD078091520290915302079734F4C8
:1080200080E398EF9093DE078093DD0720910201B3
:108030002A30A9F48091520290915302835F9340B9
:1080400034F088EE93E09093DE078093DD07809113
:108050005202909153028A5F9340DCF014C08091E9
:10806000520290915302815D974034F088EE93E084
:108070009093DE078093DD07809152029091530226
:10808000805E974034F080ED97E09093DE07809318
:10809000DD0780915002909151020F9734F488E1EE
:1080A0009CEF9093CF078093CE07809150029091E0
:1080B0005102079734F480E398EF9093CF078093B1
:1080C000CE072A30A9F48091500290915102835F2B
:1080D000934034F088EE93E09093CF078093CE07DF
:1080E00080915002909151028A5F9340DCF014C05D
:1080F0008091500290915102815D974034F088EE5A
:1081000093E09093CF078093CE0780915002909197
:108110005102805E974034F080ED97E09093CF0756
:108120008093CE076091CC01662309F4AFC04091E3
:108130001C0150911D018091AB039091AC03481B31
:10814000590B5093B2034093B10320911C0130911D
:108150001D01280F391F37FF02C02F5F3F4F359594
:1081600027953093AC032093AB03413851051CF0A5
:1081700080E890E005C040585F4F34F480E89FEFFE
:108180009093B2038093B10340911A0150911B0167
:108190008091AD039091AE03481B590B5093B003EF
:1081A0004093AF0320911A0130911B01280F391F12
:1081B00037FF02C02F5F3F4F359527953093AE03B1
:1081C0002093AD03413851051CF080E890E005C0D4
:1081D00040585F4F34F480E89FEF9093B003809352
:1081E000AF03462F55278091B1039091B203849F2E
:1081F000B001859F700D949F700D11249B0177FF36
:1082000002C0215F3F4FF4E035952795FA95E1F7DD
:108210008091DD079091DE07820F931F9093DE0718
:108220008093DD078091AF039091B003849FD001CC
:10823000859FB00D949FB00D1124AD019D01B7FF36
:1082400002C0215F3F4FE4E035952795EA95E1F7BD
:108250008091CE079091CF07820F931F9093CF0705
:108260008093CE0780911C0190911D01860F971F6E
:1082700090931D0180931C0180911A0190911B0124
:10828000840F951F90931B0180931A010091E007C2
:108290001091E1078091C5079091C607101611064D
:1082A0005CF59C0197FF04C022273327281B390B5C
:1082B000C901AA2797FDA095BA2F2091C0013327A5
:1082C00044275527BC01CD010E9496789B01AC0143
:1082D00097FF04C0215C3F4F4F4F5F4F76E05595AD
:1082E0004795379527957A95D1F78091DB0790913F
:1082F000DC07820F931F27C097FF03C090958195DD
:108300009F4FAA2797FDA095BA2F2091C001332730
:1083100044275527BC01CD010E9496789B01AC01F2
:1083200097FF04C0215C3F4F4F4F5F4F66E055956C
:108330004795379527956A95D1F78091DB079091FE
:10834000DC07821B930B9093DC078093DB07E090A4
:10835000E807F090E9078091C9079091CA071E14B9
:108360001F045CF59C0197FF04C022273327281BBC
:10837000390BC901AA2797FDA095BA2F2091C001FA
:10838000332744275527BC01CD010E9496789B01D5
:10839000AC0197FF04C0215C3F4F4F4F5F4F96E009
:1083A00055954795379527959A95D1F78091D007A0
:1083B0009091D107820F931F27C097FF03C090951C
:1083C00081959F4FAA2797FDA095BA2F2091C001B4
:1083D000332744275527BC01CD010E9496789B0185
:1083E000AC0197FF04C0215C3F4F4F4F5F4F86E0C9
:1083F00055954795379527958A95D1F78091D00760
:108400009091D107821B930B9093D1078093D00753
:1084100080913F0687FF44C0B989BB2309F040C063
:1084200080910F038823E1F5E1E0EE16E1E0FE061E
:108430004CF08091DD079091DE078E0D9F1D8050DE
:1084400091400DC0F0E0EF16FFEFFF0664F480915D
:10845000DD079091DE078E0D9F1D80509F4F9093FA
:10846000DE078093DD0721E0013012074CF0809198
:10847000CE079091CF07800F911F805091400CC084
:108480003FEF0030130764F48091CE079091CF073F
:10849000800F911F80509F4F9093CF078093CE07FE
:1084A000E2E1CD5E0C94417980912703882301F5A8
:1084B0008091F5028C7F8093F502A0E6B4E0ECEFAA
:1084C000F6E09BE080910E02882309F48C938D9155
:1084D000818312829150389697FFF4CF80910E02DB
:1084E000882359F080910E02815080930E0205C0BE
:1084F0008091F50281608093F50280917902882352
:1085000019F010927902089580937B0280937D0286
:10851000809177028E7F8093770285EA8093BC00FA
:108520000895CF93DF93A1E3B3E0C7E3D6E057E02C
:108530008991E82FFF27EE0FFF1FE35AF84F0190B4
:10854000F081E02DE158FF4FEF3FF10521F01CF0E5
:10855000EFEFF0E004C0F7FF02C0E0E0F0E04C9184
:10856000242F3327E217F307A9F0CF01821B930BC7
:1085700097FD03969595879595958795242F280FB8
:108580002C93822F9927E817F90714F4215001C082
:108590002F5F2C935150119657FFCACF80914106FF
:1085A000883F38F0EFEFF0E0E81BF109EF5CFC4F9B
:1085B00080818093D2018091D201882329F0843672
:1085C00018F084E68093D20180914306883F38F00A
:1085D000EFEFF0E0E81BF109EF5CFC4F8081809346
:1085E000D0018091D001882329F0843618F084E6E8
:1085F0008093D00180915006883F38F0EFEFF0E093
:10860000E81BF109EF5CFC4F80818093CB018091E6
:10861000CB018B3010F48AE002C08F3F11F48093BD
:10862000CB0180917D06883F38F0EFEFF0E0E81B4A
:10863000F109EF5CFC4F80818093F4078091F4078F
:10864000823010F481E002C08F3F11F48093F40770
:1086500080917F06883F38F0EFEFF0E0E81BF109EA
:10866000EF5CFC4F808180931A0880911A08823059
:1086700010F481E002C08F3F11F480931A088091BA
:108680006A06883F38F0EFEFF0E0E81BF109EF5C95
:10869000FC4F80818093F10780916B06883F38F012
:1086A000EFEFF0E0E81BF109EF5CFC4F8081809375
:1086B000CB0780916C06883F38F0EFEFF0E0E81BC5
:1086C000F109EF5CFC4F80818093F907909142069D
:1086D000983F18F49093D10109C0EFEFF0E0E91B47
:1086E000F109EF5CFC4F80818093D101983F18F431
:1086F0009093D10109C0EFEFF0E0E91BF109EF5CC5
:10870000FC4F80818093D10180914506883F38F0ED
:10871000EFEFF0E0E81BF109EF5CFC4F8081809304
:10872000CF0180914706883F38F0EFEFF0E0E81B7B
:10873000F109EF5CFC4F80818093CD0180914F0661
:10874000883F38F0EFEFF0E0E81BF109EF5CFC4FF9
:1087500080818093CE0180915106883F38F0EFEF01
:10876000F0E0E81BF109EF5CFC4F80818093CA01C7
:1087700080915206883F38F0EFEFF0E0E81BF109F6
:10878000EF5CFC4F80818093CC0180915306883F41
:1087900038F0EFEFF0E0E81BF109EF5CFC4F80816F
:1087A0008093C90180915406883F38F0EFEFF0E0E4
:1087B000E81BF109EF5CFC4F80818093C801809138
:1087C0005A06883F38F0EFEFF0E0E81BF109EF5C64
:1087D000FC4F80818093C60180915B06883F38F012
:1087E000EFEFF0E0E81BF109EF5CFC4F8081809334
:1087F0000A0380915C06883F38F0EFEFF0E0E81B59
:10880000F109EF5CFC4F80818093090380915D0644
:10881000883F38F0EFEFF0E0E81BF109EF5CFC4F28
:1088200080818093080380915E06883F38F0EFEFE7
:10883000F0E0E81BF109EF5CFC4F808180930703B7
:1088400080917806883F38F0EFEFF0E0E81BF109FF
:10885000EF5CFC4F80818093060380917906883F0E
:1088600038F0EFEFF0E0E81BF109EF5CFC4F80819E
:108870008093050380917A06883F38F0EFEFF0E0AF
:10888000E81BF109EF5CFC4F808180930403809129
:108890007B06883F38F0EFEFF0E0E81BF109EF5C72
:1088A000FC4F80818093030380915F06883F38F0FE
:1088B000EFEFF0E0E81BF109EF5CFC4F8081809363
:1088C000C50180916306883F38F0EFEFF0E0E81BC8
:1088D000F109EF5CFC4F80818093C40180916D06AB
:1088E000883F38F0EFEFF0E0E81BF109EF5CFC4F58
:1088F00080818093C30180917006883F38F0EFEF4C
:10890000F0E0E81BF109EF5CFC4F80818093C2012D
:1089100080917106883F38F0EFEFF0E0E81BF10935
:10892000EF5CFC4F80818093C10180917206883F8B
:1089300038F0EFEFF0E0E81BF109EF5CFC4F8081CD
:108940008093C00180917706883F38F0EFEFF0E028
:10895000E81BF109EF5CFC4F80818093BF0180919F
:108960009206883F38F0EFEFF0E0E81BF109EF5C8A
:10897000FC4F808180932A088091C601282F3327DD
:108980002F5F3F4F8CE398E2B9010E94D578709336
:10899000D4016093D30180914D0680931B08809190
:1089A0004C068093E20780910A03813011F08430F5
:1089B00049F481E090E0909398018093970183E0DF
:1089C00090E008C083E090E0909398018093970135
:1089D00081E090E0909396018093950190919406A8
:1089E0009333E8F181E080930203983F58F0EFEF72
:1089F000F0E0E91BF109EF5CFC4F8081823310F459
:108A0000109202038091D50120910203821799F000
:108A1000833070F4222319F08CED95E002C088ECCD
:108A200090E09093300280932F022093D50103C0F1
:108A300081508093D50180916A0890916B0897FFCF
:108A400008C080910203882321F080915B04806834
:108A500003C080915B048F7780935B0405C0109204
:108A600002038AE08093D50180916A0890916B0897
:108A700097FF1DC0809127038823C9F080910203CE
:108A80008823A9F080910801909109018F5F9F4F81
:108A900071F488E99AE39093300280932F0280E08A
:108AA00094EA909309018093080110920203809147
:108AB0000203882369F08091F40281608093F402BC
:108AC0008091C201823D48F4825E8093C20105C05C
:108AD0008091F4028E7F8093F402DF91CF9108950C
:108AE000AAE1B0E0E6E7F5E40C9425790E94A23A09
:108AF000309102013C3010F4299A01C02998E0908D
:108B00002803F0902903FA82E9828091E2079927ED
:108B10000A96E816F90614F49A8389838091300343
:108B2000843608F05CC08091C7039091C803009719
:108B300031F001979093C8038093C70307C0109248
:108B400027038091F5028F7E8093F5023A3011F071
:108B5000343110F0289A01C028988091F602909143
:108B6000F702895E9340C0F180915706282F332782
:108B70003A8329838091F50280618093F502809188
:108B80003306A82FBB27AA0FBB1FFD01EF56F84FD6
:108B90001182108280913406282F3327220F331F31
:108BA000C9018F56984FFC0111821082A35AB84F09
:108BB00011961C921E92235A384FD90111961C927D
:108BC0001E9280913606E82FFF27EE0FFF1FE35A13
:108BD000F84F11821082F6C210922703F3C28091DF
:108BE00030038D3808F4EEC28091F5028F7E8093B9
:108BF000F5029091580682E3989FC001112490934A
:108C0000C8038093C703E981FA81B9978CF08091FA
:108C10002703882369F08091F6029091F702FFEF15
:108C20008F3F9F0729F001969093F7028093F602F9
:108C30008091F6029091F7028F3F910509F008F5B7
:108C400010924A0310924B0310924C0310924D0362
:108C50001092460310924703109248031092490362
:108C60001092B3031092B4031092B5031092B6039E
:108C70001092520310925303109254031092550312
:108C800005C08091F50282608093F50280913506DF
:108C9000E82FFF27EE0FFF1FE35AF84F80819181E5
:108CA000813591050CF462C120912703222309F03C
:108CB0005DC1E0919701F0919801EE5CF94F8181DF
:108CC000E82FFF27EE0FFF1FE35AF84F80819181B5
:108CD0008C3491050CF422C18091C9038F5F80937D
:108CE000C903893C08F442C13C3010F4299801C002
:108CF000299A109227031092C9031092F70210923A
:108D0000F60220913306E22FFF27EE0FFF1FE35AF2
:108D1000F84F8081918187349105DCF4E0919501D1
:108D2000F0919601EE5CF94F8181E82FFF27EE0F5D
:108D3000FF1FE35AF84F808191810190F081E02D6F
:108D4000F7FF03C0F095E195FF4FE734F1050CF410
:108D50008AC031E04091950150919601FA01EE5C94
:108D6000F94F8181A82FBB27AA0FBB1FA35AB84F69
:108D70008D919C9111978734910544F0E22FFF2744
:108D8000EE0FFF1FE35AF84F808191818D919C91E6
:108D90008734910574F080913306E82FFF27EE0F9A
:108DA000FF1FE35AF84F80819181873491050CF0C1
:108DB00032E0FA01EE5CF94F8181E82FFF27EE0FD8
:108DC000FF1FE35AF84F808191818634910574F436
:108DD00080913306E82FFF27EE0FFF1FE35AF84F6D
:108DE00080819181873491050CF033E0FA01EE5CCB
:108DF000F94F8181E82FFF27EE0FFF1FE35AF84F4D
:108E0000808191818A5B9F4F74F480913306E82FB3
:108E1000FF27EE0FFF1FE35AF84F808191818734BF
:108E200091050CF034E04E5C594FFA018181E82F36
:108E3000FF27EE0FFF1FE35AF84F808191818A5B75
:108E40009F4F74F480913306E82FFF27EE0FFF1F2A
:108E5000E35AF84F80819181863491050CF435E016
:108E6000832F0E94E72CE0919501F0919601EE5C32
:108E7000F94F8181E82FFF27EE0FFF1FE35AF84FCC
:108E8000808191810190F081E02DF7FF03C0F09582
:108E9000E195FF4F7E97BCF480913306E82FFF27C2
:108EA000EE0FFF1FE35AF84F808191818A5B9F4F3D
:108EB00054F481E08093760488EE93E0909330023E
:108EC00080932F0253C00E94BD2D0E94B02C80E0E1
:108ED0000E943607809159060E940A7680913F06CB
:108EE00080FF10C08091140190911501875B934021
:108EF00038F480911401909115018E5E924010F427
:108F00000E94D41A10922D0280E00E94EB3781E07B
:108F10008093CC0380932D02579A1FC0808191814A
:108F2000855B9F4F0CF58091C9038F5F8093C903C8
:108F3000893CE0F03C3010F4299801C0299A109245
:108F400027031092C9031092F7021092F60281E0F3
:108F50000E94EB3781E08093CC030E94BD2D68E72F
:108F600070E00E94293702C02093C9038091350622
:108F7000E82FFF27EE0FFF1FE35AF84F8081918102
:108F80008B5A9F4F0CF01EC130912703E09197013F
:108F9000F0919801332309F0E6C0EE5CF94F81812E
:108FA000E82FFF27EE0FFF1FE35AF84F80819181D2
:108FB000855B9F4F0CF0D4C020919506E22FFF27D0
:108FC000EE0FFF1FE35AF84F80819181855B9F4F21
:108FD0001CF0222309F0C4C08091CA038F5F8093E4
:108FE000CA03893C08F4EEC03093CA0380915B0445
:108FF000882309F0AEC08091CC03882309F4A9C06E
:1090000080911504882309F0A4C081E090E090933A
:10901000F7028093F60281E0809327031092B30356
:109020001092B4031092B5031092B603109252033B
:1090300010925303109254031092550310924E0352
:1090400010924F03109250031092510380914E06DC
:10905000E82EFF2400271127809117089091180807
:109060009C01442737FD4095542FC801B7010E9449
:109070009678DC01CB018093620390936303A09305
:109080006403B093650380912708909128089C01A0
:10909000442737FD4095542FC801B7010E949678A8
:1090A000DC01CB0180935A0390935B03A0935C0394
:1090B000B0935D038091820390918303A091840318
:1090C000B091850380935E0390935F03A093600348
:1090D000B093610380917A0390917B03A0917C030C
:1090E000B0917D038093560390935703A093580348
:1090F000B093590310924A0310924B0310924C0301
:1091000010924D03109246031092470310924803A9
:10911000109249038091F50288608093F502909146
:1091200093068FE0989F900111248091E201909125
:10913000E301820F931F68E671E00E94D57897FDE6
:109140000196959587958093860384E68093CD0359
:1091500039C08CED95E09093300280932F0232C09D
:109160001092CA032FC0EE5CF94F8181E82FFF27D0
:10917000EE0FFF1FE35AF84F808191818C349105E7
:10918000FCF020919506E22FFF27EE0FFF1FE35A18
:10919000F84F80819181855B9F4F14F0222381F4E9
:1091A0008091CB038F5F8093CB03893C58F0109262
:1091B00027031092CB031092F7021092F60202C01E
:1091C0001092CB03809194018150809394018091FF
:1091D00094018F3F21F08091F50284FF72C30E94B9
:1091E00091428091D6039091D7039C01220F331FA7
:1091F000280F391FC0903306AC2DBB27AA0FBB1F09
:10920000FD01E35AF84FB09049064B2D5527808158
:109210009181849FF001859FF00D949FF00D1124A2
:109220002E0F3F1F37FF02C02D5F3F4FB9017595CD
:10923000679575956795AF56B84F80914A06082F88
:1092400011278D919C91809F7001819FF00C909FC0
:10925000F00C11246E0D7F1D7093D7036093D6031D
:109260008091D8039091D9039C01220F331F280FBE
:10927000391FD0903406AD2DBB27AA0FBB1FFD01AF
:10928000E35AF84F80819181849FF001859FF00D12
:10929000949FF00D11242E0F3F1F37FF02C02D5F4A
:1092A0003F4FA9015595479555954795AF56B84FEE
:1092B0008D919C91809F7001819FF00C909FF00C8C
:1092C00011244E0D5F1D5093D9034093D803809114
:1092D0000203882309F448C0CB0177FD0396DC0123
:1092E000B595A795B595A795CA0157FD0396FC01BD
:1092F000F595E795F595E7958091F301682F772728
:1093000067FD70956A9F90016B9F300D7A9F300DBD
:10931000112480911704482F552747FD50954E9FE3
:10932000C0014F9F900D5E9F900D1124280F391F93
:1093300037FF02C0295F3F4F03E0359527950A9517
:10934000E1F730932F0320932E036E9F90016F9FC0
:10935000300D7E9F300D11244A9FC0014B9F900D10
:109360005A9F900D11243FC080919306E82FFF274C
:10937000E056FE4F86818093F3019081909317040D
:10938000A82FBB27A7FDB095A69F9001A79F300DE2
:10939000B69F300D1124E92FFF27E7FDF095E49FDC
:1093A000C001E59F900DF49F900D1124280F391FE7
:1093B00037FF02C0295F3F4F13E0359527951A9577
:1093C000E1F730932F0320932E03A49F9001A59FD4
:1093D000300DB49F300D1124E69FC001E79F900D22
:1093E000F69F900D1124281B390B37FF02C0295F0F
:1093F0003F4FF3E035952795FA95E1F730932D032C
:1094000020932C0380913606E82FFF27EE0FFF1FD5
:10941000E35AF84F80819181909581959F4F909369
:109420002B0380932A038530910514F0049705C01F
:109430000FEF8C3F900734F4049690932B038093A6
:109440002A0304C010922B0310922A0380910B046C
:1094500090910C042091070430910804820F931F0F
:1094600000912E0310912F03081B190B10932F034B
:1094700000932E038091090490910A042091050421
:1094800030910604820F931F80902C0390902D033F
:10949000881A990A90922D0380922C0380913506A8
:1094A000E82FFF27EE0FFF1FE35AF84FE080F1800F
:1094B00028E730E0E20EF31EF0922903E092280341
:1094C0008091CB019927AA2797FDA095BA2FBC01BF
:1094D000CD010E943E78DC01CB0120E030E040E28B
:1094E00051E4BC01CD010E94DF77DC01CB01BC015E
:1094F000CD010E942178DC01CB018093210880916D
:10950000CA018093FA078091C9019927AA2797FD7C
:10951000A095BA2FBC01CD010E943E78DC01CB01A1
:1095200020E030E040E251E4BC01CD010E94DF7751
:10953000DC01CB01BC01CD010E942178DC01CB0113
:109540008093D5078091C8018093EA0780918204B7
:1095500080FF59C080912A08813808F454C0809156
:109560007B04992787FD90952B2D3327829FA0019F
:10957000839F500D929F500D1124040F151F1093BF
:109580002F0300932E0380917C04992787FD9095EB
:10959000829FB001839F700D929F700D1124860EE3
:1095A000971E90922D0380922C0380917D04282F8A
:1095B000332727FD309580912A0390912B03820F4A
:1095C000931F90932B0380932A0380917F04282F6D
:1095D000332727FD3095809144069927289FD00195
:1095E000299FB00D389FB00D1124B0939F01A09317
:1095F0009E0180917E0499278E159F0524F49093F7
:10960000290380932803809128039091290397FFD1
:1096100004C0109229031092280380913F0682FF14
:1096200002C01092FA0740912E0350912F03CA01F5
:1096300057FD03969C01359527953595279537FF5E
:1096400003C0309521953F4F8091FA029091FB0223
:1096500082179307B4F4CA0157FF03C09095819510
:109660009F4F97FD03969595879595958795909330
:10967000FB028093FA028536910544F084E690E07F
:1096800001C001979093FB028093FA0240912C0352
:1096900050912D03CA0157FD03969C0135952795DE
:1096A0003595279537FF03C0309521953F4F809121
:1096B000F8029091F90282179307B4F4CA0157FF98
:1096C00003C0909581959F4F97FD0396959587953B
:1096D000959587959093F9028093F80285369105C8
:1096E00044F084E690E001C001979093F9028093E2
:1096F000F8028091F50284FF08C01092FB021092DC
:10970000FA021092F9021092F802ED2DFF27EE0FE7
:10971000FF1FE35AF84F40916E06242F33278081B4
:1097200091812817390744F48091960682FF04C07E
:1097300081E080930E0313C0ED2DFF27EE0FFF1F76
:10974000E35AF84F842F992720916F06821B9109C5
:10975000208131812817390714F410920E034091AB
:109760003406E42FFF27EE0FFF1FE35AF84F509106
:109770006E06852F992722273327281B390B8081D6
:1097800091818217930744F48091960683FF04C069
:1097900081E080930D0316C080910D03882391F022
:1097A000E42FFF27EE0FFF1FE35AF84F80916F065B
:1097B0009927851B9109208131818217930714F421
:1097C00010920D03EC2DFF27EE0FFF1FE35AF84F09
:1097D00040916E06242F3327808191812817390705
:1097E00044F48091960680FF04C081E080930B03CF
:1097F00017C080910B03882399F0EC2DFF27EE0F03
:10980000FF1FE35AF84F842F992720916F06821B80
:109810009109208131812817390714F410920B0324
:1098200040913306E42FFF27EE0FFF1FE35AF84F56
:1098300050916E06852F992722273327281B390B35
:10984000808191818217930744F48091960681FF6D
:1098500004C081E080930C0316C080910C03882320
:1098600091F0E42FFF27EE0FFF1FE35AF84F80918E
:109870006F069927851B91092081318182179307F3
:1098800014F410920C0380910E03882319F4809134
:109890000D03811181E080930F0380910B038823D6
:1098A00021F480910C03882351F081E08093100310
:1098B00010920F0310920E0310920D0302C08093BA
:1098C000100380910F03882321F4809110038823D3
:1098D00069F080916D069927E981FA818E179F07BB
:1098E00014F49A83898381E080933C038091F5028C
:1098F00084FF1AC010922B0310922A0310922F0398
:1099000010922E0310922D0310922C039AE590933F
:10991000210888E78093FA079093D5078093EA0798
:1099200010920F03109210038091ED079091EE07B3
:10993000A091EF07B091F00720918203309183034B
:109940004091840350918503820F931FA41FB51F7C
:109950008093ED079093EE07A093EF07B093F00785
:109960008091F5079091F607A091F707B091F8075D
:1099700020907A0330907B0340907C0350907D03CD
:10998000820D931DA41DB51D8093F5079093F607D6
:10999000A093F707B093F8078091E4079091E5074B
:1099A000A091E607B091E707E0907E03F0907F0377
:1099B0000091800310918103EB82FC820D831E8352
:1099C0008E0D9F1DA01FB11F8093E4079093E507A4
:1099D000A093E607B093E7078091D6079091D70749
:1099E000A091D807B091D907E0907603F090770363
:1099F0000091780310917903EF82F88609871A871E
:109A00008E0D9F1DA01FB11F8093D6079093D7077F
:109A1000A093D807B093D907F0901003FB86FF20DE
:109A200029F480910F03882309F460C01092720317
:109A300010927303109274031092750310926E03C8
:109A400010926F0310927003109271031092ED0741
:109A50001092EE071092EF071092F0071092F507A0
:109A60001092F6071092F7071092F8071092E40789
:109A70001092E5071092E6071092E7071092D607BA
:109A80001092D7071092D8071092D90780916203DD
:109A900090916303A0916403B091650380935E038A
:109AA00090935F03A0936003B093610380915A0386
:109AB00090915B03A0915C03B0915D03809356038A
:109AC00090935703A0935803B093590310923F0209
:109AD00010923E0210921403109213031092160378
:109AE000109215030B85002309F0F9C180910F0333
:109AF000882309F0F4C180912406909125068150B5
:109B000092402CF480912703882309F4E8C16091E6
:109B1000A3086C87A0904E068091170890911808B2
:109B20009A8F898FA0912708B0912808BC8BAB8BA6
:109B300016160CF0DDC0BB24CC24DD24CA01B9010B
:109B4000A60195010E940A7979018A01E98DFA8DB1
:109B5000CF01AA2797FDA095BA2FE81AF90A0A0B98
:109B60001B0BC201B101A60195010E940A7959019E
:109B70006A012B893C89C901AA2797FDA095BA2FB4
:109B8000A81AB90ACA0ADB0A3C85232E332427FC0B
:109B90003094432C532CC801B701A20191010E94BB
:109BA000967897FF04C061507E4F8F4F9F4F3B01C7
:109BB0004C0109E095948794779467940A95D1F7BE
:109BC000C601B501A20191010E94967897FF04C0D9
:109BD00061507E4F8F4F9F4F5B016C0119E0D59410
:109BE000C794B794A7941A95D1F74C854093E00198
:109BF0008091FA029091FB02813491053CF48091AE
:109C0000F8029091F90281349105D4F0D401C30196
:109C100097FE03C00196A11DB11D3C014D01959415
:109C2000879477946794D601C501D7FE03C0019647
:109C3000A11DB11D5C016D01D594C794B794A79483
:109C400080913606E82FFF27EE0FFF1FE35AF84FEB
:109C5000808191810190F081E02DF7FF03C0F095A4
:109C6000E195FF4F7A97A4F0C401B30123E030E0FF
:109C700040E050E00E940A7939014A01C601B5016D
:109C800023E030E040E050E00E940A7959016A0187
:109C90008091A508282F332727FD3095432F532F78
:109CA000261537054805590514F439014A01992745
:109CB00087FD9095909581959F4FAA2797FDA09538
:109CC000BA2F681679068A069B0614F43C014D01EA
:109CD0002A153B054C055D0514F459016A01A816C7
:109CE000B906CA06DB060CF0D2C05C016D01CFC01C
:109CF000EA2CFF2400271127CA01B901A801970106
:109D00000E940A7939014A01698D7A8DCB01AA270F
:109D100097FDA095BA2F681A790A8A0A9B0AC20190
:109D2000B101A80197010E940A7959016A01EB89E2
:109D3000FC89CF01AA2797FDA095BA2FA81AB90AC6
:109D4000CA0ADB0AD401C30197FE03C00F96A11D06
:109D5000B11D3C014D01F4E095948794779467948C
:109D6000FA95D1F7D601C501D7FE03C00F96A11D04
:109D7000B11D5C016D01E4E0D594C794B794A7943C
:109D8000EA95D1F78091FA029091FB028134910516
:109D90003CF48091F8029091F90281349105A4F08D
:109DA000C401B30123E030E040E050E00E940A79B2
:109DB00039014A01C601B50123E030E040E050E03E
:109DC0000E940A7959016A0180913606E82FFF271F
:109DD000EE0FFF1FE35AF84F808191810190F081CF
:109DE000E02DF7FF03C0F095E195FF4F7A97A4F0BF
:109DF000C401B30123E030E040E050E00E940A7962
:109E000039014A01C601B50123E030E040E050E0ED
:109E10000E940A7959016A0189E18093E001F1E227
:109E20006F167104810491042CF070E2672E712C7E
:109E3000812C912C00EE60160FEF70060FEF80065C
:109E40000FEF900644F460EE662E6FEF762E6FEF04
:109E5000862E6FEF962E11E2A116B104C104D10433
:109E60002CF050E2A52EB12CC12CD12C20EEA21644
:109E70002FEFB2062FEFC2062FEFD20644F440EECA
:109E8000A42E4FEFB42E4FEFC42E4FEFD42E80915F
:109E9000620390916303A0916403B09165038619F6
:109EA0009709A809B9098093620390936303A0936B
:109EB0006403B093650380915A0390915B03A09172
:109EC0005C03B0915D038A199B09AC09BD098093BD
:109ED0005A0390935B03A0935C03B0935D0380915E
:109EE0003E0290913F028F3F910509F008F4C4C5EE
:109EF0003B85332309F04EC580910F03882309F079
:109F000049C580913C03882309F044C540917606F9
:109F10004D87442309F43EC58091ED079091EE07EB
:109F2000A091EF07B091F007B7FF04C081509F4F99
:109F3000AF4FBF4FE92EFA2E0B2F112707FD1A95B1
:109F4000E092ED07F092EE070093EF071093F00711
:109F50008091F5079091F607A091F707B091F80767
:109F6000B7FF04C081509F4FAF4FBF4F892F9A2F2B
:109F7000AB2FBB27A7FDBA958E879F87A88BB98B80
:109F80008093F5079093F607A093F707B093F8072F
:109F900080914E06A82EBB24CC24DD242091720390
:109FA000309173034091740350917503C601B5015C
:109FB0000E94967897FF04C061507F4F8F4F9F4F4C
:109FC000672E782E892E992487FC9A9460927203CA
:109FD00070927303809274039092750320916E03C4
:109FE00030916F034091700350917103C601B50128
:109FF0000E94967897FF04C061507F4F8F4F9F4F0C
:10A00000272E382E492E552447FC5A9420926E0351
:10A0100030926F03409270035092710380916A03F3
:10A0200090916B03A0916C03B0916D03B7FF04C0D6
:10A0300081509F4FAF4FBF4F892F9A2FAB2FBB2718
:10A04000A7FDBA9580936A0390936B03A0936C036A
:10A05000B0936D03D801C70186199709A809B909FA
:10A060008093BF039093C003A093C103B093C20336
:10A0700020917506E22EFF2400271127BC01CD0197
:10A08000A80197010E940A7959016A012093CE0321
:10A090003093CF034093D0035093D1038E859F8597
:10A0A000A889B98982199309A409B5098093C303C2
:10A0B0009093C403A093C503B093C603BC01CD0124
:10A0C000A80197010E940A792093D2033093D30309
:10A0D0004093D4035093D503D601C501D7FE04C0E5
:10A0E00081509F4FAF4FBF4F892F9A2FAB2FBB2768
:10A0F000A7FDBA95909314038093130357FF04C0F0
:10A1000021503F4F4F4F5F4FBB2757FDBA95A52FAB
:10A11000942F832F90931603809315038091FA0256
:10A120009091FB0281349105DCF48091F8029091CA
:10A13000F90281349105A4F480913606E82FFF27B7
:10A14000EE0FFF1FE35AF84F808191810190F0815B
:10A15000E02DF7FF03C0F095E195FF4F7A97E4F00B
:10A160008091A3088F3FC1F4809113039091140351
:10A1700097FD01969595879590931403809313030B
:10A18000809115039091160397FD019695958795FB
:10A1900090931603809315038091E4079091E5074F
:10A1A000A091E607B091E707B7FF04C081509F4F29
:10A1B000AF4FBF4F892F9A2FAB2FBB27A7FDBA9563
:10A1C0008093E4079093E507A093E607B093E70731
:10A1D0008091D6079091D707A091D807B091D90761
:10A1E000B7FF04C081509F4FAF4FBF4F892F9A2FA9
:10A1F000AB2FBB27A7FDBA958093D6079093D707BF
:10A20000A093D807B093D9078091820390918303DC
:10A21000A0918403B09185032B813C814D815E81A7
:10A22000281B390B4A0B5B0B2093B7033093B80301
:10A230004093B9035093BA0380917A0390917B03C2
:10A24000A0917C03B0917D03EF80F88409851A8585
:10A25000E81AF90A0A0B1B0BE092BB03F092BC034D
:10A260000093BD031093BE032093BF033093C0033C
:10A270004093C1035093C203E092C303F092C4031E
:10A280000093C5031093C60380915E0390915F0312
:10A29000A0916003B0916103821B930BA40BB50BDB
:10A2A00080935E0390935F03A0936003B093610378
:10A2B0008091560390915703A0915803B091590390
:10A2C0008E199F09A00BB10B8093560390935703EF
:10A2D000A0935803B09359035D855523E1F0209175
:10A2E0003A0330913B03213831054CF080919303C0
:10A2F0009091940301969093940380939303205834
:10A300003F4F4CF480919303909194030197909365
:10A3100094038093930310923B0310923A0381E0DD
:10A3200090E09093DB038093DA03E090BF03F0901A
:10A33000C0030091C1031091C203D801C70117FFE8
:10A3400007C088279927DC018E199F09A00BB10B44
:10A3500081509240A040B04034F084E090E090936F
:10A36000DB038093DA038091E0039091E103A091F5
:10A37000E203B091E3032091ED073091EE074091A5
:10A38000EF075091F007821B930BA40BB50B815E76
:10A39000914BAF4FBF4F8F539C49A040B04028F026
:10A3A0008091A40889310CF4FFC0F1E0EF16F0E1D0
:10A3B000FF06F0E00F07F0E01F070CF473C0809178
:10A3C000DC03882309F46AC0D801C70117FF07C05E
:10A3D00088279927DC018E199F09A00BB10B9C01DE
:10A3E000AD01B7FF04C021503E4F4F4F5F4FF9E022
:10A3F0005595479537952795FA95D1F78091DA03CA
:10A400009091DB03820F931F9093DB038093DA0319
:10A41000D801C70117FF03C00796A11DB11DE3E0D6
:10A42000B595A79597958795EA95D1F78093CE0333
:10A430009093CF03A093D003B093D1038958934155
:10A44000A040B04064F088E893E1A0E0B0E08093E1
:10A45000CE039093CF03A093D003B093D103209168
:10A46000CE033091CF034091D0035091D10357FFD9
:10A4700004C021503F4F4F4F5F4F232F342F452FA4
:10A48000552747FD5A958091130390911403820F2D
:10A49000931F909314038093130306C081E080936D
:10A4A000DC0302C01092DC0330E0E31630EFF30669
:10A4B0003FEF03073FEF13070CF073C08091DD03FC
:10A4C000882309F46AC0D801C70117FF07C088278D
:10A4D0009927DC018E199F09A00BB10B9C01AD01DE
:10A4E000B7FF04C021503E4F4F4F5F4F69E0559575
:10A4F0004795379527956A95D1F78091DA03909122
:10A50000DB03820F931F9093DB038093DA03D80160
:10A51000C70117FF03C00796A11DB11D23E0B59524
:10A52000A795979587952A95D1F78093CE03909319
:10A53000CF03A093D003B093D10388579C4EAF4F65
:10A54000BF4F64F488E79CEEAFEFBFEF8093CE037C
:10A550009093CF03A093D003B093D1032091CE0367
:10A560003091CF034091D0035091D10357FF04C0E5
:10A5700021503F4F4F4F5F4F232F342F452F5527EB
:10A5800047FD5A958091130390911403820F931FF6
:10A59000909314038093130311C081E08093DD0333
:10A5A0000DC01092DD030AC01092DB031092DA0393
:10A5B00084E690E09093DF018093DE015D85252F96
:10A5C00033278091DA039091DB032817390724F4AD
:10A5D0003093DB032093DA031091A408112379F060
:10A5E000212F332727FD30958091DA039091DB03EB
:10A5F0002817390724F43093DB032093DA034091C2
:10A60000BF035091C0036091C1037091C2034138F0
:10A6100051056105710574F080919703909198033D
:10A620002091DA033091DB03820F931F90939803FC
:10A630008093970340585F4F6F4F7F4F74F4809122
:10A640009703909198032091DA033091DB03821BEA
:10A65000930B909398038093970381E090E09093FD
:10A66000DB038093DA03C090C303D090C403E0906F
:10A67000C503F090C603D701C601F7FE07C08827BF
:10A680009927DC018C199D09AE09BF0981509240C0
:10A69000A040B04034F084E090E09093DB038093DE
:10A6A000DA038091E4039091E503A091E603B09171
:10A6B000E7032091F5073091F6074091F707509195
:10A6C000F807821B930BA40BB50B815E914BAF4F28
:10A6D000BF4F8F539C49A040B04018F019310CF483
:10A6E000FFC001E0C01600E1D00600E0E00600E097
:10A6F000F0060CF473C08091DE03882309F46AC06D
:10A70000D701C601F7FE07C088279927DC018C19FD
:10A710009D09AE09BF099C01AD01B7FF04C02150DE
:10A720003E4F4F4F5F4F09E0559547953795279519
:10A730000A95D1F78091DA039091DB03820F931F82
:10A740009093DB038093DA03D701C601F7FE03C0C1
:10A750000796A11DB11D13E0B595A795979587950F
:10A760001A95D1F78093D2039093D303A093D40387
:10A77000B093D50389589341A040B04064F088E875
:10A7800093E1A0E0B0E08093D2039093D303A09331
:10A79000D403B093D5032091D2033091D3034091D9
:10A7A000D4035091D50357FF04C021503F4F4F4F62
:10A7B0005F4F232F342F452F552747FD5A95809102
:10A7C000150390911603820F931F909316038093A5
:10A7D000150306C081E08093DE0302C01092DE0301
:10A7E00020E0C21620EFD2062FEFE2062FEFF2068E
:10A7F0000CF073C08091DF03882309F46AC0D7018D
:10A80000C601F7FE07C088279927DC018C199D092E
:10A81000AE09BF099C01AD01B7FF04C021503E4FF6
:10A820004F4F5F4FE9E05595479537952795EA9546
:10A83000D1F78091DA039091DB03820F931F9093FD
:10A84000DB038093DA03D701C601F7FE03C0079646
:10A85000A11DB11D73E0B595A795979587957A953C
:10A86000D1F78093D2039093D303A093D403B093F2
:10A87000D50388579C4EAF4FBF4F64F488E79CEEDA
:10A88000AFEFBFEF8093D2039093D303A093D40391
:10A89000B093D5032091D2033091D3034091D403D8
:10A8A0005091D50357FF04C021503F4F4F4F5F4F8A
:10A8B000232F342F452F552747FD5A958091150397
:10A8C00090911603820F931F9093160380931503A4
:10A8D00011C081E08093DF030DC01092DF030AC036
:10A8E0001092DB031092DA0384E690E09093DF018C
:10A8F0008093DE014D85242F33278091DA039091D8
:10A90000DB032817390724F43093DB032093DA03A1
:10A910008091A408882379F0282F332727FD3095CC
:10A920008091DA039091DB032817390724F43093E0
:10A93000DB032093DA034091C3035091C403609179
:10A94000C5037091C603413851056105710574F066
:10A9500080919503909196032091DA033091DB0367
:10A96000820F931F909396038093950340585F4FF7
:10A970006F4F7F4FCCF48091950390919603209177
:10A98000DA033091DB03821B930B90939603809341
:10A9900095030AC010921603109215031092140327
:10A9A0001092130310923C038091FA07882341F41C
:10A9B00010921603109215031092140310921303B1
:10A9C0008091ED079091EE07A091EF07B091F0070D
:10A9D0008093E0039093E103A093E203B093E30339
:10A9E0008091F5079091F607A091F707B091F807CD
:10A9F0008093E4039093E503A093E603B093E70309
:10AA000010927203109273031092740310927503E4
:10AA100010926E0310926F031092700310927103E4
:10AA200010926A0310926B0310926C0310926D03E4
:10AA30001092ED071092EE071092EF071092F007B8
:10AA40001092F5071092F6071092F7071092F80788
:10AA50001092E4071092E5071092E6071092E707BC
:10AA60001092D6071092D7071092D8071092D907E4
:10AA700010923F0210923E02E0902A03F0902B03C6
:10AA8000C701F7FE04C0882799278E199F090497EC
:10AA90003CF080913F0684FD03C082E38093CD03A8
:10AAA00010914B06A12EBB24CC24DD24B7018827AE
:10AAB00077FD8095982F9701F7FE04C02227332752
:10AAC0002E193F09442737FD4095542F0E94967850
:10AAD0009B01AC01C601B5010E94967897FF04C0A6
:10AAE00061507E4F8F4F9F4F59E095958795779591
:10AAF00067955A95D1F79B01812F99278E9DD0019B
:10AB00008F9DB00D9E9DB00D1124CD01B7FD039614
:10AB10009595879595958795280F391F80911703EF
:10AB200090911803280F391F442737FD4095542F63
:10AB30002093B3033093B4034093B5035093B6030B
:10AB40008091520390915303A0915403B091550307
:10AB5000821B930BA40BB50B80935203909353036A
:10AB6000A0935403B09355038155934CA040B0403B
:10AB700064F080E593ECA0E0B0E080935203909302
:10AB80005303A0935403B0935503809152039091C3
:10AB90005303A0915403B0915503805B9C43AF4F86
:10ABA000BF4F64F480EB9CE3AFEFBFEF80935203A1
:10ABB00090935303A0935403B0935503C090E201C4
:10ABC000D090E301D7FC49C180913F0683FF45C186
:10ABD0008091E10181508093E101882309F041C116
:10ABE0008DE08093E1018091820390918303A09195
:10ABF0008403B0918503B7FF04C081509E4FAF4FCF
:10AC0000BF4F09E0B595A795979587950A95D1F718
:10AC10002C0197FF04C050944194510853948091A3
:10AC20007A0390917B03A0917C03B0917D03B7FFE1
:10AC300004C081509E4FAF4FBF4F19E0B595A79507
:10AC4000979587951A95D1F79C0197FF03C030958A
:10AC500021953F4F421653060CF42901B20157FECD
:10AC600002C06D5F7F4F3B01759467947594679444
:10AC70000894611C711CACE1EA2EA2E0FA2ECE0C05
:10AC8000DF1C76010027F7FC0095102F24EE3DEF26
:10AC9000C20ED31E8091230890912408A09125080C
:10ACA000B091260880909A0190909B01A0909C0101
:10ACB000B0909D01BC01CD01A50194010E940A79CB
:10ACC000E21AF30A040B150BC801B70128E631E0BC
:10ACD00040E050E00E940A79DC01CB018C01045B6A
:10ACE00010408091DE019091DF01009731F00197D3
:10ACF0009093DF018093DE0134C039E143165104A3
:10AD000084F580913A0390913B03800F911F9093BB
:10AD10003B0380933A038091CD03882311F1815046
:10AD20008093CD038823E9F4C601AA2797FDA09557
:10AD3000BA2FBC01CD01A50194010E949678DC01D7
:10AD4000CB018093230890932408A0932508B09307
:10AD50002608BC01CD010E940A793093410320935B
:10AD600040038091DE019091DF01892B39F58091BC
:10AD7000E0019927089FA001099F500D189F500DD1
:10AD80001124CA01B3010E94D5789B01442737FDE5
:10AD90004095542F8091230890912408A091250874
:10ADA000B0912608820F931FA41FB51F809323081C
:10ADB00090932408A0932508B09326088091CD0392
:10ADC000882309F04AC080914003909141037C019F
:10ADD0000027F7FC0095102F8091230890912408FC
:10ADE000A0912508B0912608BC01CD01A5019401D0
:10ADF0000E940A79E21AF30A040B150B6CE172E067
:10AE000080E090E0E60EF71E081F191FC801B70189
:10AE100028E631E040E050E00E940A79DC01CB01F5
:10AE20009C01245B30408091CE0186959927289F14
:10AE3000D001299FB00D389FB00D11249D01B7FF9F
:10AE400002C0215F3F4FF4E035952795FA95E1F771
:10AE5000309318032093170304C010921803109224
:10AE6000170380913C03882381F0109246031092CF
:10AE70004703109248031092490310924A0310921C
:10AE80004B0310924C0310924D03F0901003FF20DF
:10AE9000F1F48091FA07282F332744275527809112
:10AEA000820390918303A0918403B0918503BC0138
:10AEB000CD010E949678DC01CB01BC01CD0128EFC9
:10AEC0003AE240E050E00E940A79390102C066246B
:10AED0007724E0900F03EE20F1F48091FA07282FF9
:10AEE00033274427552780917A0390917B03A091C3
:10AEF0007C03B0917D03BC01CD010E949678DC01FA
:10AF0000CB01BC01CD0128EF3AE240E050E00E94C5
:10AF10000A79190102C0222433248091D00790912C
:10AF2000D107893C91051CF088EC90E005C088535E
:10AF30009F4F34F488E39FEF9093D1078093D0071D
:10AF40008091DB079091DC07893C91051CF088EC2F
:10AF500090E005C088539F4F34F488E39FEF9093AF
:10AF6000DC078093DB078091DD079091DE07AA273D
:10AF700097FDA095BA2F20912108A22EBB24CC24A6
:10AF8000DD24BC01CD01A60195010E9496789B01AC
:10AF9000AC018091D0079091D107AA2797FDA09589
:10AFA000BA2FE7E0880F991FAA1FBB1FEA95D1F7B8
:10AFB000280F391F4A1F5B1F57FF04C0215C3F4FFA
:10AFC0004F4F5F4F76E055954795379527957A9582
:10AFD000D1F78301020F131F1093DE070093DD07E3
:10AFE0008091CE079091CF07AA2797FDA095BA2F01
:10AFF000BC01CD01A60195010E9496789B01AC0190
:10B000008091DB079091DC07AA2797FDA095BA2FC6
:10B0100067E0880F991FAA1FBB1F6A95D1F7280FF9
:10B02000391F4A1F5B1F57FF04C0215C3F4F4F4F22
:10B030005F4F96E055954795379527959A95D1F7A7
:10B040004101820E931E9092CF078092CE0780918D
:10B050001C0890911D08880F991FAA2797FDA0959D
:10B06000BA2F2091D507332744275527BC01CD019E
:10B070000E9496785B016C0197FF08C02FE330E0D7
:10B0800040E050E0A20EB31EC41ED51E86E0D5944B
:10B09000C794B794A7948A95D1F78091EA07282F8F
:10B0A0003327442755278091660390916703A09129
:10B0B0006803B0916903BC01CD010E949678DC0160
:10B0C000CB01BC01CD0120EF35E540E050E00E940E
:10B0D0000A79B501620F731F70931D0860931C08F5
:10B0E0000150104134F080E090E19093DE078093AE
:10B0F000DD078091DD079091DE078050904F34F49A
:10B1000080E090EF9093DE078093DD0751E0851695
:10B1100050E1950634F080E090E19093CF07809362
:10B12000CE078091CE079091CF078050904F34F496
:10B1300080E090EF9093CF078093CE0761507041ED
:10B1400034F080E090E190931D0880931C0880917A
:10B150001C0890911D088050904F34F480E090EFCF
:10B1600090931D0880931C0880910001482F55275B
:10B1700080911E0190911F014817590794F4209166
:10B180001E0130911F0109811A81049FC001059F92
:10B19000900D149F900D1124B9010E94C1787A83FB
:10B1A000698329813A81220F331F220F331F3A838B
:10B1B000298340913F0640FF92C7EE2009F08FC7D8
:10B1C000FF2009F08CC7AA24BB24450180911103FC
:10B1D000909112039093080680930706209199039B
:10B1E00030919A032115310509F03FC08091140177
:10B1F000909115018959934058F087B5853F20F407
:10B2000080914202815011C081E08093F3034EC0CF
:10B2100080911401909115018436910508F587B548
:10B220008B30D0F0809142028F5F809342029AE08F
:10B2300089029001112480912E06821B87BD8CE229
:10B2400091E09093300280932F028EE591E09093ED
:10B250009A03809399032AC081E08093F20326C069
:10B26000F092F203F092F30321C0809122039091B7
:10B270002303A0912403B091250314E0880F991FA4
:10B28000AA1FBB1F1A95D1F78093430290934402E3
:10B29000A0934502B0934602B0924102A0924002B0
:10B2A0002150304030939A03209399032091D1018B
:10B2B00041FF24C02233D8F48091E801815080936B
:10B2C000E8018F3FD9F510923D03809122039091C0
:10B2D0002303A0912403B091250380931E03909330
:10B2E0001F03A0932003B093210381E004C081E0F9
:10B2F00080933D0388EC8093E80120C080919E01FB
:10B3000090919F01820F911D209144063327829FC7
:10B31000A001839F500D929F500D1124CA01AA27AE
:10B3200097FDA095BA2F80931E0390931F03A093BF
:10B330002003B093210381E080933D038091820339
:10B3400090918303A0918403B0918503E0909A01CA
:10B35000F0909B0100919C0110919D01BC01CD01D9
:10B36000A80197010E940A7959016A0180917A0324
:10B3700090917B03A0917C03B0917D03BC01CD0132
:10B38000A80197010E940A79B901C5010E94B86F0E
:10B390008C01CC9714F00CE310E0C8010E94B36B51
:10B3A0008C0180E28093990180913D03882309F408
:10B3B00008C58091F50299279C012071307084FDA9
:10B3C00000C58091F40282608093F4027091980627
:10B3D00070FD04C080913F0681FD0CC0C980DA80F9
:10B3E0003093E9032093E8038091F502806C809309
:10B3F000F50255C28091F50281FF27C24091E40118
:10B400005091E501CA010F9620912803309129033C
:10B4100082179307BCF56091F203662399F580913A
:10B42000F50287FF15C08091F5028F778093F502B2
:10B430008091220390912303A0912403B0912503CE
:10B4400080931E0390931F03A0932003B0932103C6
:10B450008091F50280648093F502241B350B2F50F8
:10B46000304037FF03C0309521953F4F8091E8036E
:10B470009091E903820F931F9093E9038093E8036F
:10B480008BE23BC0CA010F9728173907DCF56091A2
:10B49000F3036623B9F58091F50286FF15C080910C
:10B4A000F5028F7B8093F502809122039091230314
:10B4B000A0912403B091250380931E0390931F0352
:10B4C000A0932003B09321038091F50280688093BC
:10B4D000F502241B350B215F3F4F37FF03C030952A
:10B4E00021953F4F8091E8039091E903821B930BD4
:10B4F0009093E9038093E8038DE280939901609330
:10B50000F403BFC08DE38093990160911903662312
:10B5100091F120911A0330911B0340911C0350912B
:10B520001D0380911E0390911F03A0912003B091F1
:10B53000210382179307A407B507ECF48091F50265
:10B5400080648093F5028091E8039091E903860F6F
:10B55000911D9093E9038093E8038AE08093F403BC
:10B560008EE5809399018091F50287FF8AC08091D2
:10B57000F5028F7734C0662309F444C020911A0382
:10B5800030911B0340911C0350911D0380911E03B9
:10B5900090911F03A0912003B09121032817390730
:10B5A0004A075B077CF58091F50280688093F5027D
:10B5B0008091E8039091E903861B91099093E90338
:10B5C0008093E80386EF8093F40386E780939901E4
:10B5D0008091F50286FF55C08091F5028F7B8093A4
:10B5E000F5028091220390912303A0912403B0914E
:10B5F000250380931E0390931F03A0932003B09311
:10B6000021033FC08091F502807CD9F18091F40341
:10B61000882389F48091220390912303A09124032D
:10B62000B091250380931E0390931F03A0932003E2
:10B63000B093210302C01092F4038091F5028F733E
:10B640008093F5021092E9031092E80371FF06C09F
:10B6500084EF91E09093300280932F028091260333
:10B66000882379F48091220390912303A0912403ED
:10B67000B0912503C397A105B1051CF081E080932B
:10B6800026032091E8033091E903C90137FF04C084
:10B6900088279927821B930B815092400CF4BEC0DF
:10B6A0004091F4034423E9F080911A0390911B0325
:10B6B00020911E0330911F03821B930B0996439721
:10B6C00048F480911A0390911B03A0911C03B09140
:10B6D0001D0327C0242F332727FD3095432F532FD9
:10B6E00014C0809144069927289FB001299F700DAE
:10B6F000389F700D1124CB0160E075E00E94D57871
:10B700009B01442737FD4095542F80911E03909153
:10B710001F03A0912003B0912103820F931FA41F48
:10B72000B51F80931E0390931F03A0932003B09333
:10B7300021031092E9031092E803C0902203D090F5
:10B740002303E0902403F0902503D701C601805025
:10B750009440A040B04020911E0330911F034091BF
:10B7600020035091210382179307A407B5075CF4C7
:10B77000D701C60180509C4FAF4FBF4F28173907E4
:10B780004A075B0744F080931E0390931F03A09326
:10B790002003B09321038091980681FF06C084E6C0
:10B7A00090E09093300280932F0280914806882386
:10B7B000A9F580911903882389F5409111035091CF
:10B7C000120357FF02C04D5F5F4F55954795559542
:10B7D000479580911E0190911F0120910001332710
:10B7E000489FD001499FB00D589FB00D1124CD0145
:10B7F000B9010E94D5787093E5016093E401663445
:10B8000071051CF486E490E005C06739710534F0D9
:10B8100086E990E09093E5018093E401809199039B
:10B8200090919A03892BB9F180912203909123037F
:10B83000A0912403B091250380931E0390931F03CE
:10B84000A0932003B093210326C0809122039091FE
:10B850002303A0912403B091250380599140A04077
:10B86000B04080931E0390931F03A0932003B093D6
:10B87000210380914806882311F0992702C088E7A8
:10B8800090E09093E5018093E401E981FA81F093DF
:10B890001203E0931103C0901103D0901203209182
:10B8A00022033091230340912403509125032D8BD3
:10B8B0003E8B4F8B588F20911E0330911F03409178
:10B8C0002003509121036D897E898F89988D2617D9
:10B8D00037074807590724F08091980680FDBDC2BC
:10B8E0008091990390919A03892B39F0C0901103AC
:10B8F000D0901203AA24BB24D9C08D899E89AF8918
:10B90000B88D821B930BA40BB50B8093B703909358
:10B91000B803A093B903B093BA03823070E89707D5
:10B920007FEFA7077FEFB7072CF481E090E8AFEF38
:10B93000BFEF09C08F5F9F47A040B04064F08FEF1A
:10B940009FE7A0E0B0E08093B7039093B803A09383
:10B95000B903B093BA03A090B703B090B803809135
:10B96000D001282F3327442755278091B703909182
:10B97000B803A091B903B091BA03BC01CD010E94F4
:10B98000967897FF04C0615E7F4F8F4F9F4FA5E071
:10B990009595879577956795AA95D1F76093B703A5
:10B9A0007093B8038093B9039093BA036530FEEFA8
:10B9B0007F07FFEF8F07FFEF9F072CF484E09EEFD8
:10B9C000AFEFBFEF09C0605074408040904064F01A
:10B9D00080E094E0A0E0B0E08093B7039093B803D8
:10B9E000A093B903B093BA038090B7039090B803C3
:10B9F000209140023091410237FF02C0295F3F4F42
:10BA0000F3E035952795FA95E1F74FEF22383407A3
:10BA10001CF421E83FEF05C02038310514F020E880
:10BA200030E0C901AA2797FDA095BA2F2091D20135
:10BA3000332744275527BC01CD010E94967897FFF4
:10BA400004C06D5F7F4F8F4F9F4FE2E095958795C4
:10BA500077956795EA95D1F79B015FEF61307507A0
:10BA60001CF420E03FEF06C06F3F710519F014F0A1
:10BA700020E031E08091F502807C49F0C90137FD7A
:10BA800003969C0135952795359527950DC0809196
:10BA9000980680FF09C0C90137FD07969C0143E065
:10BAA000359527954A95E1F7820E931E2091CF0197
:10BAB000222309F454C060914203709143038091A2
:10BAC00044039091450397FF04C061587F4F8F4F07
:10BAD0009F4F37E095958795779567953A95D1F77C
:10BAE0003327442755270E94967897FF04C0615E4C
:10BAF0007F4F8F4F9F4FB5E09595879577956795C9
:10BB0000BA95D1F76093B7037093B8038093B903E4
:10BB10009093BA036138AFEF7A07AFEF8A07AFEFC0
:10BB20009A072CF480E89FEFAFEFBFEF0AC06F3F9A
:10BB300071058105910569F064F080E091E0A0E075
:10BB4000B0E08093B7039093B803A093B903B09388
:10BB5000BA038091B7039091B803880E991E809123
:10BB6000CD01282F33278091A708992787FD90952D
:10BB7000289FF001299FF00D389FF00D11249F019F
:10BB8000F7FF02C021583F4F220F232F221F330BF4
:10BB9000FFEF21383F071CF420E83FEF06C02F3F9E
:10BBA000310519F014F020E031E0820E931EC4013B
:10BBB000AA2797FDA095BA2FE0901103F0901203E9
:10BBC0009701442737FD4095542FBC01CD010E94B9
:10BBD000967897FF04C061507E4F8F4F9F4FF9E0DA
:10BBE0009595879577956795FA95D1F7C61AD70AEF
:10BBF0008091E8039091E903892B09F060C01E143D
:10BC00001F040CF05CC09501B7FE03C03095219570
:10BC10003F4F2D33310540F48091EC039091ED03BB
:10BC20008C159D0574F526C02C533040E5E0369503
:10BC30002795EA95E1F72031310510F02FE030E04B
:10BC40004091EC035091ED031A141B04E4F480E1DD
:10BC500090E0821B930B489F9001499F300D589FA5
:10BC6000300D112474E0369527957A95E1F72C155F
:10BC70003D0520F58091E6019091E701C816D906AF
:10BC8000F4F06C011CC0205F3F4F8091E601909161
:10BC9000E701829FB001839F700D929F700D112468
:10BCA0009B0164E0369527956A95E1F74C155D0593
:10BCB00014F06A0104C0C216D30608F06901C60177
:10BCC000AA2797FDA095BA2F2DE0880F991FAA1FCC
:10BCD000BB1F2A95D1F79801442737FD4095542F73
:10BCE000BC01CD010E940A792093BB033093BC03B1
:10BCF0004093BD035093BE03C090BB03D090BC03E0
:10BD00008091EA039091EB039C01220F331F280FCF
:10BD1000391F2C0D3D1D37FF02C02D5F3F4FA9017C
:10BD200055954795559547955093EB034093EA03F6
:10BD300080914006282F3327220F331F220F331FF5
:10BD4000241735076CF480911B08282F3327220F06
:10BD5000331F220F331F205530404217530724F062
:10BD60003093EB032093EA038091980680FF14C080
:10BD70008091EA039091EB03A981BA818A179B070E
:10BD800024F0B093EB03A093EA03E091EA03F0916F
:10BD9000EB03FA83E98361C029813A812E193F09B7
:10BDA00037FF02C02D5F3F4F359527953595279575
:10BDB000E090EA03F090EB03E20EF31EFA82E982D0
:10BDC0004CC080914806882301F560911103709161
:10BDD000120377FF02C06D5F7F4F7595679575956C
:10BDE000679540911E0150911F0180910001282FFD
:10BDF0003327649FC001659F900D749F900D11249F
:10BE0000B9010E94D578CB0101C099279093E50133
:10BE10008093E4018091E4019091E50187349105DC
:10BE20001CF486E490E005C08639910534F086E97B
:10BE300090E09093E5018093E40129813A81309369
:10BE4000EB032093EA038091F502806C8093F50266
:10BE50008091F4028D7F8093F4028091F5029927FE
:10BE60009C012270307081FF2BC18091EE03909174
:10BE7000EF03A091F003B091F1030097A105B10584
:10BE800021F0809126038130B1F449815A81CA01A1
:10BE9000AA2797FDA095BA2F2EE0880F991FAA1FF9
:10BEA000BB1F2A95D1F78093EE039093EF03A093E5
:10BEB000F003B093F10380912603813019F482E0FE
:10BEC0008093260369817A81CB01AA2797FDA095EB
:10BED000BA2F9801442737FD4095542FBC01CD015E
:10BEE0000E949678DC01CB018093BB039093BC0346
:10BEF000A093BD03B093BE03B7FF04C08150904E22
:10BF0000AF4FBF4F7C018D01ADE015950795F794BC
:10BF1000E794AA95D1F7E092BB03F092BC0300939B
:10BF2000BD031093BE036091F6027091F7028FE09B
:10BF3000603A780750F58091EE039091EF03A0915D
:10BF4000F003B091F1039C01AD01FAE056954795DD
:10BF500037952795FA95D1F7821B930BA40BB50B58
:10BF6000A8019701E4E0220F331F441F551FEA95F3
:10BF7000D1F7820F931FA41FB51F8093EE039093F8
:10BF8000EF03A093F003B093F10360547F4118F5E1
:10BF90008091EE039091EF03A091F003B091F10333
:10BFA0009C01AD016CE056954795379527956A95AC
:10BFB000D1F7821B930BA40BB50BA8019701F2E0FC
:10BFC000220F331F441F551FFA95D1F7820F931F7D
:10BFD000A41FB51F38C0809140029091410280910A
:10BFE00040029091410297FF03C0909581959F4F29
:10BFF0008436910584F5809122039091230320914A
:10C000001E0330911F03821B930B81509F4F8F5F44
:10C01000914008F58091EE039091EF03A091F00319
:10C02000B091F1039C01AD01EEE05695479537952F
:10C030002795EA95D1F7821B930BA40BB50B8E0DB8
:10C040009F1DA01FB11F8093EE039093EF03A09359
:10C05000F003B093F1038091EE039091EF03A09170
:10C06000F003B091F1037EE0B695A795979587957B
:10C070007A95D1F79093120380931103409146066D
:10C08000442399F055279C01BA010E94D578C90133
:10C09000861B970B9093ED038093EC03260F371FBD
:10C0A0003093E7012093E6011FC01092ED03109238
:10C0B000EC038FEF93E09093E7018093E60114C0C7
:10C0C000109226031092EE031092EF031092F003E9
:10C0D0001092F103309312032093110305C0809155
:10C0E000F502806C8093F502B091E207BA8B2B2F9A
:10C0F0003327220F331F220F331F285D3F4FE98163
:10C10000FA812E173F0714F03A83298340901B08C9
:10C11000842D9927880F991F880F991F805590406B
:10C12000E980FA808E159F0514F49A8389838091A3
:10C130007802882321F48091AE088F3FA1F080918E
:10C14000F6029091F7020297C09768F409811A816C
:10C150001016110644F481E090E09093F70280936A
:10C16000F6023A83298329813A813093EC052093A2
:10C17000EB058091B3039091B403A091B503B09106
:10C18000B60342E0880F991FAA1FBB1F4A95D1F73B
:10C1900000911C0810911D08081B190B213A31054C
:10C1A0008CF0C90137FD0196959587958017910709
:10C1B0000CF48C01909581959F4F081719076CF42A
:10C1C0008C010BC00135110514F000E510E03FEFC4
:10C1D000003B130714F400EB1FEF242D3327220F2D
:10C1E000331F220F331FC90149815A81841B950BCC
:10C1F000801791070CF48C0169817A81621B730BA3
:10C20000061717070CF48B018091DD079091DE076C
:10C2100060912E0370912F03861B970B9093EC0770
:10C220008093EB07D090FA0720914A0330914B039B
:10C2300040914C0350914D03DD2041F0661A770A7E
:10C24000C301AA2797FDA095BA2F04C0AA2797FD7E
:10C25000A095BA2F280F391F4A1F5B1F20934A034E
:10C2600030934B0340934C0350934D0380914A030A
:10C2700090914B03A0914C03B0914D0381509A4F84
:10C28000A040B04064F080E09AEFA0E0B0E080937E
:10C290004A0390934B03A0934C03B0934D038091BA
:10C2A0004A0390914B03A0914C03B0914D038050F1
:10C2B0009640AF4FBF4F64F480E096E0AFEFBFEF22
:10C2C00080934A0390934B03A0934C03B0934D0388
:10C2D000C09055062091EB073091EC07F8E0FC1573
:10C2E00098F08C2D9927829F7001839FF00C929F6C
:10C2F000F00C1124C701F7FC07967C01B3E0F5941C
:10C30000E794BA95E1F712C08C2D86959927829F04
:10C31000A001839F500D929F500D1124CA0157FD1B
:10C3200003967C01F594E794F594E794A090D301EB
:10C33000B090D4019501442737FD4095542F80914A
:10C340004A0390914B03A0914C03B0914D03BC0163
:10C35000CD010E940A79E20EF31E9090BF01692D73
:10C36000772788279927980117FF04C022273327AA
:10C37000201B310B37FF02C02F5F3F4F35952795AC
:10C38000A981BA812A0F3B1F442737FD4095542FBE
:10C390000E94967897FF04C0615C7F4F8F4F9F4F3C
:10C3A000E6E09595879577956795EA95D1F79B0196
:10C3B0006E157F050CF47B01309521953F4FE216F9
:10C3C000F3060CF479018091CE079091CF0760912C
:10C3D0002C0370912D03861B970B9093CD078093B0
:10C3E000CC07209146033091470340914803509178
:10C3F0004903DD2041F0261A370AC101AA2797FD1B
:10C40000A095BA2F04C0AA2797FDA095BA2F280F90
:10C41000391F4A1F5B1F2093460330934703409305
:10C420004803509349038091460390914703A0919C
:10C430004803B091490381509A4FA040B04064F046
:10C4400080E09AEFA0E0B0E080934603909347032A
:10C45000A0934803B093490380914603909147030A
:10C46000A0914803B091490380509640AF4FBF4F11
:10C4700064F480E096E0AFEFBFEF809346039093C3
:10C480004703A0934803B09349032091CC07309110
:10C49000CD0748E04C1598F08C2D9927829FB0016C
:10C4A000839F700D929F700D1124CB0177FD07962D
:10C4B0006C0173E0D594C7947A95E1F712C0C694E5
:10C4C0008C2D9927829FD001839FB00D929FB00D34
:10C4D0001124CD01B7FD03966C01D594C794D59472
:10C4E000C7949501442737FD4095542F809146030A
:10C4F00090914703A0914803B0914903BC01CD013D
:10C500000E940A79C20ED31E692D772788279927A2
:10C51000980117FF04C022273327201B310B37FF58
:10C5200002C02F5F3F4F35952795E981FA812E0F85
:10C530003F1F442737FD4095542F0E94967897FF60
:10C5400004C0615C7F4F8F4F9F4F46E09595879564
:10C55000779567954A95D1F79B016C157D050CF48D
:10C560006B01309521953F4FC216D3060CF469013B
:10C570003CEF832E36E0932E23EBA22E26E0B22E44
:10C580009BE0592E8BEF682E87E0782ED5012C91F9
:10C5900012160CF0DEC0203419F429803A801EC037
:10C5A000E981FA81CF01AA2797FDA095BA2F3327F9
:10C5B00027FD3095432F532FBC01CD010E94967863
:10C5C00097FF04C0615C7F4F8F4F9F4FB6E09595FA
:10C5D000879577956795BA95D1F71B01F50121816C
:10C5E000203419F42E0C3F1C22C0203C19F42E18C4
:10C5F0003F081DC0C701AA2797FDA095BA2F332772
:10C6000027FD3095432F532FBC01CD010E94967812
:10C6100097FF04C0615C7F4F8F4F9F4FA6E09595B9
:10C62000879577956795AA95D1F7260E371EF50160
:10C630002281203419F42C0C3D1C22C0203C19F41A
:10C640002C183D081DC0C601AA2797FDA095BA2F3A
:10C65000332727FD3095432F532FBC01CD010E9476
:10C66000967897FF04C0615C7F4F8F4F9F4FF6E035
:10C670009595879577956795FA95D1F7260E371E8C
:10C68000F5012381203419F4200E311E22C0203CF4
:10C6900019F4201A310A1DC0C801AA2797FDA095D8
:10C6A000BA2F332727FD3095432F532FBC01CD01DF
:10C6B0000E94967897FF04C0615C7F4F8F4F9F4F19
:10C6C000E6E09595879577956795EA95D1F7260EDB
:10C6D000371ED3018D919C91821593055CF4BC01AA
:10C6E000620D731D77FF02C06F5F7F4F1B01359492
:10C6F000279404C0220C331C281A390ABA898B2FBC
:10C700009927880F991F880F991F821593054CF45C
:10C71000842D9927880F991F880F991F281639068D
:10C720000CF01C01C10137FC0396959587959595F2
:10C730008795F4018183880F991F880F991F9101B4
:10C74000281B390BC901880F8283D3012D923C929B
:10C7500003C0F401118212825A9422E030E0620E8A
:10C76000731E44E050E0A40EB51E68E070E0860E33
:10C77000971E57FE0BCFE2E1C65E0C944179809183
:10C78000010490910204A0910304B09104048093E9
:10C79000F9039093FA03A093FB03B093FC038091F9
:10C7A000FD039091FE03A091FF03B09100048093DC
:10C7B000F5039093F603A093F703B093F80308955D
:10C7C00010920C0410920B0410920A0410920904A7
:10C7D000089584B1806A84B93D9A82E58CBD1DBC00
:10C7E000459A81E080932D088AEA80933E0883E889
:10C7F00080933F088AE0809340081092420810928C
:10C80000410810924408109243081092A608109212
:10C810006208089530912D08332309F085C00DB4C6
:10C8200007FE82C084E080932E02459A2EB5809147
:10C83000180499278130910589F0823091051CF404
:10C84000892B21F03EC00297B9F03BC030936108BC
:10C85000209319042138A9F581E008C0253549F451
:10C8600080911904820F8093190482E08093180448
:10C8700028C03093180425C080916108E82FFF2755
:10C88000ED57F74F20838F5F8093610890911904D3
:10C890008032A0F0291769F480E2A3E8B8E0E3E66B
:10C8A000F8E00D9001928A95E1F781E080936208AB
:10C8B00002C0309362081092180403C0920F909344
:10C8C000190420913D08223208F028C04598000044
:10C8D0000000000000000000000000000000000058
:10C8E0000000000000000000000000000000000048
:10C8F0000000000000000000000000000000E091C7
:10C900003608F0913708E20FF11D80818EBD8091CD
:10C910005F089081890F80935F0803C081E0809356
:10C920002D082F5F20933D080895EF92FF920F93FB
:10C930001F9380914E069927880F991F880F991F82
:10C940007C010027F7FC0095102F809182039091C5
:10C950008303A0918403B0918503BC01CD01A8019C
:10C9600097010E940A7930934208209341088091F0
:10C970007A0390917B03A0917C03B0917D03BC016D
:10C98000CD01A80197010E940A79309344082093B1
:10C9900043082091230830912408409125085091A4
:10C9A0002608DA01C90103E0880F991FAA1FBB1FDF
:10C9B0000A95D1F7820F931FA41FB51F820F931FF3
:10C9C000A41FB51F20919A0130919B0140919C01B9
:10C9D00050919D01BC01CD010E940A7930934A0813
:10C9E00020934908809193039091940320914E02E3
:10C9F00030914F02821B930B9093500880934F0805
:10CA0000E0918903F0918A038091F2079091F307F6
:10CA1000BF010E94D5789B01220F331F220F331FC5
:10CA2000260F371F260F371F37FF02C02D5F3F4FDE
:10CA300035952795359527953093460820934508D9
:10CA400080911F0890912008BF010E94D5789B011A
:10CA5000220F331F220F331F260F371F260F371FBA
:10CA600037FF02C02D5F3F4F3595279535952795A8
:10CA7000309348082093470810928A031092890344
:10CA80001092F3071092F2071092200810921F08DC
:10CA90008091400899278D30910509F46CC08E3043
:10CAA00091055CF48B30910509F494C08C309105AC
:10CAB0000CF015C10A9761F0B3C18F30910509F4EC
:10CAC00087C18F3091050CF462C14097A9F1A8C1CC
:10CAD00080910A038093530880910903809354083E
:10CAE000809108038093550880910703809356082E
:10CAF000809106038093570880910503809358081E
:10CB000080910403809359088091030380935A080D
:10CB10008091F50280935B088091F502837F80937A
:10CB2000F5020E94BD2D80935C088091860380935E
:10CB30005D088091F40228C18091A8089091A9080D
:10CB400090935408809353088091AC089091AD085D
:10CB5000909356088093550880911E0190911F0173
:10CB60008093570880910001809358088091990123
:10CB70008093590855C18091820680935308809113
:10CB80008306809354088091840680935508809191
:10CB90008506809356088091860680935708809179
:10CBA0008A068093580880918B068093590880915B
:10CBB0008C0680935A0880918F0680935B08809141
:10CBC0008D0680935C0880918E0680935D0880912D
:10CBD0009006DAC0F89480913506E82FFF27EE0F13
:10CBE000FF1FE35AF84F0190F081E02DE038F10586
:10CBF0001CF0EFE7F0E006C02FEFE138F20714F485
:10CC0000E1E8FFEFE093530880913606E82FFF2715
:10CC1000EE0FFF1FE35AF84F0190F081E02DE0384E
:10CC2000F1051CF0EFE7F0E006C06FEFE138F60722
:10CC300014F4E1E8FFEFE093540880913406E82F04
:10CC4000FF27EE0FFF1FE35AF84F0190F081E02D10
:10CC5000E038F1051CF0EFE7F0E006C08FEFE138B7
:10CC6000F80714F4E1E8FFEFE093550880913306EC
:10CC7000E82FFF27EE0FFF1FE35AF84F0190F081D6
:10CC8000E02DE038F1051CF0EFE7F0E006C02FEFF3
:10CC9000E138F20714F4E1E8FFEF7894E0935608E6
:10CCA0008091310380935708809132038093580814
:10CCB00080913303809359088091340380935A08FC
:10CCC0008091350380935B088091360380935C08E4
:10CCD0008091370380935D088091380355C080911F
:10CCE0007604863018F01092760485E0809353081D
:10CCF00080919106809354088091220390912303A0
:10CD0000A0912403B0912503BC01CD0125E030E0C2
:10CD100040E050E00E940A7930935608209355086D
:10CD200080911E0390911F03A0912003B0912103D5
:10CD3000BC01CD0125E030E040E050E00E940A79DE
:10CD4000309358082093570880918706809359089C
:10CD50008091880680935A088091890680935B08A9
:10CD60008091300380935C0880915D0790915E070D
:10CD700080935D088091EB059091EC0597FD0396FB
:10CD8000959587959595879580935E0849C01092F3
:10CD9000530884E5809354081092550883E18093EA
:10CDA0005608809102018093570880915B0480931C
:10CDB000580880915C048093590880915D048093A9
:10CDC0005A0880915E0480935B0880915F0426C0BE
:10CDD000809167068093530880919706809354084A
:10CDE0008091C50180935508809160068093560814
:10CDF000809161068093570880916206809358085D
:10CE00008091C401809359088091640680935A08E8
:10CE10008091650680935B088091660680935C082C
:10CE200080916208882309F44DC18AEF8093F20152
:10CE300081E08093E1014091640850916508CA0146
:10CE400081509E4F8F5F9340B0F4209166083091DF
:10CE50006708C90181509E4F8F5F934060F48091B5
:10CE60003F0685FF08C050930C0440930B04309399
:10CE70000A042093090480916C0890916D089093A6
:10CE80000E0480930D0480916E0890916F0890932A
:10CE9000100480930F048091700890917108909312
:10CEA00012048093110480916A0890916B0821E02C
:10CEB0008936920724F49093E3018093E2018091F4
:10CEC000E2019091E3012091400330914103821BE4
:10CED000930B845E9D4F68E671E00E94D578845B79
:10CEE000904090933F0380933E03209174083091CB
:10CEF000750880912F02909130028217930720F4D9
:10CF00003093300220932F0280916308992788364E
:10CF1000910509F460C08936910524F4873691059E
:10CF200031F0D8C08936910509F47CC0D3C0809116
:10CF300076088093A308809177088093A508809154
:10CF400078088093A408809179088093A60880913E
:10CF50007A088093A70880917B088093F3018091E1
:10CF60007C0880931704809102038823F9F02091B4
:10CF70007E0830917F0837FD19C03093410320931C
:10CF8000400390916906992389F08FE0989FC00132
:10CF90001124281B390BC90188599E4F68E671E09E
:10CFA0000E94D5789093410380934003209113040D
:10CFB000309114048091800890918108280F391FC6
:10CFC00037FF02C02F5F3F4F3595279530931404EC
:10CFD000209313047FC08091760880933808809155
:10CFE0007708809339088091780880933A08809177
:10CFF000790880933B0880917A0880933C0880915F
:10D00000DB0590917B08892B8093DB0590917C0850
:10D01000909315048091DC0583709C70892B80931C
:10D02000DC0558C08091760880932E08809177089F
:10D0300080932F0880917808809330088091790838
:10D040008093310880917A0890917B0890933308FF
:10D050008093320880917C0890917D0890933508E8
:10D060008093340880917E08992787FD909590934E
:10D07000900780938F0780917F0880931903809198
:10D080008008909181089C01442737FD4095542FDA
:10D09000DA01C90163E0880F991FAA1FBB1F6A95B7
:10D0A000D1F7820F931FA41FB51F820F931FA41FD8
:10D0B000B51F80931A0390931B03A0931C03B09396
:10D0C0001D0308C010920C0410920B0410920A0465
:10D0D000109209041F910F91FF90EF900895809195
:10D0E0002D08882309F43BC045988EE398E090937F
:10D0F00037088093360890911604E92FFF27E751EF
:10D10000FE4F9F5F90931604808180934008993072
:10D1100010F01092160410922D080E94956481E080
:10D1200080933D08000000000000000000000000A7
:10D1300000000000000000000000000000000000EF
:10D1400000000000000000000000000000000000DF
:10D150000000000080913E0880935F088EBD089516
:10D1600087B18C6087B94298439810921B0480E87D
:10D170008093F50110921A048093F4010895809130
:10D1800020048150809320048F3F09F0FBC024E0ED
:10D19000209320048091F502992780739070892B49
:10D1A00021F480915C0480FF1CC08091800688235C
:10D1B00049F080912304882311F420931B0481E01B
:10D1C00080932304809181068823B9F08091240400
:10D1D000882319F484E080931A0481E08093240466
:10D1E0000CC0109223041092240480917C0680933A
:10D1F000210480917E068093220480912304882359
:10D2000009F040C080919606282F332724FF07C0DD
:10D2100080912703882319F425FD4DC04EC09091BD
:10D220007D06983F50F08091F4078D3D30F080915D
:10D23000210488230CF43FC040C0983F48F08091FF
:10D24000F4078A3028F4809121048823B4F133C094
:10D2500080911B04815080931B048F3F79F580914E
:10D26000F407815080931B048091F501813011F403
:10D2700080E801C086958093F5018091F501909139
:10D28000210417C080911B04815080931B048F3FA1
:10D29000A9F489E080931B048091F501813011F499
:10D2A00080E801C086958093F5018091F501909109
:10D2B0008006892311F0429A01C04298809124048B
:10D2C000882309F043C080919606282F332724FF36
:10D2D00007C080912703882319F426FD50C034C06D
:10D2E00090917F06983F50F080911A088D3D30F064
:10D2F0008091220488230CF442C026C0983F48F055
:10D3000080911A088A3028F4809122048823E4F05E
:10D3100036C080911A04815080931A048F3F91F592
:10D3200080911A08815080931A048091F401813011
:10D3300011F480E801C086958093F4018091F40196
:10D34000909122048923D9F44398089580911A0476
:10D35000815080931A048F3FA9F489E080931A04C6
:10D360008091F401813011F480E801C086958093AA
:10D37000F4018091F40190918106892311F0439A80
:10D380000895439808954FB724E130E0F8948091D0
:10D39000C9008F778093C9008091C9008F7B8093EB
:10D3A000C9008091C9008F7D8093C9005A9A529814
:10D3B0005B9A539A832F99278093CD002093CC00BA
:10D3C0008091C80082608093C80080E18093C9008A
:10D3D0008091CA008F778093CA008091CA008F7BAA
:10D3E0008093CA008091CA008F7D8093CA0080918B
:10D3F000CA008F7E8093CA008091CA00877F809385
:10D40000CA008091C9008B7F8093C9008091CA00B7
:10D4100084608093CA008091CA0082608093CA00B1
:10D420008091C80087FF03C08091CE00F9CF809122
:10D43000C90080688093C9004FBF0895EF92FF92A2
:10D440000F931F93CF93DF93482F00E010E080915C
:10D45000F601813061F41092F60184E48093250492
:10D460001092270410922604109228042BC1809158
:10D470002504882319F421E030E001C0980190913F
:10D480002604992371F4232B11F081E010C084E469
:10D490008093250490932704909326049093280466
:10D4A000FAC0913069F4232B09F0EBC082E080933D
:10D4B0002604809127048F5F8093270483E0E9C0CE
:10D4C0009230D1F4232B09F0DCC083E08093250453
:10D4D0004093280490912704923039F41092290443
:10D4E00047FF03C081E08093290483E080932604F2
:10D4F0009F5F90932704CFC0933009F0C2C0232BC5
:10D5000009F0BFC09093250482E0809326048091A7
:10D5100027048F5F8093270420912804822F992766
:10D52000782F6627842F9927682B792B80915906AD
:10D53000813049F47370CB018050924063E070E019
:10D540000E94D57817C0823061F47770CB0180508B
:10D55000944066E070E00E94D57826952695269541
:10D560000BC0737068567140CB0177FD0196BC010A
:10D570007595679526952695022F11270F701070C7
:10D580000F5F1F4F0D30110508F074C07801E00ED9
:10D59000F11EF701E35AF84F808191819B01281B0E
:10D5A000390BC90137FF03C0909581959F4F0697AE
:10D5B00094F480913003883C30F480913003865F8E
:10D5C0008093300308C088EC8093300380916F0013
:10D5D0008F7D80936F00F701E35AF84F808191812E
:10D5E0009C01220F331F280F391F260F371F37FFCB
:10D5F00002C02D5F3F4FE901D595C795D595C795D9
:10D60000CB0101968C179D0714F4219706C0615039
:10D610007040C617D7070CF4219680913003843BE5
:10D62000D0F0F701E35AF84F80819181FE01E81BA9
:10D63000F90BCF0163E070E00E94D578CB01880F31
:10D64000991F860F971F21E937E0E20EF31EF701BD
:10D650009183808307C021E937E0E20EF31EF701D2
:10D6600011821082000F111F035A184FF801D18345
:10D67000C08311C00231110570F081E08093F60182
:10D680000AC081E08093F6011092270410922904C9
:10D6900084E48093250480912704803198F0809160
:10D6A0002904882331F48091F601882311F48093B2
:10D6B000940110922704109229041092260484E405
:10D6C00080932504E6E0CDB7DEB70C944D79CF9377
:10D6D000FC0197FF05C0CFEFF095E195FF4F01C02A
:10D6E000C1E028E631E0CF01B9010E94D578FC0104
:10D6F0008B35910554F08B5590408A35910538F45F
:10D7000084EB90E08E1B9F0BFC0141E00DC0CF012C
:10D71000855B90408A35910518F4E45BF04003C0C6
:10D720002E1B3F0BF9014FEFEE0FFF1FE15DF54F91
:10D73000259134918C2F992787FD9095289FB001D2
:10D74000299F700D389F700D1124842F992787FD14
:10D750009095689FA001699F500D789F500D1124EE
:10D76000CA01CF9108952AE530E0281B390BC90181
:10D770000E94676B0895CF93DF9380E00E949E71B3
:10D7800080911E0190911F016AE070E00E94D5789F
:10D790009F938F9380911E0190911F016AE070E02A
:10D7A0000E94D5787F936F938DEF9AE09F938F932C
:10D7B000C1E9D1E7DF93CF93E0914204F0914304B4
:10D7C00009952DB73EB7285F3F4F2DBF8091F201DD
:10D7D0008823B9F186E00E949E7180913208909171
:10D7E00033086AE070E00E94C1787F936F938FEDF9
:10D7F00090E09F938F938091230890912408A091AB
:10D800002508B091260820919A0130919B01409102
:10D810009C0150919D01BC01CD010E940A793F936A
:10D820002F9386E09BE09F938F93DF93CF93E091BC
:10D830004204F091430409958DB79EB70A968DBFB7
:10D8400012C086E00E949E7182E19BE09F938F93BD
:10D85000DF93CF93E0914204F091430409950F9038
:10D860000F900F900F90809115048823C1F086E0EF
:10D870000E949E718091150499279F938F9389E14F
:10D880009BE09F938F93DF93CF93E0914204F091BD
:10D89000430409952DB73EB72A5F3F4F2DBF80E166
:10D8A0000E949E718091FE019091FF016CE370E0F7
:10D8B0000E94C1789F938F938091FE019091FF0108
:10D8C0006CE370E00E94C1787F936F938091AC0805
:10D8D0009091AD089F938F9384E29BE09F938F93E9
:10D8E000C1E9D1E7DF93CF93E0914204F091430483
:10D8F000099580913F062DB73EB7265F3F4F2DBF5C
:10D9000080FF29C08AE10E949E7180919901992728
:10D910009F938F938091220390912303A0912403DE
:10D92000B0912503BC01CD0124E630E040E050E099
:10D930000E940A793F932F9381E39BE09F938F93FB
:10D94000DF93CF93E0914204F091430409958DB7A2
:10D950009EB708968DBFDF91CF910895CF93DF9347
:10D9600080E00E949E7180911B07992787FD90950A
:10D970009F938F9380911307992787FD90959F938D
:10D980008F9380910B07992787FD90959F938F9395
:10D9900080910307992787FD90959F938F9388E344
:10D9A0009BE09F938F93C1E9D1E7DF93CF93E09101
:10D9B0004204F0914304099580E10E949E712DB7C5
:10D9C0003EB7245F3F4F2DBF80913B07992787FDCE
:10D9D00090959F938F9380913307992787FD90951A
:10D9E0009F938F9380912B07992787FD90959F9305
:10D9F0008F9380912307992787FD90959F938F930D
:10DA000088E49BE09F938F93DF93CF93E091420450
:10DA1000F09143040995809131062DB73EB7245FFC
:10DA20003F4F2DBF853098F480E10E949E7188E5BC
:10DA30009BE09F938F93DF93CF93E0914204F0910B
:10DA4000430409950F900F900F900F9018C08730E6
:10DA5000B0F488E10E949E718FED90E09F938F93C8
:10DA600089E69BE09F938F93DF93CF93E0914204ED
:10DA7000F091430409958DB79EB706968DBFDF914F
:10DA8000CF9108950F931F9380E00E949E712AE02A
:10DA900030E08091A8089091A908B9010E94C1784E
:10DAA0009F938F938091A8089091A908B9010E9433
:10DAB000C1787F936F9380911E0190911F01B901EE
:10DAC0000E94D5789F938F9380911E0190911F01A2
:10DAD000B9010E94D5787F936F9382E79BE09F9373
:10DAE0008F9301E911E71F930F93E0914204F091A6
:10DAF0004304099580E10E949E718DB79EB70C96F4
:10DB00008DBF8091AC089091AD089F938F938091C9
:10DB1000AA089091AB089F938F9385E89BE09F9311
:10DB20008F931F930F93E0914204F0914304099562
:10DB30008DB79EB708968DBF1F910F9108950F93D3
:10DB40001F93CF93DF938091F201C1E9D1E788233E
:10DB500009F478C080E00E949E7180912F08992777
:10DB60009F938F938091310899279F938F9381E999
:10DB70009BE09F938F938E01DF93CF93E0914204BC
:10DB8000F091430409958DB79EB708968DBF80919B
:10DB90003008833031F48CE00E949E7180EA9BE073
:10DBA00005C08CE00E949E7185EA9BE09F938F9355
:10DBB000DF93CF93E0914204F091430409950F90D5
:10DBC0000F900F900F9080912E0881FF12C08CE073
:10DBD0000E949E718AEA9BE09F938F931F930F93FD
:10DBE000E0914204F091430409950F900F900F903B
:10DBF0000F9080E10E949E718FED90E09F938F9334
:10DC000080913408909135089F938F9380913208CA
:10DC1000909133086AE070E00E94C1787F936F931F
:10DC20008FEA9BE09F938F9381E991E79F938F9376
:10DC3000E0914204F091430409958DB79EB70A968E
:10DC40008DBF12C082E00E949E718FEB9BE09F937C
:10DC50008F93DF93CF93E0914204F09143040995B1
:10DC60000F900F900F900F90DF91CF911F910F9118
:10DC70000895CF93C82F20912A0420932B0499272D
:10DC80008F32910509F1803391051CF44F97A1F073
:10DC90002CC08F34910501F18F38910531F5222385
:10DCA00019F481E090E038C086E0289FF00111244B
:10DCB000EB51F54F849117C086E0289FF0011124A5
:10DCC000EA51F54F84910FC086E0289FF00111249E
:10DCD000E951F54F849107C086E0289FF001112497
:10DCE000E851F54F849180932A0490912A04809101
:10DCF0002B049813C0E00E94A47190912A0486E03E
:10DD0000989FF0011124E751F54F259134918C2F04
:10DD1000F901099580E090E0CF9108951092A9084B
:10DD20001092A8081092AD081092AC081092AB089F
:10DD30001092AA081092AE088AE090E00E94211783
:10DD400090932D0480932C040895CF93DF938091BA
:10DD50002C0490912D040E942A17882309F4AFC047
:10DD600080912C0490912D040A9690932D04809319
:10DD70002C04E0E0F0E09F0190E05FEFACEFB6E054
:10DD80004BE0ED018B8187FF0BC09F5F8D81E80F1A
:10DD9000F11D8981280F311D8E81851708F4582FB8
:10DDA0004150189647FFEDCF5093AE08232B41F515
:10DDB0002091320430913304409134045091350461
:10DDC000BB27A52F942F832F909331048093300489
:10DDD000AA27BB27281B390B4A0B5B0BCF01AA27AD
:10DDE000BB27280F391F4A1F5B1F20933204309333
:10DDF00033044093340450933504E5E0F0E013C05D
:10DE000020913004309131042E173F0718F4E21BA3
:10DE1000F30B02C0E0E0F0E0892F9927880F991FEB
:10DE2000E80FF91F3596F093A908E093A808EF3F93
:10DE3000F10578F480911E0190911F018E9F900151
:10DE40008F9F300D9E9F300D1124C90164E670E054
:10DE500013C0CF01969587959695879520911E01C1
:10DE600030911F01289FA001299F500D389F500D10
:10DE70001124CA0169E170E00E94C1787093AB0877
:10DE80006093AA0820912E0430912F042E0F3F1F7B
:10DE900030932F0420932E045EE02131350778F073
:10DEA0008091AC089091AD0801969093AD08809355
:10DEB000AC0820513E4030932F0420932E04DF9174
:10DEC000CF910895002422273327442751E0BB2710
:10DED000EE27FF27A0E1660F771F881F991F001C00
:10DEE000221F331F441F660F771F881F991F001CB6
:10DEF000221F331F441F2AF4050E2B1F3E1F4F1FE6
:10DF000004C0051A2B0B3E0B4F0B550FBB1FEE1F0A
:10DF1000587F556047FD5250AA95E9F6E695B795AA
:10DF20005795E695B7955795852F9B2F08952227EE
:10DF3000332741E0552768E0880F991F221F331FC0
:10DF4000880F991F221F331F1AF4240F351F02C098
:10DF5000241B350B440F551F487F456037FD425049
:10DF60006A9551F75695479556954795842F08958C
:10DF7000AA2797FF04C0809590958A1F9A1F77FF64
:10DF800004C0609570956A1F7A1F669F9001779F05
:10DF9000A001679F300D411D5A1F300D411D5A1FB2
:10DFA000889FF001999F2E0F3F1F401D511D899F93
:10DFB000300D411D5A1F300D411D5A1FCA01B901B4
:10DFC000112480CF4FB720E430E0F8948091C9004D
:10DFD0008F778093C9008091C9008F7B8093C9009F
:10DFE0008091C9008F7D8093C9005A9A52985B9A9C
:10DFF000539A832F99278093CD002093CC00809152
:10E00000C80082608093C80088E18093C900809135
:10E01000CA008F778093CA008091CA008F7B80935B
:10E02000CA008091CA008F7D8093CA008091CA0087
:10E030008F7E8093CA008091CA00877F8093CA0038
:10E040008091C9008B7F8093C9008091CA00846051
:10E050008093CA008091CA0082608093CA00809138
:10E06000C80087FF03C08091CE00F9CF8091C9001E
:10E0700080688093C9004FBF08950F931F93CF937B
:10E08000DF93482F4F5F893108F08BC080915C0788
:10E09000841720F44F5F40935C074150CB018353BA
:10E0A0009B4268E170E00E94D578A42FBB27FD0158
:10E0B000EA0FFB1FE35AF84F808191819B01281BD7
:10E0C000390BC90137FF03C0909581959F4F069783
:10E0D00094F480913003883C30F480913003865F63
:10E0E0008093300308C088EC8093300380916F00E8
:10E0F0008F7D80936F00FD01EA0FFB1FE35AF84FFD
:10E10000808191819C01220F331F280F391F260F18
:10E11000371F37FF02C02D5F3F4FE901D595C795E7
:10E12000D595C795CB0101968C179D0714F42197BF
:10E1300006C061507040C617D7070CF42196809135
:10E140003003843BD8F08D010A0F1B1FF801E35AFE
:10E15000F84F80819181FE01E81BF90BCF0163E04C
:10E1600070E00E94D578CB01880F991F860F971F0A
:10E170000F56184FF8019183808307C0AA0FBB1F69
:10E18000AF56B84F11961C921E92E42FFF27EE0F48
:10E19000FF1FE35AF84FD183C083443011F410922B
:10E1A0009401DF91CF911F910F910895CF93DF9349
:10E1B0002091AF08822F9927807F9070409709F0B7
:10E1C0006CC02F3109F046C08091B00880933A04AA
:10E1D0002091B20820933C048091B30880933B04C3
:10E1E000822F992790935E0780935D07222309F081
:10E1F00054C080913306282F3327220F331FF90193
:10E20000EF56F84F1182108280913406A82FBB2759
:10E21000AA0FBB1FFD01EF56F84F118210828091AB
:10E220003606E82FFF27EE0FFF1FCF018F56984FBE
:10E23000EC0119821882235A384FE9011982188299
:10E24000A35AB84F11961C921E92E35AF84F1182AE
:10E25000108223C0C22FCF70CA30F8F48091B0086A
:10E260008093D9088091B1088093D8088091B20832
:10E270008093DB088091B3088093DA086091D80816
:10E280007091D9088C2F0E943D706091DA087091CE
:10E29000DB088C2F8F5F0E943D70DF91CF91089536
:10E2A000CF93C82F8F3F49F480913D048F3F29F4CD
:10E2B00010923F0410923E0432C020913F0422236A
:10E2C00039F4CF3111F485E001C084E0809340043B
:10E2D0008091400490913E048217A0F4892F80958C
:10E2E00080933E048F3F19F48EEF80933E0480911B
:10E2F0003E04C81711F40E94D67010923F04109289
:10E300003E040BC0E22FFF27E155F74FC0832F5F7C
:10E3100020933F049C0F90933E04C0933D04CF9103
:10E32000089590913904933240F4E92FFF27EB547C
:10E33000F74F80839F5F909339040895833218F4D8
:10E340008D5F80933904089590E2E8EBF8E08FE167
:10E350009193815087FFFCCF0895CF93CFB723E0EF
:10E3600031E0F8948091C9008F778093C900809143
:10E37000C9008F7B8093C9008091C9008F7D8093F5
:10E38000C9005A9A52985B9A539A832F992780937F
:10E39000CD002093CC008091C80082608093C8009B
:10E3A00088E18093C9008091CA008F778093CA006A
:10E3B0008091CA008F7B8093CA008091CA008062DE
:10E3C0008093CA008091CA0080618093CA008091C6
:10E3D000CA0088608093CA008091C90084608093DD
:10E3E000C9008091CA0084608093CA008091CA00ED
:10E3F00082608093CA008091C80087FF03C080912B
:10E40000CE00F9CF8091C90080688093C9008091C7
:10E41000C90080648093C9000E94A471CFBFCF91CE
:10E420000895282F99278F709070892B31F42095AB
:10E4300080913804822B8093380408958091F901EB
:10E44000882309F449C08091F50285FD04C08091BC
:10E45000FC01882371F082E98093B50883E2809300
:10E46000B6088091FC01882309F485E58093B708FC
:10E4700002C08093B5088091FA018F3071F48091C9
:10E4800038040E94396E882341F081E98093B508F1
:10E490008093B60881E38093B7081092F9018091C8
:10E4A000C80085FFFCCF8091C9008F7E8093C90092
:10E4B0008091C9008E7F8093C9008091B508882320
:10E4C00011F48EEF01C08EE78093CE008091380466
:10E4D0008093FA011092380408951F920F920FB69C
:10E4E0000F9211248F939F93EF93FF939091F901D3
:10E4F000992309F040C080914104882361F4809100
:10E50000B508882311F483E003C0813999F481E0D0
:10E51000809341040FC0833099F48091B50888231B
:10E5200049F09093B5088091C9008E7F8093C9000F
:10E530008EEF1EC08091C90081608093C9000EC01B
:10E54000833261F48091C9008E7F8093C9008FEF80
:10E550008093CE0081E08093F90114C08091410442
:10E56000E82FFF27EB54F74F8F5F809341048081A2
:10E570008093CE0007C0109241048091C900806151
:10E580008093C900FF91EF919F918F910F900FBEE3
:10E590000F901F901895EF92FF920F931F93CF93B8
:10E5A000DF937C018B01EA01452B39F0F801819161
:10E5B0008F01F70109952197C9F7E6E0CDB7DEB7DE
:10E5C0000C944D79EF92FF920F931F93CF93DF93AB
:10E5D0007C018B01EA01452B41F0F8010F5F1F4FD1
:10E5E0008491F70109952197C1F7E6E0CDB7DEB731
:10E5F0000C944D790F931F93CF938C01C62F161651
:10E6000034F480E2F8010995C1501C16D4F3CF917F
:10E610001F910F9108950F931F93CF938C01C62FD5
:10E62000161634F480E3F8010995C1501C16D4F392
:10E63000CF911F910F910895A5E3B0E0E2E2F3E7D7
:10E640000C9425792E96EEADFFAD2E978824992453
:10E65000540180913704882321F42C961FAE1EAEFE
:10E660002C975EE4452E512C4C0E5D1E6F01B601B9
:10E6700005C0153239F00894C11CD11CF601149163
:10E680001123B9F7A601461B570B31F02C968EAD1E
:10E690009FAD2C970E94E272112309F46AC208947C
:10E6A000C11CD11CFF24FDA6FCA64FEFE42EF9A649
:10E6B000F6010894C11CD11C1491153721F0812F4B
:10E6C00080628837B1F4F0FE0AC0F20124E030E045
:10E6D000420E531E80809180A280B3800AC0F20156
:10E6E00042E050E0440E551E808191814C01AA24E5
:10E6F000BB24103221F489A58823D1F61DC0133222
:10E7000019F458E0F52AD4CF1A3211F01D3291F4E1
:10E710001A3259F4F20182E090E0480E591EE0816D
:10E72000ECA7EE232CF6E195ECA790E1F92AAFEDEA
:10E73000FA22BECF1B3211F419A7BACF1E32C1F58F
:10E74000F6010894C11CD11C14911A3279F4F2011B
:10E7500022E030E0420E531E408151813FEF4F3F97
:10E76000530714F44FEF5FEFE42EA2CF40E050E0E8
:10E77000812F80538A30A0F4CA0133E0880F991F9B
:10E780003A95E1F7840F951F480F591F410F511D0E
:10E7900040535040F6010894C11CD11C1491E8CF9D
:10E7A0008FEF4F3F580714F44FEF5FEFE42E85CF04
:10E7B000103329F4F4FC7CCF90E2F92A79CF812F31
:10E7C00081538930D8F440E050E0CA0123E0880F3B
:10E7D000991F2A95E1F7840F951F480F591F410F84
:10E7E000511D40535040F6010894C11CD11C149196
:10E7F000812F80538A3048F34CA75FCF183619F425
:10E80000A4E0FA2A55CF1C3619F4B1E0FB2A50CF08
:10E81000133661F43E010894611C711CF20122E080
:10E8200030E0420E531E808189833CC1143421F0B4
:10E83000143611F0193651F5143411F431E0F32A7D
:10E84000F0FE0AC0F20144E050E0440E551E808004
:10E850009180A280B3800CC0F20182E090E0480E6B
:10E86000591E808191814C01AA2497FCA094BA2C56
:10E87000B7FE0AC0B094A09490948094811C911C1F
:10E88000A11CB11C8DE289A70AE06FC01F3411F0F2
:10E890001F3631F41F3411F491E0F92A08E064C006
:10E8A000103779F4F201A2E0B0E04A0E5B1E8081DD
:10E8B00091814C01AA24BB2400E1B0E4FB2A18E7B3
:10E8C00053C01337C1F5F20122E030E0420E531E6F
:10E8D000608071806114710489F43E010894611CA8
:10E8E000711C88E289838EE6F301818385E78B833F
:10E8F0008CE68C838D8389E28E831F82E7FC13C0B4
:10E900008E2D992787FD9095AC0160E070E0C301E2
:10E910000E94D177009729F0382E3618E3140CF0B6
:10E92000C3C03E2CC1C0F30101900020E9F731972C
:10E930003E2E3618B9C0153511F0153731F415359E
:10E9400011F4F1E0FF2A0AE00FC0183519F018376A
:10E9500009F0A0C000E1F3FE07C081149104A104F6
:10E96000B10411F020E4F22A19A6EDA6E7FC02C0DA
:10E970003FEDF32289E2682E712C6C0E7D1E81140E
:10E980009104A104B10421F44DA5442309F47BC0F2
:10E99000802F9927AA27BB278EA79FA7A8ABB9AB23
:10E9A000202E332490E0891690E0990691E0A90684
:10E9B00090E0B90648F0C501B4012EA53FA548A9CD
:10E9C00059A90E94E87817C0AFEF8A169104A104F4
:10E9D000B10449F040F0C401B1010E94C1789B012B
:10E9E0004427552708C0882D602F0E94B578282F0E
:10E9F0003327442755272AAB3BAB4CAB5DAB0A30E2
:10EA000059F48AA9880F880F880F9AA9990F890F3E
:10EA1000382D381B832F10C0003139F48AA9829514
:10EA2000807F482D481B842F07C08AA9880F880F34
:10EA3000880F582D581B852F90E02EA53FA548A97B
:10EA400059A982169306A406B50608F091E08AA893
:10EA50009BA8ACA8BDA88A3010F4805D04C0895A78
:10EA6000183509F48F7DD3018E933D01992309F068
:10EA700099CF083041F4F3FE06C0803321F080E3E3
:10EA8000FD0182933F01CE010196382E3618F8E23F
:10EA90003F0E0BC0112309F46CC03E010894611CA9
:10EAA000711C1983B1E03B2E19A6032D2DA4231848
:10EAB00027FC222489A5882311F00F5F02C0F6FCF1
:10EAC0000E5F020DEF2CFF24C70180739070892B1D
:10EAD00049F48CA5801B682F2C968EAD9FAD2C978A
:10EAE0000E94FA7289A5882331F041E050E0BE010E
:10EAF000675D7F4F0AC0E6FE0EC080E38AA71BA7B2
:10EB000042E050E0BE01665D7F4F2C968EAD9FAD1A
:10EB10002C970E94CB72C70180739070809749F444
:10EB20008CA5801B682F2C968EAD9FAD2C970E94D4
:10EB30000B73622D2C968EAD9FAD2C970E940B739C
:10EB4000832D992787FD9095AC01B3012C968EAD4E
:10EB50009FAD2C970E94CB72E4FE89CD2CA5201B83
:10EB60002CA7622F2C968EAD9FAD2C970E94FA7227
:10EB70007ECDE2E1CB5C0C9441792FB740E0F89474
:10EB8000E0E0F0E081E2809357009491E2E0F0E071
:10EB9000809357003491E4E0F0E080935700849133
:10EBA0002FBF9E3199F4363941F4893011F441E098
:10EBB0000DC08A3059F442E009C0373939F4863043
:10EBC00011F443E003C0853009F444E0842F992711
:10EBD00008959FB7F8948091C900877F8093C900FA
:10EBE0008091C9008F7E8093C9008091C9008F7782
:10EBF0008093C9008091C9008F7B8093C900809168
:10EC0000C9008F7D8093C90052985A9A53985B9A95
:10EC10009FBF08951F93CF93DF93182F80913704E0
:10EC2000882309F48DC08091F801181709F488C071
:10EC300080913604882321F40E94BD7580933604A8
:10EC400088EB9CE09F938F93CBEFD2E1DF93CF9340
:10EC5000E0914204F091430409950F900F900F90BA
:10EC60000F90812F99278230910501F18330910512
:10EC70002CF4009761F0019769F024C0843091056D
:10EC8000D9F084309105ACF00597C9F01BC088EA33
:10EC90009CE002C086E99CE09F938F93DF93CF9323
:10ECA000E0914204F0914304099518C08DE79CE07F
:10ECB000F3CF8AE59CE0F0CF8CE49CE0EDCF84E4D8
:10ECC0009CE0EACF85EC9CE09F938F93DF93CF93FA
:10ECD000E0914204F0914304099510E00F900F90E9
:10ECE0000F900F9080913604843011F0823099F4A7
:10ECF0000E94E975812F8150833018F40E94C36906
:10ED00001DC0143019F40E94AD7118C01530B1F453
:10ED10000E94E26F13C0112389F08BED9CE09F935A
:10ED20008F938BEF92E19F938F93E0914204F09148
:10ED3000430409950F900F900F900F901093F801D6
:10ED4000DF91CF911F9108950F931F9381E08093DE
:10ED500037044091F701E4EFFBE020E030E05FE4AE
:10ED6000849199272F5F3F4F829FB001839F700D41
:10ED7000929F700D112446275150319657FFF0CFC6
:10ED80004093F701ECECFBE020E030E057E28491A7
:10ED900099272F5F3F4F829FB001839F700D929FF5
:10EDA000700D112446275150319657FFF0CF4093F4
:10EDB000F70180913604882321F40E94BD75809369
:10EDC00036048091F701833459F088E190E029E21C
:10EDD0000FB6F894A895809360000FBE2093600052
:10EDE0008CE193E7909343048093420486EF9CE088
:10EDF0009F938F930BEF12E11F930F93E0914204C7
:10EE0000F091430409950F900F900F900F9081E6B9
:10EE100090E09F938F9384E590E09F938F931F9250
:10EE20001F92809102016AE00E94B578892F99278C
:10EE30009F938F93809102010E94B57899279F93A9
:10EE40008F938CE19DE09F938F931F930F93E0919D
:10EE50004204F0914304099584EF9BE09F938F93C4
:10EE60001F930F93E0914204F091430409958CECB9
:10EE70009BE09F938F931F930F93E0914204F09137
:10EE8000430409958DB79EB746968DBF80E59DE0FA
:10EE90009F938F931F930F93E0914204F09143044B
:10EEA000099583EC8093810080916F00806280934C
:10EEB0006F000F900F900F900F901F910F9108957A
:10EEC00080913704882361F08091F801843011F437
:10EED0000E941E728091F701833411F01092370462
:10EEE00008951F920F920FB60F9211242F933F9304
:10EEF0004F935F936F937F938F939F93AF93BF9342
:10EF0000EF93FF932091CE00809105028823B1F00A
:10EF10002093C60080910502823029F52F3F19F514
:10EF20008FEF94E3ACE0B0E0C297A109B109B7FF5D
:10EF3000FBCF809185048093CE0015C09091F8019D
:10EF4000892F8150833020F4822F0E941E6A0BC0CB
:10EF5000943021F4822F0E94117205C0953019F46B
:10EF6000822F0E945071FF91EF91BF91AF919F91BD
:10EF70008F917F916F915F914F913F912F910F9062
:10EF80000FBE0F901F901895FB01DC0140FF05C0DC
:10EF900002C005900D9205900D9242505040C8F766
:10EFA0000895FC014150504030F001900616D1F711
:10EFB0003197CF0108958827992708955058192E21
:10EFC00084D001D06AC0BA17620773078407950717
:10EFD000B1F188F40EF410940B2EBA2FA02D062E4A
:10EFE000622F202D072E732F302D082E842F402DB9
:10EFF000092E952F502DFF275523B9F0591B49F0A5
:10F00000573E98F0469537952795A795F04053952C
:10F01000C9F776F0BA0F621F731F841F30F487950B
:10F0200077956795B795F040939517FA0F2E089549
:10F03000BF1BBB27BA0B620B730B840BF6CFDEF63C
:10F0400070C097FB4ED09F3738F0FEE9F91B982F20
:10F05000872F762F6B2F05C061C096958795779582
:10F060006795F150D0F73EF4909580957095619535
:10F070007F4F8F4F9F4F0895E89403C097FB0EF486
:10F08000F3DFB62F672F782F892F9EE9002405C064
:10F090009A95BB0F661F771F881F11249923A1F033
:10F0A0008823B2F79F3F59F0BB0F48F421F40020AA
:10F0B00011F460FF04C06F5F7F4F8F4F9F4F881F19
:10F0C0009795879597F9089529C0052E092607FA7F
:10F0D000440F551F5F3F79F0AA27A51708F051E0AC
:10F0E0004795880F991F9F3F31F0BB27B91708F04C
:10F0F00091E0879508959F919F91112414C097FBEB
:10F10000880F991F9F3F31F0BB27B91708F091E096
:10F11000879508959F919F91112405C066277727B1
:10F120008827992708959FEF80EC0895629FD0016A
:10F13000739FF001829FE00DF11D649FE00DF11DB2
:10F14000929FF00D839FF00D749FF00D659FF00D61
:10F150009927729FB00DE11DF91F639FB00DE11D4E
:10F16000F91FBD01CF0111240895991B79E004C056
:10F17000991F961708F0961B881F7A95C9F78095F6
:10F180000895AA1BBB1B51E107C0AA1FBB1FA617EE
:10F19000B70710F0A61BB70B881F991F5A95A9F740
:10F1A00080959095BC01CD01089597FB092E072607
:10F1B0000AD077FD04D0E5DF06D000201AF4709560
:10F1C00061957F4F0895F6F7909581959F4F08952B
:10F1D000A1E21A2EAA1BBB1BFD010DC0AA1FBB1F5B
:10F1E000EE1FFF1FA217B307E407F50720F0A21BCD
:10F1F000B30BE40BF50B661F771F881F991F1A943A
:10F2000069F760957095809590959B01AC01BD0163
:10F21000CF01089597FB092E05260ED057FD04D087
:10F22000D7DF0AD0001C38F45095409530952195D1
:10F230003F4F4F4F5F4F0895F6F79095809570952B
:10F2400061957F4F8F4F9F4F08952F923F924F921E
:10F250005F926F927F928F929F92AF92BF92CF9266
:10F26000DF92EF92FF920F931F93CF93DF93CDB76F
:10F27000DEB7CA1BDB0B0FB6F894DEBF0FBECDBFE7
:10F2800009942A88398848885F846E847D848C84B8
:10F290009B84AA84B984C884DF80EE80FD800C81C1
:10F2A0001B81AA81B981CE0FD11D0FB6F894DEBFA4
:10F2B0000FBECDBFED010895EE0FFF1F0590F49135
:10F2C000E02D0994F999FECFB2BDA1BDF89A11962F
:10F2D00000B40895F7DF01921A94E1F70895F2DF80
:10F2E000E02DF0DFF02D0895F999FECFB2BDA1BD5C
:10F2F00000BC11960FB6F894FA9AF99A0FBE0895C9
:10F30000F3DF012CF1DF112408950190EDDF1A9451
:04F31000E1F7089584
:10F314005E010A010164FF01FFFFC01FC01F01015C
:10F3240001737373FF03007D0000C409C409640002
:10F334001148656C6C6F20576F726C64000000009C
:10F3440000000000000000000000000000000000B9
:10F3540000000000000000000000000000000000A9
:10F364000000000000000000000000000000000099
:10F374000000000000000000000000000000000089
:10F384000053706F727400004E6F726D616C0000F8
:10F39400426567696E6E6572000051756164726FD3
:10F3A400000064000101000300200B050000ECFFD5
:10F3B40000020406070808080706040200FEFCFA17
:10F3C400F9F8F8F8F9FAFCFE0002040607080864E4
:10F3D40040415A4664640A02969696960840403A1A
:10F3E40010FB3038013290D0030090D0030032007B
:10F3F4002064FFFF7800FF03640B0A0D0B0C0E0B57
:0CF404000F10FA2001010170FF010F0041
:00000001FF
